:100000000C94320B0C94630B0C94630B0C94630BE9
:100010000C94630B0C94630B0C94630B0C94630BA8
:100020000C94630B0C94630B0C94630B0C94630B98
:100030000C94630B0C94B4120C94630B0C94630B30
:100040000C94630B0C94630B0C94630B0C94630B78
:100050000C94630B0C94630B0C94630B0C9478AAB4
:100060000C94630B0C94089D0C94DE9C0C94630B15
:100070000C94630B0C94630B0C94630B0C94630B48
:100080000C94630B0C94630B0C94630B0C94630B38
:100090000C94B49C0C948A9C0C94630B0C943F14A9
:1000A0000C94630B0C94630B0C94630B0C94630B18
:1000B0000C94630B0C94630B0C94630B0C94630B08
:1000C0000C94630B0C94630B0C94630B0C94609C6A
:1000D0000C94369C0C94630B0C940C9C0C94E29B3B
:1000E0000C94630B084AD73B3BCE016E84BCBFFD2A
:1000F000C12F3D6C74319ABD56833DDA3D00C77FF8
:1001000011BED9E4BB4C3E916BAAAABE0000008090
:100110003F07634236B79BD8A71A39685618AEBA5C
:10012000AB558C1D3CB7CC5763BD6DEDFD753EF6F0
:10013000177231BF000000803F08000000BE92240B
:1001400049123EABAAAA2ABECDCCCC4C3E00000040
:1001500080BEABAAAAAA3E00000000BF000000803B
:100160003F0000000000084178D3BB4387D1133D16
:10017000190E3CC3BD4282AD2B3E68EC8276BED9DF
:100180008FE1A93E4C80EFFFBE01C4FF7F3F00001E
:10019000000000000C94AD0B0C94A08A0C94778A9C
:1001A0000C948C8A0C940A8A0C94C48B0C94FD0BCE
:1001B0000C94A48A0C946F860C94650B0C94A88AFA
:1001C0000C94040D0C94AE8A0C9469740C940488FD
:1001D0000C94857C0C94FD730C940F740C94597FD3
:1001E0000C949F880C9428750C9419850C945D7B55
:1001F0000C94EF880C9472740C94B4870C94FC8764
:100200000C94888A0C9445890C9458740C94487307
:100210000C9459890C948F830C94AD8A0C94C67FEE
:100220000C946E870C94DF730C946D8A0C94F473A9
:100230000C94010D0C94F0880C94CF780C949A8A4D
:100240000C94AB0B0C947B8A0C9420740C94738AE2
:100250000C94B28A0C94C1760C94CF870C94BD0B8D
:100260000C947B740C9436890C94968A0C94828A34
:100270000C949D120C94AE7F0C94AA7A0C94BD89B8
:100280000C94C2AB0C94AE0B0C94AF870C94B6815B
:100290000C94928A0C94D00B0C94C37F0C945C7ECB
:1002A0000C94B9870C944D8B0C94E5850C9467865F
:1002B0000C9473830C9406740C94D6780C946C0B89
:1002C0000C9447770C942F0C0C94B68A0C94080D60
:1002D0000C9456760C941F750C9429740C94AC0BEA
:1002E0000C9431750C9467890C9484740C947F8AF7
:1002F0000C940A800C942C0C0C94AD840C94078004
:100300000C9407AB4E414E494E495459494E46CD87
:10031000CCCC3D0AD7233C17B7D13877CC2B3295BC
:1003200095E6241FB14F0A000020410000C842009A
:10033000401C4620BCBE4CCA1B0E5AAEC59D740064
:10034000407A10F35A00A0724E18090010A5D4E8A4
:100350000000E87648170000E40B54020000CA9A37
:100360003B000000E1F50500008096980000004089
:10037000420F000000A086010000001027000000CE
:1003800000E803000000006400000000000A000014
:100390000000000100000000002C76D888DC674FC8
:1003A0000823DFC1DFAE59E1B1B796E5E3E453C6F8
:1003B0003AE651997696E8E6C28426EB898C9B62F0
:1003C000ED407C6FFCEFBC9C9F40F2BAA56FA5F49A
:1003D00090055A2AF75C936B6CF9676DC11BFCE0C2
:1003E000E40D47FEF520E6B500D0ED902E03009415
:1003F0003577050080841E080000204E0A000000AA
:10040000C80C333333330F986E12831141EF8D21B3
:1004100014893BE65516CFFEE6DB18D1844B381B1A
:10042000F77C1D901DA4BBE424203284725E2281DF
:1004300000C9F124ECA1E53D274E6F2073656E7372
:100440006F72210049522054656D70657261747538
:100450007265004D6561737572696E672E2E004E70
:100460006F2073656E736F723F0049522054656D43
:100470007065726174757265004D6561737572693E
:100480006E672E2E004E6F2053656E736F722100C3
:100490004E6F20445320546865726D6F6D657465AE
:1004A000722100445320546865726D2E004D6F74A4
:1004B000696F6E0046696E64696E672057694669A8
:1004C000204950007365703D006976616C3D006E97
:1004D000697465723D00230043616C2E204661699A
:1004E0006C65640043616C2E20446F6E65004E6F36
:1004F000206E6565642100496E76616C69642050E8
:1005000028506129005365614C6576656C20502840
:100510005061293A0043616C6962726174652050D0
:10052000004169722054656D70286F43293A004379
:10053000616C2E204D6F74696F6E004453542054CB
:10054000656D702073656E736F72004375727265AE
:100550006E742073656E736F72004F322073656E18
:10056000736F720055562073656E736F720043612E
:100570006C696272617465004661696C65640054FF
:10058000422063616C2E20646F6E6500557070654B
:1005900072204C696D69743A3E004C6F7765722029
:1005A0004C696D69743A3E0054757262696469748D
:1005B00079004661696C65640070482063616C2E47
:1005C00020646F6E6500704831302050726573731F
:1005D00020420070483420507265737320410043FC
:1005E000616C696272617465004E45543D426C7580
:1005F00065746F6F7468204C45004E45543D426CE5
:100600007565746F6F7468004E45543D576946694F
:100610000053657474696E67204661696C65640097
:1006200053657474696E6720446F6E65004368613A
:100630006E6765204E6574776F726B3E00547970FB
:10064000653A0042542F57694669204E6574776FAA
:10065000726B004368616E67652053656E736F72DD
:100660003E0043757272656E742053656E736F72CF
:10067000004F7468657200496E642E20342D32304C
:100680006D4100414353373132203C33304100410A
:100690004353373132203C323041004143533731EC
:1006A00032203C3541003E4D617820566F6C743AE3
:1006B0003E004368616E676520766F6C74616765A4
:1006C0003E00547970652000566F6C746167652038
:1006D00053656E736F72004368616E67652074794D
:1006E000706520746F0053656E736F723D4448549B
:1006F0000054656D702048756D69646974790020D7
:1007000028303D6175746F3B313D616363656C3BBF
:10071000323D696E636C20616E676C652900234110
:100720003D00556E6B6E6F776E00496E6475737425
:100730007269616C20342D32306D41004143533772
:100740003132204D61783D35410023437572726529
:100750006E742073656E736F723A00696E70757493
:100760002044535463616C6962726174653A00207D
:10077000766F6C746167653D0023547572626964BD
:10078000697479205570706572204C696D69743A8E
:10079000200020766F6C746167653D00235475728C
:1007A000626964697479204C6F776572204C696D59
:1007B00069743A20002354757262696469747920FF
:1007C0004C6F776572204C696D69742056696E664E
:1007D0003A20004D61782072616E67653D002356B6
:1007E0006F6C746167652073656E736F723A003465
:1007F0002D32306D4100414353373132204D617805
:100800003D00414353373132204D61783D35410041
:100810002343757272656E742073656E736F723ADE
:100820000023445320546865726D6F6D6574657262
:100830002063616C6962726174656420666F722006
:10084000230044535400234E6F206E65656420746A
:100850006F2063616C696272617465206375727286
:10086000656E742073656E736F722100234143536C
:100870003731322063757272656E742073656E73E2
:100880006F72206F666673657420563D002355565F
:10089000207A65726F20766F6C74616765203D0009
:1008A00055565A00234F3220766F6C253D00234F5A
:1008B000322063616C6962726174696F6E3A200004
:1008C00023566F6C746167652870483D3130293A52
:1008D0000023566F6C746167652870483D34293A6F
:1008E00000504834005554454D503D004448543D57
:1008F00000413D002354696D65206475726174691F
:100900006F6E3D002354696D6520696E7465727663
:10091000616C3D00576946692049503A00234D53A8
:1009200020456E61626C656400234D5320446973F9
:1009300061626C656400235265737420706172613A
:100940006D657465727320746F2064656661756C83
:10095000742076616C756573004C6F6767657220F3
:100960004E616D653A2000697465726174696F6EDD
:100970003D0073656E736F72233D0043757272653F
:100980006E74207374617475733A206379636C6557
:100990003D006E6379636C653D006E73656E736FC9
:1009A00072733D006D61786E73656E736F72733D27
:1009B00000656E61626C65643D00234D756C746901
:1009C00073656E736F7273206D6561737572656D9B
:1009D000656E742073657474696E67733A0023538F
:1009E000657474696E6773206F6620616C6C207328
:1009F000656E736F72733A002353697A65206F6670
:100A000020686561646572202B20616C6C207365C1
:100A10006E736F72733A20002353697A65206F6694
:100A2000206865616465723A20004F6666206169DE
:100A3000722D636F6E6421004974277320746F6F89
:100A400020636F6F6C210054656D702069732066A0
:100A5000696E6521004973206169722D636F6E6450
:100A6000206F6E3F0049742773207175697465208B
:100A7000686F742100497427732076657279206845
:100A80006F742120004F6666206169722D636F6E5E
:100A90006421004974277320746F6F20636F6F6C3B
:100AA000210054656D702069732066696E652100B0
:100AB0004973206169722D636F6E64206F6E3F0011
:100AC0004974277320717569746520686F742100FB
:100AD00049742773207665727920686F74210054F9
:100AE000656D702048756D696469747900232061B3
:100AF0006E6420726561647920746F20757365215E
:100B000000206D6F62696C65206C6F67676572208D
:100B100073746172746564200043616C6962726110
:100B200074696F6E2050726573737572653D005302
:100B30006561206C6576656C20502863616C632963
:100B40003D00234572726F723A70726573737572ED
:100B50006520424D503038352C20636865636B202A
:100B6000776972696E67210049522054656D702063
:100B700073656E736F7220666F756E6400206D6FA3
:100B800062696C65206C6F6767657220737461724F
:100B9000746564202E2E2E20005769466920495026
:100BA0003A002357694669204950206164647265A0
:100BB00073733A2000456455484B205345534C6F9E
:100BC000676765720053656E736F7220736C6F7424
:100BD00020616E6420747970653A0057656C636FAC
:100BE0006D6520746F20456455484B00005EBCE283
:100BF000613FDD83C29C7E20A3FD1F41009D23BE7B
:100C000046DB65F88C11AF32CA57E974232D2D2DC0
:100C10002D2D2D2D2D2D2D2D2D2D2D2D2D2D2D2D04
:100C20002D2D2D2D2D2D2D2D2D2D2D2D2D2D2D2DF4
:100C30002D00235265736F6C7574696F6E3A2020B6
:100C40002000234D696E2056616C75653A20202086
:100C50002000234D61782056616C75653A20202074
:100C6000200023556E697175652049443A20202083
:100C7000200023447269766572205665723A2020FE
:100C800020002353656E736F723A202020202020AD
:100C90002000232D2D2D2D204D61676E6574696315
:100CA0002053656E736F72202D2D2D2D2D2D2D2D22
:100CB0002D2D2D2D2D2D2D2D2D2D2D2D00482D663D
:100CC00069656C643A202800202020202020202004
:100CD0002020202020202020002020202020202034
:100CE0002020202020202020200020202020202024
:100CF0002020202020202020202000202020202014
:100D00002020202020202020202020002020202003
:100D100020202020202020202020200020202020F3
:100D2000202020202020202020202000233A53684B
:100D30006F772F48696465204C4344002A3A546811
:100D400069732048656C700044233A43616C6962A2
:100D5000726174696F6E00442A3A53657474696EE7
:100D600067730044423A5265736574204C6F67673D
:100D700065720044433A436C656172204C43440001
:100D800044443A4D756C746953656E736F727300A9
:100D900044393A43757272656E7400566F6C7461B3
:100DA00067652B43757272656E740044383A456C02
:100DB0006563747269630044373A4D6F74696F6E8E
:100DC0000044363A44532054656D700044353A551A
:100DD0005620496E74656E736974790044343A4FD5
:100DE0003220636F6E632E0044333A434F322063E8
:100DF0006F6E632E0044323A504D28313A322E3510
:100E00003A3130290044323A504D28313A322E35A9
:100E10003A3130292A0044313A5475726269646962
:100E200074790044303A566F6C7461676500393AE2
:100E30006F7220334420616363656C2E00393A4938
:100E40006E636C2E20616E672E00383A70482076F3
:100E5000616C756500373A49522054656D700037F2
:100E60003A49522054656D702A00363A4D61676EDA
:100E700065746963206669656C6400353A4761731F
:100E8000204C6576656C00343A495220466C616DA1
:100E90006500333A4C6967687420496E742E0032DD
:100EA0003A616E642048656967687400323A546537
:100EB0006D7020507265737375726500313A5465B8
:100EC0006D702048756D696469747900303A536FAC
:100ED000756E64204C6576656C00303A536F756EA4
:100EE00064204C6576656C2A0054696D65206C61E0
:100EF0007073653A00576946692049503A004D6F52
:100F000074696F6E00555620496E742E0055562038
:100F1000496E74656E73697479004F3220436F6E49
:100F20006300434F3220436F6E630053656E736FEF
:100F300072206572726F722100234E6F2073656E8E
:100F4000736F722100434F3220436F6E63004D6513
:100F500061737572696E6700234E6F2073656E73DF
:100F60006F7220666F7220504D21004E6F207365A6
:100F70006E736F722100206E672F4C00504D313A16
:100F8000322E353A3130004D6561737572696E6786
:100F90002E2E00234E6F2054422073656E736F72A5
:100FA0003F00234E6F2073656E736F722100536F85
:100FB000756E64204C6576656C004D656173757265
:100FC000696E672E2E00234E6F2073656E736F72ED
:100FD0002100536F756E64204C6576656C00234E5E
:100FE0006F2073656E736F7220666F722074656D0B
:100FF0007020262068756D696469747921004E6FD0
:101000002053656E736F72210020666F72207465C5
:101010006D7020262068756D6964697479210023DC
:1010200053656E736F72204572726F722000536544
:101030006E736F72204572726F7221002357726F48
:101040006E672073656E736F7220666F72207465B1
:101050006D7020262068756D696469747921005768
:10106000726F6E672053656E736F72210054656DE9
:10107000702048756D6964697479004C696768749B
:1010800020496E74656E7369747900466C616D6594
:1010900020495200482D6669656C64005365617291
:1010A000636820446972656374696F6E00234E6FD4
:1010B0002070482073656E736F722100704820762F
:1010C000616C75650023496E76616C6964206B659F
:1010D000792100204D756C746973656E736F72733E
:1010E000004D756C746973656E736F72730044693B
:1010F0007361626C6500456E61626C650052656289
:101100006F6F74696E672E2E2E002344413A2D3284
:101110003300237265706C6965733D0067657453B5
:10112000656C665465737442697428293A200069B5
:1011300073496E74657272757074456E61626C6528
:10114000642831293A2000676574496E74657272AB
:101150007570744D617070696E672831293A20008E
:10116000676574496E74657272757074536F7572C9
:1011700063652831293A2000676574496E74657289
:1011800072757074536F7572636528293A20006711
:1011900065745261746528293A20332E3134313513
:1011A000393F00616363656C2E69734C6F77506FD4
:1011B00077657228293A2000616363656C2E697334
:1011C00041736C65657028293A2000616363656C22
:1011D0002E6973546170536F757263654F6E5A2830
:1011E000293A2000616363656C2E69735461705302
:1011F0006F757263654F6E5928293A2000616363E9
:10120000656C2E6973546170536F757263654F6EB0
:101210005828293A2000616363656C2E6973416325
:10122000746976697479536F757263654F6E5A2865
:10123000293A2000616363656C2E697341637469A8
:1012400076697479536F757263654F6E5928293AC0
:10125000200069734163746976697479536F75729C
:1012600063654F6E5828293A2000697354617044B1
:101270006574656374696F6E4F6E5A28293B2066EA
:10128000616C73653F2000697354617044657465D7
:101290006374696F6E4F6E5A28293B2074727565AE
:1012A0003F20006973546170446574656374696FAD
:1012B0006E4F6E5928293B2066616C73653F200094
:1012C0006973546170446574656374696F6E4F6EC1
:1012D0005928293B20747275653F20006973546159
:1012E00070446574656374696F6E4F6E5828293B4E
:1012F0002066616C73653F200069735461704465BA
:1013000074656374696F6E4F6E5828293B20747240
:1013100075653F20006765745375707072657373EF
:1013200042697428293B2066616C73653F20006721
:101330006574537570707265737342697428293BC4
:1013400020747275653F2000697341637469766922
:101350007479416328293A20006973496E61637486
:1013600069766974795A456E61626C656428293AB8
:1013700020006973496E61637469766974795945AF
:101380006E61626C656428293A20006973496E6158
:101390006374697669747958456E61626C65642816
:1013A000293A2000697341637469766974795A45F2
:1013B0006E61626C656428293A2000697341637428
:1013C000697669747959456E61626C656428293A59
:1013D00020006973416374697669747958456E6158
:1013E000626C656428293A200067657446726565F9
:1013F00046616C6C4475726174696F6E28293A207D
:10140000006765744672656546616C6C5468726508
:1014100073686F6C6428293A200067657454696D9D
:1014200065496E616374697669747928293A200088
:10143000676574496E61637469766974795468721A
:101440006573686F6C642829200067657441637454
:1014500069766974795468726573686F6C64282959
:101460002000676574446F75626C655461705769DC
:101470006E646F7728292000676574446F75626C0D
:10148000655461704C6174656E637928293A200057
:101490006765745461704475726174696F6E282950
:1014A0003A2000676574417869734F6666736574A6
:1014B0002826782C2026792C20267A293A200067A5
:1014C00065745461705468726573686F6C64282920
:1014D0003A200058595A2047733A200058595A2048
:1014E000434F554E54533A20007365742067616929
:1014F0006E735B5D3A006761696E735F6F726967F7
:101500005B5D3A00416E676C65732F00496E636CDA
:101510002E20616E672E0000002100240027002A83
:10152000002D003000330001010000040107010A12
:101530000100002200250028002B002E003100347D
:101540000002010000050108010B0100002000233A
:1015500000260029002C002F0032000001000003AB
:101560000106010901050505050705080808080227
:101570000202020A0A08080404040401010101012C
:101580000101010303030303030303040707070C1B
:101590000C0C0C0C0C0C0C020202020606060606D1
:1015A0000606060B0B0B0B0B0B0B0B01021020207E
:1015B00008081020401020408002010201080402A7
:1015C000010102040810204080804020100804021D
:1015D0000180040201804020100804020108040276
:1015E000010102040810204080010204081020407C
:1015F0008000000A0B02090C0D0E0807030401000D
:1016000000000000000000000000000000000000DA
:101610000000000000000000000000000012111097
:1016200000000000000000000000000000000000BA
:101630000000000000000023456E64206F66204D0E
:10164000756C746973656E736F72204379636C6532
:101650002300496E76616C6964206B657921000016
:10166000C2AB07AB11241FBECFEFD1E2DEBFCDBFAF
:1016700000E00CBF1BE0A0E0B2E0E6E7FCE701E021
:101680000BBF02C007900D92A43FB107D9F723E129
:10169000A4EFBBE001C01D92A83EB207E1F71BE03A
:1016A000C1E3DBE000E006C021970109802FFE01C5
:1016B0000E9449BBC033D10780E00807A9F70E9408
:1016C00055AE0C9429BE0C9400008091330D90917E
:1016D000340D891B990B08950895DC0180E0615059
:1016E00090F09D919827E92FEF70F0E0E451F44FCE
:1016F0002491E92FE295EF70F0E0E450F44FE4918B
:10170000822F8E27ECCF089520918E0C260F332741
:10171000331F21323105ECF42091AD0DFC0190E036
:1017200080E0243069F082E00895A0918E0C219130
:10173000AC014259534FA40FB52FB11D2C93019604
:10174000861798F380918E0C680F60938E0C80E062
:10175000089581E00895089508950895E091340D65
:101760008091330DE81730F4F0E0ED5EF24F8081A8
:1017700090E008958FEF9FEF08959091340D809140
:10178000330D2FEF3FEF981748F4E92FF0E0ED5EAF
:10179000F24F208130E09F5F9093340DC90108958E
:1017A000CF92DF92EF92FF920F931F93CF93DF932D
:1017B0007C01CB018A012091B30D222389F0EB013A
:1017C0006B01C40ED51ECC15DD0569F06991D701FA
:1017D000ED91FC910190F081E02DC7011995F3CFB7
:1017E000642F0E94840BC801DF91CF911F910F914C
:1017F000FF90EF90DF90CF900895CF93DF931F92EB
:10180000CDB7DEB769832091B30D2223F9F0209183
:10181000D50D203258F021E030E0FC0133832283E3
:1018200090E080E00F90DF91CF9108958091B40D0A
:10183000E82FF0E0EB54F24F998190838F5F809313
:10184000B40D8093D50D81E090E0ECCF61E0CE0146
:1018500001960E94840BF7CF90E080E00895AF924C
:10186000BF92CF92DF92EF92FF920F931F93CF938D
:10187000DF938C01EB0184E2FB0111928A95E9F779
:101880008EE10E94168C83E090E00E94118C0E94F1
:10189000FD9E66E08EE10E94159F1092340D8093AC
:1018A000330D8630F0F30E941D8FA82E0E941D8FED
:1018B000B82E0E941D8FE82E0E941D8FF82E0E94C8
:1018C0001D8FC82E0E941D8FD82E60E07A2D6B29A7
:1018D000072E000C880B990B0E9425B6F801658332
:1018E00076838783908760E07C2D6D29072E000C1E
:1018F000880B990B0E9425B6F80161877287838750
:10190000948760E07E2D6F29072E000C880B990BC1
:101910000E9425B6F801658776878787908B118AA4
:10192000128A138A148A84E290E0A0E0B0E08883EF
:101930009983AA83BB8385899689A789B08D8C8377
:101940009D83AE83BF8382E090E0A0E0B0E0888713
:101950009987AA87BB87188A198A1A8A1B8AC09016
:10196000E404D090E504E090E604F090E704A701D9
:10197000960165817681878190850E949DB820E0DF
:1019800030E048EC52E40E9484B66C8B7D8B8E8BE9
:101990009F8BA7019601F8016185728583859485E7
:1019A0000E949DB820E030E048EC52E40E9484B6EA
:1019B000688F798F8A8F9B8F2091E0043091E104AA
:1019C0004091E2045091E304F801658576858785AE
:1019D00090890E949DB820E030E048EC52E40E94DB
:1019E00084B66C8F7D8F8E8F9F8F81E0DF91CF913A
:1019F0001F910F91FF90EF90DF90CF90BF90AF902D
:101A00000895862F0C94329D862F642F0C945B9D35
:101A1000862F642F0C94899D1F93CF93DF93EC0145
:101A2000162F60E0812F0E94899D612F70E0FB01DD
:101A3000E555FA4EE491E883FB01EB59FA4EE49147
:101A4000F0E0EE0FFF1FE55BFA4E859194919A83CB
:101A500089831B861D861C861A86198618861F8216
:101A60001E821D821C821B82DF91CF911F910895DF
:101A7000E8E2F1E114A215A216A217A210A611A67F
:101A800012A613A681E084A729E130E036A725A796
:101A900087A780E090E0A0EAB0E480AB91ABA2AB76
:101AA000B3AB80E090E0A8EAB1E484AB95ABA6AB21
:101AB000B7AB8093DC049093DD04A093DE04B09375
:101AC000DF0480E090E0A0E8BFE380937211909380
:101AD0007311A0937411B09375118093D8049093EF
:101AE000D904A093DA04B093DB0410929F111092F2
:101AF0009E118BE090E09093A1118093A0119093A0
:101B0000D7048093D6041092AF111092AE1190E0DA
:101B100080E00C94888E2F923F924F925F926F924A
:101B20007F928F929F92AF92BF92CF92DF92EF926D
:101B3000FF920F931F93CF93DF936C01CDE3D5E01A
:101B400087E9882E84E0982E08E211E1EE24E394E0
:101B5000F12C22E1222E312C33E1432E512C40E195
:101B6000642E712C51E1A52EB12C80919704909197
:101B700098048E159F050CF4C9C021E0C216D1044B
:101B800009F0BDC0F80182AD93ADF4019383828367
:101B9000F40182819381009709F58A819B8190935A
:101BA000050280930402F4018281938184309105BF
:101BB000C1F52A813B8130930702209306028531CB
:101BC000910509F47BC08631910509F040C02A8156
:101BD0003B8130937C0420937B044EC0813091057F
:101BE00039F48A819B8190938B0480938A04DBCFA4
:101BF0008230910539F48A819B819093030280930E
:101C00000202D1CF039779F68A819B8190930102DA
:101C1000809300026EED7BE089E193E10E9467967C
:101C2000C2CF8530910539F42A813B8130937A0403
:101C300020937904C4CF8630910529F2873091052D
:101C4000B9F42A813B813093800420937F0487314B
:101C5000910591F42A813B8128303105B1F57092CC
:101C6000930460929204B0929104A092900404C0F4
:101C70008A30910509F0A3CF9C012B5031092A30FD
:101C8000310590F42A813B813093010220930002B8
:101C900039E1389FB001399F700D1124685F7D4F85
:101CA00089E193E10E94CA968FEFE81AF80A22961A
:101CB000E2E08E0E911C0E5F1F4F57CF2A813B81B1
:101CC00030937E0420937D04D7CF2730310549F42B
:101CD0003092930420929204509291044092900486
:101CE000CBCF2630310541F621E030E0309393042C
:101CF000209392041092910410929004BDCFF401AD
:101D000082819381F80193AF82AF42CFDF91CF916F
:101D10001F910F91FF90EF90DF90CF90BF90AF9009
:101D20009F908F907F906F905F904F903F902F90FB
:101D300008950F931F93CF93DF938C011092F50BAF
:101D40001092F40BC091F40BD091F50BC832D10571
:101D5000A4F4809106020E94C59DCC0FDD1FC95CD2
:101D6000D24F998388838091F40B9091F50B019663
:101D70009093F50B8093F40BE5CF0E945E8C20E0EE
:101D800030E040EA50E40E9484B620E030E040E8D1
:101D90005AE30E9484B60430110599F420E030E043
:101DA00040E650E40E9484B69B01AC0160E070E024
:101DB00080E890E40E94BEB7DF91CF911F910F9110
:101DC00008950A30110569F420E030E040E650E45F
:101DD0000E9484B69B01AC0160E070E080E291E477
:101DE000E9CF60E070E0CB01E7CF0F931F9360E095
:101DF000809192040E945B9D83E090E00197F1F74F
:101E000061E0809192040E945B9D83E290E00197E3
:101E1000F1F760E0809192040E945B9D80919004B4
:101E2000909191049927FC01E555FA4E6491FC01CB
:101E3000EB59FA4EE491F0E0EE0FFF1FE55BFA4E2E
:101E40008591949100E717E120E030E0462F0E9451
:101E5000C2AA611571058105910529F06F5F7F4F59
:101E60008F4F9F4F9F700E9425B620E030E44CE1D9
:101E700056E40E949DB82091120C3091130C4091B1
:101E8000140C5091150C0E9484B620E030E048E418
:101E900053E40E949DB81F910F910895DF92EF9235
:101EA000FF920F931F93CF93DF937C018B01D42E6E
:101EB000DC011696ED91FC91138615861486128628
:101EC0001186108617821682158214821382C0E052
:101ED000B801F701868197810E94D095D82F882379
:101EE00029F0DC1629F0CF5FDC1690F7D0E009C0AE
:101EF00067E0C8010E946D0BD80117969C91891369
:101F0000F2CF8D2FDF91CF911F910F91FF90EF9026
:101F1000DF900895DC012C911196ED91FC91F894DD
:101F20008181822B81839281322F309593239283FA
:101F300087E090E00197F1F781818323818383E239
:101F400090E00197F1F790817894EFECF0E0319711
:101F5000F1F7922381E009F480E00895FC0190817B
:101F60000180F281E02D292F209560FF14C0F894A4
:101F70008281822382838181892B8183A3E2B0E0E5
:101F80001197F1F78281982B9283789487ED90E0F6
:101F90000197F1F70895F8948281822382838181E9
:101FA000892B8183AFEFB0E01197F1F78281982BF5
:101FB000928378948FE090E0EBCFDF92EF92FF92E4
:101FC0000F931F93CF93DF93EC01D62EE42E08E0FE
:101FD00010E0FF24F39461E08D2D8F2109F460E07F
:101FE000CE010E94AE0FFF0C01501109A1F7E110C4
:101FF00010C0F894E981FA819181888180958923C4
:102000008183E981FA819281888180958923828305
:102010007894DF91CF911F910F91FF90EF90DF9017
:102020000895EF92FF920F931F93CF93DF938C014C
:102030007B0140E065E50E94DD0FE70188E0E80EE6
:10204000F11C699140E0C8010E94DD0FCE15DF054B
:10205000C1F7DF91CF911F910F91FF90EF900895FD
:10206000FC0190810180F281E02DF8948181292F7B
:1020700020958223818378943DE743E050E03150FE
:1020800029F1DA011197F1F780818923C1F3F894DE
:102090008281822382838181892B81837894ABE73B
:1020A000B7E01197F1F7F894818182238183A3E14E
:1020B000B1E01197F1F78081982381E009F080E089
:1020C0007894E3E6F6E03197F1F7089580E008951B
:1020D0008F929F92AF92BF92CF92DF92EF92FF9238
:1020E000CF93DF93EC018E819F810E94301040E0FE
:1020F0006CEC8E819F810E94DD0F488164E48E81AB
:102100009F810E94DD0F8A81882371F1E981E95066
:102110008EEEC82E82E0D82EE33038F4F0E0EE0FD9
:10212000FF1FEB5AFA4FC080D1808B81882339F191
:102130008881811124C00E94D6A74B015C010D2C1F
:10214000000CEE08FF088E819F810E948A0F81306B
:1021500059F00E94D6A76C197D098E099F09681550
:1021600079058A059B0578F3DF91CF91FF90EF9079
:10217000DF90CF90BF90AF909F908F900895B60161
:10218000DD0C880B990BDF91CF91FF90EF90DF90E2
:10219000CF90BF90AF909F908F900C943AA16F9288
:1021A0007F928F929F92AF92BF92CF92DF92EF92E7
:1021B000FF920F931F93CF93DF93EC017B018A0172
:1021C0008E819F810E943010811102C090E037C043
:1021D000B7018E819F810E94111040E06EEB8E81CD
:1021E0009F810E94DD0F7801680189E0C80ED11C33
:1021F000AE80BF8088E0882E912C712C6624639479
:10220000C5010E948A0F81117628660CE1E08E1AC2
:102210009108B1F7F70171927F01EC15FD0541F7C7
:102220008E819F810E943010813081F668E0C80164
:102230000E946D0B91E0F80120852813C7CF892FEC
:10224000DF91CF911F910F91FF90EF90DF90CF9092
:10225000BF90AF909F908F907F906F900895CF9395
:10226000DF9300D000D000D0CDB7DEB7AE014F5F16
:102270005F4F0E94CF10882331F08D818F33A9F0FA
:1022800020F48F31A1F080E007C08F3521F08F3727
:10229000D1F78CE001C08BE029960FB6F894DEBF31
:1022A0000FBECDBFDF91CF9108958AE0F5CF89E0D1
:1022B000F3CF0F931F93CF93DF93CDB7DEB7619723
:1022C0000FB6F894DEBF0FBECDBF8C01462FBE0106
:1022D000665F7F4F0E944E0F81110FC060E070E07B
:1022E0008EEF92EC61960FB6F894DEBF0FBECDBFB5
:1022F000DF91CF911F910F910895AE014F5F5F4F16
:10230000BE01665F7F4FC8010E94CF10882331F362
:102310006A8170E0762F6627770F770F770F298114
:1023200048E0249F90011124262B372B8A85803189
:10233000D1F4688570E08F81AB01481B5109CA0157
:102340009695982F8827979587950E9435BBCB0146
:102350004097B90153E0660F771F5A95E1F760780F
:102360009C01260F371F213854EE35070CF4B6CFE9
:10237000B901330F880B990B0E9425B620E030E09D
:1023800040E05CE30E9484B6ADCFEF92FF920F93E2
:102390001F93CF93DF9300D000D01F921F92CDB731
:1023A000DEB78C01DC011696ED91FC911797138630
:1023B000158614861286118610861782168215825B
:1023C0001482138214961C92149715961C92EE2474
:1023D000E394BE016F5F7F4FF801868197810E9471
:1023E000D095882309F46FC067E0CE0101960E9462
:1023F0006D0B98858913EDCFD8018C91811125C083
:1024000016968D919C910E943010BE016F5F7F4F98
:10241000F801868197810E94111040E064EBD80199
:1024200016968D919C910E94DD0FF801868197810F
:102430000E948A0FF82ED80116968D919C910E94C9
:102440003010F11002C0F801E082D8011196FC9022
:1024500089818031A1F1BE016F5F7F4FC8010E9469
:102460002F118F15D0F4F8018181D80111968C932A
:10247000119714968C9114978F5F14968C93898181
:10248000883231F0B0F4803119F0823209F0A1CFF6
:10249000F80185818F5F85839CCF8981803111F41C
:1024A0008CE0E3CFBE016F5F7F4FC8010E942F1108
:1024B000DCCF8B3369F3823409F08BCFE9CFFCE0BA
:1024C000FF1588F2EDCF28960FB6F894DEBF0FBE49
:1024D000CDBFDF91CF911F910F91FF90EF900895A5
:1024E0000F931F93CF938C01C62FFC0184810E9410
:1024F000168CF80183858C2B90E00E94118CCF9173
:102500001F910F910C94FD9E0F931F93CF938C01FD
:10251000C62F0E9470126C2F6460C8010E94701256
:102520006C2F6B7FC8010E94701283EC90E00197C2
:10253000F1F7CF911F910F9108950F931F93CF93B0
:102540008C01C62F607F61600E94841280E1C89F69
:10255000B00111246160C8010E94841281E090E002
:10256000CF911F910F9108951F920F920FB60F9266
:1025700011240BB60F922F933F934F935F936F935A
:102580007F938F939F93AF93BF93EF93FF9380912C
:1025900057100E94329D20915A1030915B102F5F8E
:1025A0003F4F30935B1020935A10909159109536FD
:1025B00018F096E09093561090915610943009F4CC
:1025C0006EC0F8F4923031F1933009F44CC0909120
:1025D0005810992319F0811171C02F9AFF91EF9132
:1025E000BF91AF919F918F917F916F915F914F912B
:1025F0003F912F910F900BBE0F900FBE0F901F9029
:102600001895953009F457C0963009F791E09093EA
:1026100026114FC08111DBCF20915A1030915B10F1
:102620002436310528F410925B1010925A10CFCF47
:102630001092261110925910E091591091E09E0FBE
:1026400090935910F0E020915A1030915B10EE0FEA
:10265000FF1FE45AFF4E3183208310925B101092CB
:102660005A1093E019C0813009F0B1CFE0915910B0
:1026700091E09E0F90935910F0E020915A10309104
:102680005B10EE0FFF1FE45AFF4E31832083109240
:102690005B1010925A1094E09093561098CF8823B4
:1026A00059F220915A1030915B102536310508F40B
:1026B0008ECF95E0F1CF81118ACFB5CF2F988ECFF5
:1026C000CF92DF92EF92FF92CF93DF93EC01072E30
:1026D000000C880B990B0E9425B66B017C0120E051
:1026E00030E040E45FE30E9484B620E030E048E45C
:1026F00052E40E949DB80E9449B9C617D707D4F08A
:1027000020E030E040EA5FE3C701B6010E9484B6F2
:1027100020E030E048E452E40E949DB820E030E040
:1027200040E85FE30E94BFB70E9449B921E06C17FF
:102730007D070CF420E0822F90E0DF91CF91FF9095
:10274000EF90DF90CF9008950F931F93CF93DF9377
:10275000082F6DE77BE08DEA9FE00E949C9BC7E01D
:10276000D0E010E0B8010C2E02C0759567950A9470
:10277000E2F76170772742E050E08DEA9FE00E9427
:102780004F9B219778F7DF91CF911F910F9108957B
:102790001092AD0D81E08093AC0D1092870D61E039
:1027A00084E10E945B9D61E085E10E945B9DE9EB15
:1027B000F0E080818E7F808380818D7F808388E4BC
:1027C0008093B80085E48093BC000895CF93DF9395
:1027D00091E090936D0C8823B9F0C091B800D0912E
:1027E000BA008091BC008A7B8093BC0060E084E1E9
:1027F0000E945B9D60E085E10E945B9D0E94C81382
:10280000D093BA00C093B800DF91CF91089585EDC1
:102810008093BC008091AF0D9091B00DA091B10D4F
:10282000B091B20D0796A11DB11D23E0B695A795F5
:10283000979587952A95D1F72091BC0024FD03C078
:102840001092AD0D08954091AF0D5091B00D609173
:10285000B10D7091B20D452B462B472B69F30097B4
:10286000A105B10541F025E32A95F1F70000019794
:10287000A109B109E1CF8091AE0D0C94E6131F922E
:102880000F920FB60F9211240BB60F922F933F9316
:102890004F935F936F937F938F939F93AF93BF9368
:1028A000EF93FF938091B900887F803609F44DC083
:1028B00008F040C0883209F4A9C028F5803109F435
:1028C0009DC0C8F4882309F4FBC0883009F496C081
:1028D000FF91EF91BF91AF919F918F917F916F91F8
:1028E0005F914F913F912F910F900BBE0F900FBEB4
:1028F0000F901F901895883109F488C0803241F7F5
:102900008093AB0D14C0803409F49DC040F4803333
:10291000B9F38833E9F68093AB0D85ECB0C0803510
:1029200009F485C0883509F496C0883489F60E9478
:102930000714CECF883909F48CC038F5883729F0D0
:1029400050F4883611F0803719F683E08093AD0D8E
:102950001092B00C57C0883809F47BC0803919F048
:10296000803809F0B5CF8091B00C803208F071C08A
:10297000E091B00C81E08E0F8093B00C8091BB0091
:10298000F0E0E057F34F80833DC0803B39F0E0F446
:10299000803A09F479C0883A09F09ACF84E08093AC
:1029A000AD0D10928F0C10928E0CE091110DF091E4
:1029B000120D199580918E0C81110FC081E08093CA
:1029C0008E0C10926E0C09C0803C09F4A6CF883C96
:1029D00009F4A3CF883B09F07BCFE0918F0C81E015
:1029E0008E0F80938F0CF0E0E259F34F808180933B
:1029F000BB0090918F0C80918E0C29C08091880D26
:102A00008093BB0085EC8093BC0062CF9091AA0DAF
:102A10008091A90D981758F5E091AA0D81E08E0FCD
:102A20008093AA0DF0E0E757F24F8081E9CFE09163
:102A3000AA0D81E08E0F8093AA0D8091BB00F0E07B
:102A4000E757F24F80839091AA0D8091A90D9817B6
:102A5000C8F285E8D8CFE091AA0D81E08E0F80936F
:102A6000AA0D8091BB00F0E0E757F24F8083809180
:102A7000AC0D81115CCF81E08093870D84EA809357
:102A8000BC001092AD0D24CF85EC8093BC00109259
:102A9000AD0D8091B00C803230F4E091B00CF0E0DC
:102AA000E057F34F10826091B00C70E0E0910F0D91
:102AB000F091100D80E99CE019951092B00C08CFB0
:102AC0001092AB0D34CF23E333E948E853E40E947E
:102AD0009DB820E030E040E85FE30E94BFB70E946D
:102AE000C7BA26E636EA45EA53E40E9484B6609304
:102AF000120C7093130C8093140C9093150C089582
:102B0000CF92DF92EF92FF920E94F50E6B017C0153
:102B100020E030E040E050E40E94A6B9181624F40A
:102B20000E94F50E6B017C0120E030E040E050E4B3
:102B3000C701B6010E94A6B9181624F40E94F50E2A
:102B40006B017C0120E030E040E050E4C701B601B9
:102B50000E94A6B9181624F40E94F50E6B017C01A0
:102B600020E030E040E050E4C701B6010E94A6B981
:102B7000181624F40E94F50E6B017C0120E030E071
:102B800040E050E4C701B6010E94A6B918162CF423
:102B9000C12CD12CE12C80E4F82EC701B601FF90A6
:102BA000EF90DF90CF90089581E08093E9048091C9
:102BB0008904882341F088E08093D71360E08CEC8F
:102BC00093E10C947012089580918904811110C0D2
:102BD00081E0809389048093E9048091D213982F37
:102BE00094609093D2138C600E94208C0C94D41526
:102BF0008091E9048823D1F31092D71360E08CEC24
:102C000093E10E9470121092E9048091D2138B7F9D
:102C10008093D21388600E94208C109289040895BA
:102C20002F923F924F925F926F927F928F929F92DC
:102C3000AF92BF92CF92DF92EF92FF920F931F93CA
:102C4000CF93DF93CDB7DEB766970FB6F894DEBFAC
:102C50000FBECDBF1C0180E19FE00E94FF8E40E8C7
:102C600055E260E070E080E19FE00E94E35964E695
:102C700070E080E090E00E943AA18CED95E0A0E049
:102C8000B0E08093140F9093150FA093160FB0939C
:102C9000170F64E670E080E090E00E943AA18FEFA9
:102CA0008A8781E08B8786E88C871D861E861F8633
:102CB000188A198A89E78A8BC101880F991F9E8B10
:102CC0008D8BD12CC12CF12CE12C412C512C3201BB
:102CD00080E19FE00E94368908974CF049E050E07F
:102CE000BE01665F7F4F80E19FE00E94F08865E053
:102CF00070E080E090E00E943AA110E000E0812CBA
:102D0000912C540180E19FE00E946789892B39F45E
:102D1000F4E08F169104A104B1040CF04EC002300F
:102D200011050CF04AC080E19FE00E946789892B61
:102D300069F080E19FE00E944589E1E0F0E0EC0F5E
:102D4000FD1FE00FF11F80830F5F1F4F65E070E0F4
:102D500080E090E00E943AA10230110509F073C0B2
:102D600099818A8598136FC09A818C8598136BC05E
:102D7000FE013396FC8BEB8B80E19FE00E9467891C
:102D8000892B39F4F4E08F169104A104B1040CF0FE
:102D900053C00930110509F05CC08B8190E0982F79
:102DA00088272C81820F911D092E000CAA0BBB0BCA
:102DB000480E591E6A1E7B1E43C08FEFC81AD80AE0
:102DC000E214F30434F4ED89FE89EC15FD0509F0F5
:102DD0007FCF80E19FE00E94FF8EE114F10409F4AF
:102DE0007101C301B2010E9425B64B015C01B7011C
:102DF000FF0C880B990B0E9425B69B01AC01C50105
:102E0000B4010E949DB866960FB6F894DEBF0FBE5F
:102E1000CDBFDF91CF911F910F91FF90EF90DF9089
:102E2000CF90BF90AF909F908F907F906F905F906A
:102E30004F903F902F900895043011050CF0ADCFC6
:102E4000FFEFEF1AFF0A8FEF881A980AA80AB80A4C
:102E500059CF80E19FE00E944589EB89FC898193ED
:102E6000FC8BEB8B0F5F1F4F87CF4F925F926F9260
:102E70007F929F92AF92BF92CF92DF92EF92FF929A
:102E80000F931F93CF93DF93982E8EE0A82EB12C33
:102E9000EE24EA9493E0F92E0FEF13E0D12CC12C2D
:102EA000D0E0C0E0412C512C3201892D0E94C59DFB
:102EB000C817D90708F44AC0C816D90608F46C0127
:102EC0008017910708F444C08E159F0508F47C0113
:102ED000BC0190E080E00E9423B69B01AC01C301DD
:102EE000B2010E94BFB72B013C0165E070E080E0B9
:102EF00090E00E943AA181E0A81AB108B1F6BE01A3
:102F00006C0D7D1D6E0D7F1D600F711F90E080E0C8
:102F10000E9423B69B01AC01C301B2010E94BEB75F
:102F200020E030E040E251E40E949DB8DF91CF9173
:102F30001F910F91FF90EF90DF90CF90BF90AF90D7
:102F40009F907F906F905F904F900895EC01B8CF65
:102F50008C01BECF4F925F926F927F92AF92BF92E1
:102F6000CF92DF92FF920F931F93CF93DF9300D006
:102F700000D0CDB7DEB75C0180E19FE00E94FF8EFC
:102F800040E052EC61E070E080E19FE00E94E35994
:102F90008CED95E0A0E0B0E08093140F9093150FB6
:102FA000A093160FB093170F64E670E080E090E0F6
:102FB0000E943AA1D12CC12CF12C65E070E080E098
:102FC00090E00E943AA110E000E0412C512C320127
:102FD000F1103AC080E19FE00E946789892B31F4AB
:102FE00085E1481651046104710474F5033011053C
:102FF0005CF580E19FE00E946789892B69F080E1A0
:103000009FE00E944589E1E0F0E0EC0FFD1FE00F3A
:10301000F11F80830F5F1F4F65E070E080E090E05C
:103020000E943AA1023011054CF089818B3B31F4AA
:10303000FF24F3948A818A3A09F0F12C8FEF481A21
:10304000580A680A780AC4CF8FEFC81AD80A64E60B
:1030500070E080E090E00E943AA1AC14BD0409F059
:10306000ACCF8F2D26960FB6F894DEBF0FBECDBF26
:10307000DF91CF911F910F91FF90DF90CF90BF9084
:10308000AF907F906F905F904F9008951F93CF9374
:10309000DF93182FC7E3DDE0812F0E94C59D899340
:1030A00099936CE370E080E090E00E943AA18DE09B
:1030B000C738D80789F70E945E8C20E030E040EAEC
:1030C00050E40E9484B620E030E040E85AE30E94D9
:1030D00084B6DF91CF911F910895CF92DF92EF9246
:1030E000FF920F931F93CF93DF93CDB7DEB7629715
:1030F0000FB6F894DEBF0FBECDBF20911E0C222369
:1031000009F4D5C02091430C3091440C263531058B
:103110000CF0CDC04091870450918804493D5F4038
:103120000CF0C5C08C012F5F3F4F3093440C2093AF
:10313000430C0E94D6A7C090160CD090170CE090BC
:10314000180CF090190C6C197D098E099F090E94CA
:1031500023B620E030E04AE754E40E949DB8609333
:103160001A0C70931B0C80931C0C90931D0C809177
:103170008704909188048835924034F488E592E081
:1031800090938804809387048091870490918804A9
:103190003AE1E32E3CE0F32E9C012A513C406901C8
:1031A000C6018E0D9F1D9A838983F70161917F016E
:1031B000CE0101960E94CA59FEE1EF16FCE0FF061F
:1031C00079F78091870490918804049690938804FD
:1031D00080938704B801CE0101960E944A99CE01DE
:1031E00001960E945298BC01CE010D960E944A9908
:1031F000CE0101960E94E798F80184819581849719
:1032000008F123E230E050E040E0B801CE01019641
:103210000E946499BE016F5F7F4FCE0107960E94A6
:103220004A99CE0107960E945298BC01CE010D9694
:103230000E949798CE0107960E94E798CE010196CA
:103240000E94E79849895A894115510531F06FE18B
:103250007CE0CE010D960E94B28E80918704909101
:10326000880423E4C22E2CE0D22E0FE11CE09C0146
:103270002F513C407901C701800F911F9A838983A8
:10328000F80161918F01CE0101960E94CA59C016C2
:10329000D10689F780918704909188048496909351
:1032A000880480938704CE010D960E94E798629669
:1032B0000FB6F894DEBF0FBECDBFDF91CF911F9147
:1032C0000F91FF90EF90DF90CF900895AF92BF9253
:1032D000CF92DF92EF92FF920F931F93CF93DF93E2
:1032E000CDB7DEB72C970FB6F894DEBF0FBECDBFBB
:1032F00080910D0D811102C00E9415598091950495
:1033000090919604029751F080910E0C90910F0CC1
:10331000009709F4B4C1039709F4B1C163E574E0FF
:103320008FEB92E10E9472986FEB72E1CE010196F1
:103330000E944A9944E150E070E060E0CE010196BD
:103340000E94DD5ACE0101960E94E79864E474E081
:103350008FEB92E10E9472986FEB72E1CE010196C1
:103360000E944A9944E150E06FEF7FEFCE01019651
:103370000E945759CE0101960E94E79887E00E946B
:1033800015A18C0186E00E9415A1BC0190E080E0AF
:103390000E9423B62AE037ED43EA5CE30E9484B63C
:1033A00023E333E948E853E40E94BEB76B017C0194
:1033B00084E0A82EB12C20E030E048EC52E4C701B4
:1033C000B6010E94A6B918160CF05FC081E0A81AD9
:1033D000B108E9F064E670E080E090E00E943AA174
:1033E00086E00E9415A1BC0190E080E00E9423B617
:1033F0002AE037ED43EA5CE30E9484B623E333E935
:1034000048E853E40E94BEB76B017C01D4CF69E366
:1034100074E08FEB92E10E9472986FEB72E1CE0143
:1034200001960E944A994AE050E070E060E0CE01C7
:1034300001960E94DD5ACE0101960E94E79867EB43
:1034400075E0CE0101960E9453996FEB72E1CE01B7
:1034500001960E940198BC0185EC92E10E94979828
:10346000CE0101960E94E79880910E0C90910F0C6E
:10347000049721F410920F0C10920E0C81E090E052
:103480009093960480939504D9C0B80190E080E0B1
:103490000E9423B62AE037ED43EA5CE30E9484B63B
:1034A00023E333E948E853E40E94BEB7AB01BC0113
:1034B00021E0CE0101960E94EF9869EC75E0CE0103
:1034C00007960E945399BE016F5F7F4FCE0107960A
:1034D0000E940198BC0185EC92E10E949798CE0170
:1034E00007960E94E798CE0101960E94E79865EC46
:1034F00072E1CE0101960E944A9942E350E06FEFDB
:103500007FEFCE0101960E945759CE0101960E948D
:10351000E79863ED75E0CE0101960E945399CE01C4
:1035200001960E943959CE0101960E94E79862EDFA
:1035300075E085EC92E10E94619821E0B701A60157
:10354000CE0101960E94EF9868EF76E0CE010796D3
:103550000E945399BE016F5F7F4FCE0107960E9474
:103560000198BC018BEC92E10E949798CE010796DE
:103570000E94E798CE0101960E94E79862E67AE001
:10358000CE0101960E9453996BEC72E1CE01019637
:103590000E940198BC018FEB92E10E949798CE01A6
:1035A00001960E94E7986FEB72E1CE0101960E94AE
:1035B0004A994AE050E070E060E0CE0101960E9436
:1035C000335ACE0101960E94E79863ED75E0CE0173
:1035D00001960E945399CE0101960E943959CE015D
:1035E00001960E94E79862ED75E08BEC92E10E94F3
:1035F00061986BEC72E1CE0101960E944A9962E6F5
:103600007AE0CE0101960E94EB9765EC72E10E9490
:103610000198BC0185EC92E10E949798CE01019639
:103620000E94E79880910E0C90910F0C039731F453
:1036300084E090E090930F0C80930E0C64E670E0B1
:1036400080E090E00E943AA180910D0D882331F036
:1036500060E273E080E090E00E943AA12C960FB601
:10366000F894DEBF0FBECDBFDF91CF911F910F91B8
:10367000FF90EF90DF90CF90BF90AF90089583E7D9
:103680009EE00E94FF8E64E670E080E090E00E9481
:103690003AA169E774E08FEB92E10E9472986FEBB8
:1036A00072E1CE0101960E944A9944E150E070E037
:1036B00060E0CE0101960E94DD5ACE0101960E9483
:1036C000E7986AE674E08FEB92E10E9472986FEBE4
:1036D00072E1CE0101960E944A9944E150E06FEFF9
:1036E0007FEFCE0101960E945759CE0101960E94AC
:1036F000E7988CE40E9414A86B017C0104E010E0C0
:10370000A7019601C701B6010E940BBB882309F4EB
:1037100049C00150110961F068EC70E080E090E070
:103720000E943AA18CE40E9414A86B017C01E8CFAE
:103730006FE574E08FEB92E10E9472986FEB72E19B
:10374000CE0101960E944A994AE050E070E060E0A4
:10375000CE0101960E94DD5ACE0101960E94E798A3
:1037600067EB75E0CE0101960E9453996FEB72E111
:10377000CE0101960E940198BC0185EC92E10E9465
:103780009798CE0101960E94E79880910E0C909137
:103790000F0C039721F410920F0C10920E0C82E084
:1037A00090E06ECE21E0B701A601CE0107960E94FF
:1037B000EF9869EC75E0CE0101960E945399BE0125
:1037C000695F7F4FCE0101960E940198BC0185EC94
:1037D00092E10E949798CE0101960E94E798CE014F
:1037E00007960E94E79865EC72E1CE0101960E946F
:1037F0004A9942E350E06FEF7FEFCE0101960E94BD
:103800005759CE0101960E94E79863ED75E0CE010D
:1038100001960E945399CE0101960E943959CE011A
:1038200001960E94E79862ED75E085EC92E10E94B6
:10383000619886E60E9414A86B017C0104E010E008
:10384000A7019601C701B6010E940BBB882381F036
:103850000150110909F484C068EC70E080E090E048
:103860000E943AA186E60E9414A86B017C01E8CF71
:1038700021E0B701A601CE0107960E94EF9868EFFC
:1038800076E0CE0101960E945399BE01695F7F4F99
:10389000CE0101960E940198BC018BEC92E10E943E
:1038A0009798CE0101960E94E798CE0107960E9454
:1038B000E79862E67AE0CE0101960E9453996BEC9C
:1038C00072E1CE0101960E940198BC018FEB92E15A
:1038D0000E949798CE0101960E94E7986FEB72E1E3
:1038E000CE0101960E944A994AE050E06FEF7FEFC7
:1038F000CE0101960E94335ACE0101960E94E798AC
:1039000063ED75E0CE0101960E945399CE010196B8
:103910000E943959CE0101960E94E79862ED75E048
:103920008BEC92E10E9461986BEC72E1CE01019602
:103930000E944A9962E67AE0CE0101960E94EB97D6
:1039400065EC72E10E940198BC0185EC92E10E9455
:103950009798CE0101960E94E79883E090E06ACEA6
:103960006EED7BE08BEC92E10E946796DDCFEF92EB
:10397000FF920F931F93CF93DF93CDB7DEB7689776
:103980000FB6F894DEBF0FBECDBF8C0162E67AE0C1
:10399000CE010D960E94539965ED75E0CE014396D8
:1039A0000E9453996AEB79E0C8010E944199BE01D7
:1039B0006D5E7F4FC8010E946B9861EB79E0C80192
:1039C0000E9414988FEBE82E81E1F82EF7016081B8
:1039D00070E0CE0101960E949E96BE016F5F7F4F00
:1039E000CE0107960E944A99BE01635F7F4FCE01C8
:1039F00007960E940198BC01C8010E946B98CE01F5
:103A000007960E94E798CE0101960E94E79864EA23
:103A100079E0C8010E941498F7016181062E000C1C
:103A2000770BCE0101960E949E96BE016F5F7F4F7D
:103A3000CE0107960E944A99BE01635F7F4FCE0177
:103A400007960E940198BC01C8010E946B98CE01A4
:103A500007960E94E798CE0101960E94E7986AE9CE
:103A600079E0C8010E941498F7016281062E000CCB
:103A7000770BCE0101960E949E96BE016F5F7F4F2D
:103A8000CE0107960E944A99BE01635F7F4FCE0127
:103A900007960E940198BC01C8010E946B98CE0154
:103AA00007960E94E798CE0101960E94E79862E986
:103AB00079E0C8010E941498F70163817481CE01F6
:103AC00001960E949E96BE016F5F7F4FCE010796C2
:103AD0000E944A99BE016D5E7F4FCE0107960E94FB
:103AE0000198BC01C8010E946B98CE0107960E9404
:103AF000E798CE0101960E94E7986BE779E0C8014C
:103B00000E941498F70165817681CE0101960E948A
:103B10009E96BE016F5F7F4FCE0107960E944A9925
:103B2000BE01635F7F4FCE0107960E940198BC01E2
:103B3000C8010E946B98CE0107960E94E798CE01BB
:103B400001960E94E79862E779E0C8010E94149804
:103B5000F7016781062E000C770B6F5F7F4FCE0158
:103B600001960E949E96BE016F5F7F4FCE01079621
:103B70000E944A99BE01635F7F4FCE0107960E9463
:103B80000198BC01C8010E946B98CE0107960E9463
:103B9000E798CE0101960E94E79867E679E0C801B0
:103BA0000E941498F7016085062E000C770BCE0159
:103BB00001960E949E96BE016F5F7F4FC8010E94D2
:103BC0006B98CE0101960E94E798CE0143960E9421
:103BD000E798CE010D960E94E798C80168960FB647
:103BE000F894DEBF0FBECDBFDF91CF911F910F9133
:103BF000FF90EF9008954F925F926F927F929F9205
:103C0000AF92BF92CF92DF92EF92FF920F931F93EA
:103C1000CF93DF93CDB7DEB7A8970FB6F894DEBF8A
:103C20000FBECDBF63EE72E18DED92E10E949798D9
:103C30000E94509665E076E0CE0101960E9453996D
:103C4000BE016F5F7F4F8DED92E10E94D097182FDC
:103C5000CE0101960E94E798112309F4F7C08091E4
:103C6000E7129091E8124097B8F080E0A8960FB65E
:103C7000F894DEBF0FBECDBFDF91CF911F910F91A2
:103C8000FF90EF90DF90CF90BF90AF909F907F908C
:103C90006F905F904F90089542E050E063EE72E1C4
:103CA000CE0101960E94275ABE016F5F7F4F8FEBB6
:103CB00092E10E94AE98CE0101960E94E7986FEBC8
:103CC00072E1CE0101960E944A99CE0101960E94AE
:103CD000DF5CCE0101960E94E7988FEB92E10E9493
:103CE000D99620E030E048EC52E40E9484B60E946D
:103CF00049B9AB01BC014093C9045093CA04609315
:103D0000CB047093CC04CE0101960E947196CE0133
:103D100001960E94DF5CCE0101960E94E7986091B7
:103D2000C9047091CA048091CB049091CC048B019A
:103D30009C0100591F452140310901341C492105CE
:103D40003105C8F168ED75E0CE0101960E945399E6
:103D50006FEB72E1CE0101960E9401986BEE75E067
:103D60000E94EB97BC0185EC92E10E949798CE01EE
:103D700001960E94E79866ED75E0CE0101960E94DB
:103D8000539965EC72E1CE0101960E940198BC0145
:103D9000CE0145960E944A99CE0145960E94E1586F
:103DA000CE0145960E94E798CE0101960E94E798C1
:103DB0001092EE0489C01A821982FE01339626E021
:103DC000DF011D922A95E9F70E9425B620E030E038
:103DD00048EC52E40E949DB88E010F5F1F4F22E015
:103DE00047E00E947AB1BC0185EC92E10E94CA963C
:103DF0006BEF75E0CE0145960E94539965EC72E138
:103E0000CE0145960E94019868E076E00E94EB970B
:103E1000BC0185EC92E10E949798CE0145960E94E4
:103E2000E7988091C9049091CA04A091CB04B09105
:103E3000CC048093281190932911A0932A11B09358
:103E40002B1190E080E00E94888E95CF61EF78E0A2
:103E5000CE0101960E944199BE016F5F7F4F8DEDAB
:103E600092E10E94D097182FCE0101960E94E79808
:103E7000112389F142E050E063EE72E1CE01019638
:103E80000E94275ABE016F5F7F4F8FEB92E10E9425
:103E9000AE98CE0101960E94E7988FEB92E10E94C6
:103EA000E4966330710590F47093110C6093100CDC
:103EB0008091100C9091110C9093AF118093AE11E2
:103EC00090E080E00E94888E81E0D0CE1092110CAC
:103ED0001092100CEDCF6CEE78E0CE0101960E94AE
:103EE0004199BE016F5F7F4F8DED92E10E94D097A7
:103EF000182FCE0101960E94E7981123A1F126E028
:103F000030E044E050E063EE72E1CE0101960E94A1
:103F10006499BE016F5F7F4F8FEB92E10E94AE9874
:103F2000CE0101960E94E7988FEB92E10E94E49601
:103F30007093A1116093A0117093D7046093D6047D
:103F400063EE72E1CE0101960E944A99CE0101967C
:103F50000E94DF5CCE0101960E94E79890E080E02D
:103F60000E94888E25CF65EE78E0CE0101960E94F2
:103F70004199BE016F5F7F4F8DED92E10E94D09716
:103F8000182FCE0101960E94E7981123A1F146E077
:103F900050E063EE72E1CE0101960E94275ABE0105
:103FA0006F5F7F4F8FEB92E10E94AE98CE0101963A
:103FB0000E94E7988091C3129091C412892B61F0FE
:103FC0008FEB92E10E94D99660938C0470938D04DC
:103FD00080938E0490938F0463EE72E1CE0101967C
:103FE0000E944A99CE0101960E94DF5CCE010196A3
:103FF0000E94E798DDCE6DE076E0CE0101960E944A
:104000005399BE016F5F7F4F8DED92E10E94D09773
:10401000182FCE0101960E94E798112309F4BEC023
:1040200061EE78E0CE0101960E944199BE016F5F7A
:104030007F4F8DED92E10E94D097182FCE0101960F
:104040000E94E7981123D1F184E090E00E94990E3C
:104050006093AD047093AE048093AF049093B0046A
:1040600061ED78E085EC92E10E9472984091AD0498
:104070005091AE046091AF047091B00422E0CE0183
:1040800001960E94EF98BE016F5F7F4F85EC92E131
:104090000E946B98CE0101960E94E7988091AD0432
:1040A0009091AE04A091AF04B091B00480934C11F4
:1040B00090934D11A0934E11B0934F1160E176E0B3
:1040C000CE0101960E945399BE016F5F7F4F8DED27
:1040D00092E10E94D097182FCE0101960E94E79896
:1040E0001123F1F18AE090E00E94990E6093A904F7
:1040F0007093AA048093AB049093AC0460EC78E0D6
:1041000085EC92E10E9472984091A9045091AA0412
:104110006091AB047091AC0422E0CE0101960E9444
:10412000EF98BE016F5F7F4F85EC92E10E946B9824
:10413000CE0101960E94E7988091A9049091AA046B
:10414000A091AB04B091AC048093501190935111A5
:10415000A0935211B093531190E080E00E94888E9A
:1041600066ED75E0CE0101960E94539965EC72E10F
:10417000CE0101960E940198BC01CE0145960E9495
:104180004A99CE0145960E94E158CE0145960E947B
:10419000E798CE0101960E94E79896CE65E176E019
:1041A000CE0101960E945399BE016F5F7F4F8DED46
:1041B00092E10E94D097182FCE0101960E94E798B5
:1041C000112309F4BDC08091E7129091E81207977E
:1041D000F8F046E050E063EE72E1CE0101960E94F5
:1041E000275ABE016F5F7F4F8FEB92E10E94AE981E
:1041F000CE0101960E94E7988FEB92E10E94D9963A
:104200006093DC047093DD048093DE049093DF04FC
:1042100080917F049091800499270E9435172DE0AA
:1042200038E643E55BE30E9484B66B017C01209194
:104230000705309108054091090550910A050E9433
:104240001EB618160CF460C06091EF047091F00473
:104250008091F1049091F20420E030E048EC52E4C7
:104260000E9484B66B017C0120E030E0A9010E942D
:104270001EB6181634F0C12CD12C38EAE32E31E4E6
:10428000F32EC092DC04D092DD04E092DE04F092C2
:10429000DF04C0925C11D0925D11E0925E11F09249
:1042A0005F1180910E0D882381F06EEA78E08DEA2F
:1042B0009FE00E94BE9B6091DC047091DD048091C0
:1042C000DE049091DF040E94409B90E080E00E9419
:1042D000888E64EA78E085EC92E10E9472984091C1
:1042E000DC045091DD046091DE047091DF0422E073
:1042F000CE0101960E94EF98BE016F5F7F4F85EC63
:1043000092E10E946B98A7C020911B0530911C057B
:1043100040911D0550911E05C701B6010E94A6B926
:1043200087FF05C0C701B6010E94888D95CF6091B7
:1043300003057091040580910505909106058CCFC9
:1043400060EA78E0CE0101960E944199BE016F5F5C
:104350007F4F8DED92E10E94D097182FCE010196EC
:104360000E94E798112309F47BC060E080917D04EE
:104370000E94899D09E110E0C12CD12C7601809129
:104380007D040E94C59DBC01990F880B990B0E946A
:1043900025B69B01AC01C701B6010E94BFB76B01F6
:1043A0007C016AE070E080E090E00E943AA1015058
:1043B000110929F720E030E040EA50E4C701B601D6
:1043C0000E9484B620E030EC4FE754E40E949DB890
:1043D00020E030E048EC51E40E949DB86093D8049E
:1043E0007093D9048093DA049093DB046093721184
:1043F00070937311809374119093751190E080E025
:104400000E94888E6DE878E085EC92E10E947298B7
:104410004091D8045091D9046091DA047091DB0482
:1044200022E0CE0101960E94EF98BE016F5F7F4FA0
:10443000CE0145960E944A996BE176E0CE01459601
:104440000E94EB97BC0185EC92E10E946B98CE0133
:1044500045960E94E798CE0101960E94E79856C0C3
:104460006EE176E0CE0101960E945399BE016F5F26
:104470007F4F8DED92E10E94D097182FCE010196CB
:104480000E94E798112309F44CC080915711082E1F
:10449000000C990B0197039798F589E390E00E942F
:1044A00035172AE137E64CE950E40E9484B6609360
:1044B00058117093591180935A1190935B1190E0A9
:1044C00080E00E94888E6CE678E085EC92E10E94A4
:1044D0007298409158115091591160915A117091F0
:1044E0005B1122E0CE0101960E94EF98BE016F5F42
:1044F0007F4FCE0145960E944A9964E276E09ECFB6
:1045000066E478E085EC92E10E94729865EC72E1D5
:10451000CE0101960E944A99CE0101960E94E1586F
:1045200065CD62E478E0CE0101960E944199BE011A
:104530006F5F7F4F8DED92E10E94D097182FCE01D3
:1045400001960E94E798112309F43CC126E030E06F
:1045500044E050E063EE72E1CE0101960E9464995E
:10456000BE016F5F7F4F8FEB92E10E94AE98CE014C
:1045700001960E94E7988FEB92E10E94E4966B010E
:104580005B016CE679E0CE0101960E945399BE0171
:104590006F5F7F4F83EE92E10E949A978E010B5ED0
:1045A0001F4FAC014F5F5F4F63EE72E1C8010E9485
:1045B000275AB8018FEB92E10E94AE98C8010E9481
:1045C000E798CE0101960E94E79890907B048FEBCC
:1045D00092E10E94D9962B013C0180910E0D882317
:1045E000B9F06BE577E08DEA9FE00E94BE9B4AE060
:1045F00050E0B6018DEA9FE00E944F9B62E67AE0B0
:104600008DEA9FE00E949C9BC301B2010E94409BE7
:10461000692DC8010E940C0D18870F831D821E8210
:10462000198289E08A8381E08B838C831C8A1B8AB0
:10463000CE0101960E94C511CE0101960E9468101C
:10464000CE0101960E942AA40E8110E00B301105C4
:1046500014F00AE010E0BBE5CB16D10408F44EC01C
:1046600025E4C22E2CE0D22E5601412C512C3201D1
:10467000F12CE12C0E151F05B9F06E2DCE0101961F
:104680000E9459119B01AC01F50121933193419393
:1046900051935F01C301B2010E94BFB72B013C01DE
:1046A000FFEFEF1AFF0AE6CFB7010F2C000C880BC3
:1046B000990B0E9425B69B01AC01C301B2010E9477
:1046C0009DB82B013C0110E000E0E016F106B9F1C5
:1046D000D6012D913D914D915D916D015D01B4E04B
:1046E000AB1AB108C301B2010E94BEB7F5016083E5
:1046F0007183828393830F5F1F4FE7CF1A141B04CC
:104700000CF041C00A151B050CF08601015011097F
:10471000602FCE0101960E9459119B01AC01000F40
:10472000111F000F111F0B5B134FC301B2010E9439
:10473000BEB7D8016D937D938D939C931397E5E459
:10474000FCE0A6E7B1E18DE69CE0419151916191D9
:1047500071914D935D936D937D938E179F07A9F78C
:1047600090E080E00E94888E61E278E085EC92E142
:104770000E94729844E050E063EE72E1CE0101962F
:104780000E94275AB9CDA114B104C9F685E4E82ED8
:104790008CE0F82E0A151B0591F26A2DCE010196C8
:1047A0000E9459119B01AC01C301B2010E94BEB726
:1047B000F70161937193819391937F01FFEFAF1A9A
:1047C000BF0AE8CF67E276E0CE0101960E945399D6
:1047D000BE016F5F7F4F8DED92E10E94D097182F41
:1047E000CE0101960E94E798112309F423C127E026
:1047F00030E046E050E063EE72E1CE0101960E94A7
:104800006499BE016F5F7F4F8FEB92E10E94AE987B
:10481000CE0101960E94E7988FEB92E10E94E49608
:104820007B016093571183EE92E10E94EF9662E65E
:104830007AE0CE0101960E945399BE016F5F7F4FCF
:1048400083EE92E10E949A97AC014F5F5F4F63EE57
:1048500072E1CE0145960E94275ACE0145960E94EC
:10486000D996609358117093591180935A1190936F
:104870005B11CE0145960E94E798CE0101960E94F9
:10488000E79860E178E085EC92E10E94729844E05C
:10489000E416F1041CF582E0E816F1040CF09FC068
:1048A000E114F10431F1EA94EF2809F471C0609148
:1048B0005711062E000C770BCE0145960E949E964E
:1048C00069E376E0CE0101960E945399BE016B5ECA
:1048D0007F4FCE0101960E9401984CC0B4E0EB16C8
:1048E000F10429F76FEE77E085EC92E10E941498CD
:1048F00071C020E030E0A901609158117091591108
:1049000080915A1190915B110E941EB6181664F0A6
:1049100080E090E0A0E8BFE3809358119093591194
:10492000A0935A11B0935B112091581130915911F5
:1049300040915A1150915B1160E070E080EA90E480
:104940000E949DB8AB01BC0122E0CE0145960E94B9
:10495000EF986EE276E0CE0101960E945399BE0177
:104960006B5E7F4FCE0101960E94019862E07BE072
:104970000E94EB97BC0185EC92E10E946B98CE01FE
:1049800001960E94E798CE0145960E94E79822C0C2
:1049900062E078E085EC92E10E94149820E030E03B
:1049A00048E453E4609158117091591180915A1163
:1049B00090915B110E941EB6181664F080E090E49E
:1049C000ACE1B5E48093581190935911A0935A111A
:1049D000B0935B1190E080E00E94888E97CD66EFE7
:1049E00077E085EC92E10E9414988AE08E9DB001F8
:1049F0008F9D700D1124CE0101960E949E96BE01DE
:104A00006F5F7F4FCE0145960E944A996BEF7AE027
:104A1000CE0145960E94EB97BC0185EC92E10E9485
:104A20006B98CE0145960E94E798CE0101960E94B0
:104A3000E798B4CF60E476E0CE0101960E945399E6
:104A4000BE016F5F7F4F8DED92E10E94D097182FCE
:104A5000CE0101960E94E798112309F4CCC027E00B
:104A600030E046E050E063EE72E1CE0101960E9434
:104A70006499BE016F5F7F4F8FEB92E10E94AE9809
:104A8000CE0101960E94E7988FEB92E10E94E49696
:104A90006093541183EE92E10E94EF968FEB92E1C6
:104AA0000E94E496611571058105910509F074C0B5
:104AB00085E090E0909356118093551190E080E04E
:104AC0000E94888E6EED77E085EC92E10E947298EC
:104AD00080915411833044F563ED77E085EC92E1E9
:104AE0000E9414986091551170915611CE01019653
:104AF0000E949E96BE016F5F7F4FCE0145960E9439
:104B00004A996CE37AE0CE0145960E94EB97BC018E
:104B100085EC92E10E946B98CE0145960E94E79841
:104B2000CE0101960E94E7988091541183300CF4D5
:104B3000EDCC6091551170915611CE0183960E9473
:104B40009E9660915411062E000C770BCE0145966F
:104B50000E949E9669E376E0CE0101960E945399E9
:104B6000BE016B5E7F4FCE0101960E940198BE018F
:104B70006D5D7F4F0E940198BC0185EC92E10E941F
:104B80006B98CE0101960E94E798CE0145960E944F
:104B9000E798CE01839661CC61307105810591055E
:104BA00019F489E190E086CF62E67AE0CE010196C1
:104BB0000E945399BE016F5F7F4F83EE92E10E9486
:104BC0009A97AC014F5F5F4F63EE72E1CE0145965D
:104BD0000E94275ACE0145960E94E4967093561182
:104BE00060935511CE0145960E94E798CE0101963B
:104BF0000E94E79863CF67E476E0CE0101960E94B9
:104C00005399BE016F5F7F4F8DED92E10E94D09767
:104C1000182FCE0101960E94E798112309F468C06D
:104C20008091790490917A040E9446186093B104AF
:104C30007093B2048093B3049093B40460934011D2
:104C400070934111809342119093431180E090E55D
:104C5000A3ECB7E48093B9049093BA04A093BB0487
:104C6000B093BC048093381190933911A0933A11FA
:104C7000B0933B1180910E0D882381F065EB77E0B6
:104C80008DEA9FE00E94BE9B6091B1047091B204D6
:104C90008091B3049091B4040E94409B90E080E026
:104CA0000E94888E4091B1045091B2046091B30487
:104CB0007091B40422E0CE0145960E94EF986BE417
:104CC00076E0CE0101960E945399BE016B5E7F4F44
:104CD000CE0101960E940198BC0185EC92E10E94F0
:104CE0009798CE0101960E94E798CE014596B5CBE4
:104CF00066E576E0CE0101960E945399BE016F5F92
:104D00007F4F8DED92E10E94D097182FCE01019632
:104D10000E94E798112309F488C08091E7129091CE
:104D2000E8120497F8F044E050E063EE72E1CE013F
:104D300001960E94275ABE016F5F7F4F8FEB92E171
:104D40000E94AE98CE0101960E94E7988FEB92E107
:104D50000E94D9966093BD047093BE048093BF04F3
:104D60009093C0048091BD049091BE04A091BF04B3
:104D7000B091C0048093341190933511A0933611F3
:104D8000B093371180910E0D882389F06CE977E09C
:104D90008DEA9FE00E94BE9B6091BD047091BE04AD
:104DA0008091BF049091C00442E00E945E9A80917D
:104DB000790490917A040E9446186093B504709328
:104DC000B6048093B7049093B80460933C11709339
:104DD0003D1180933E1190933F1180910E0D8823D9
:104DE00081F062E977E08DEA9FE00E94BE9B6091CE
:104DF000B5047091B6048091B7049091B8040E94F4
:104E0000409B90E080E00E94888E4091B5045091D4
:104E1000B6046091B7047091B80422E0CE014596C3
:104E20000E94EF986AE576E04CCF62E676E0CE012C
:104E300001960E945399BE016F5F7F4F8DED92E105
:104E40000E94D097182FCE0101960E94E798112357
:104E500011F40C94351E8091E7129091E81204979A
:104E6000F8F044E050E063EE72E1CE0101960E945A
:104E7000275ABE016F5F7F4F8FEB92E10E94AE9881
:104E8000CE0101960E94E7988FEB92E10E94D9969D
:104E90006093B9047093BA048093BB049093BC04EC
:104EA0008091B9049091BA04A091BB04B091BC0464
:104EB0008093381190933911A0933A11B0933B111C
:104EC00080910E0D882389F069E777E08DEA9FE0F5
:104ED0000E94BE9B6091B9047091BA048091BB049A
:104EE0009091BC0442E00E945E9A80917904909176
:104EF0007A040E9446186093B1047093B2048093C0
:104F0000B3049093B4046093401170934111809363
:104F100042119093431180910E0D882381F06FE62A
:104F200077E08DEA9FE00E94BE9B6091B104709192
:104F3000B2048091B3049091B4040E94409B90E02D
:104F400080E00E94888E4091B1045091B20460913B
:104F5000B3047091B40461CFCF93DF93CDB7DEB7C4
:104F60002C970FB6F894DEBF0FBECDBF81309105F0
:104F700009F06EC090939F1180939E1168E076E0D7
:104F8000CE0101960E944199CE0101960E94DF5CFC
:104F9000CE0101960E94E79866E676E0CE01019682
:104FA0000E94539964EB73E1CE0101960E9401982F
:104FB000BC01CE0107960E944A9948EC50E06FEF81
:104FC0007FEFCE0107960E94DD5ACE0107960E9420
:104FD000E798CE0101960E94E79886ED9DE00E9439
:104FE000FF8E40E052EC61E070E086ED9DE00E94B3
:104FF000E35990E080E00E94888E65E776E0CE017C
:1050000001960E94539960EC73E1CE0101960E94D3
:105010000198BC01CE0107960E944A9940ED57E0E5
:105020006FEF7FEFCE0107960E945759CE0107968A
:105030000E94E798CE0101960E94E79881E02C96A5
:105040000FB6F894DEBF0FBECDBFDF91CF910895AC
:105050000097E1F510929F1110929E116AEF75E092
:10506000CE0101960E944199CE0101960E94DF5C1B
:10507000CE0101960E94E7986CE676E0CE0101969B
:105080000E94539964EB73E1CE0101960E9401984E
:10509000BC01CE0107960E944A9948EC50E06FEFA0
:1050A0007FEFCE0107960E94DD5ACE0107960E943F
:1050B000E798CE0101960E94E79886ED9DE00E9458
:1050C000FF8E40E855E260E070E08FCF82309105BE
:1050D000A9F490939F1180939E1169EE75E0CE0123
:1050E00001960E944199CE0101960E94DF5CCE019B
:1050F00001960E94E79860E776E0C0CF80E09FCFFE
:105100000F931F93CF93DF93CDB7DEB72C970FB6D6
:10511000F894DEBF0FBECDBF8C016EED7BE083EE59
:1051200092E10E9467960830110509F0F8C06FED12
:1051300075E0CE0101960E94419944E650E06FEF80
:105140007FEFCE0101960E94DD5ACE0101960E94AA
:10515000E79863ED75E0CE0101960E94419944E61F
:1051600050E070E060E0CE0101960E945759CE01F8
:1051700001960E94E79886ED9DE00E940A8A4CE223
:1051800051E061E070E0CE0107960E9407A5809192
:105190000E0D8823D1F06AE776E0CE0101960E94D9
:1051A0005399BE01695F7F4FCE0101960E9401981D
:1051B0006DE776E00E94EB97BC018DEA9FE00E94CC
:1051C000AC9BCE0101960E94E7986BEF7AE0CE018E
:1051D00001960E945399BE016F5F7F4FCE010796E3
:1051E0000E94D097182FCE0101960E94E7981123B4
:1051F00009F478C06FE776E083EE92E10E9467964B
:1052000088E090E090930D0C80930C0C0E94FB1DA5
:10521000182F66EC75E0CE0101960E94419944E694
:1052200050E070E060E0CE0101960E945759CE0137
:1052300001960E94E79886ED9DE00E940A8A48E563
:1052400052E061E070E0CE0101960E9407A5BE0128
:105250006F5F7F4FCE0107960E94AE98CE010196F8
:105260000E94E79880910E0D8823D1F06AE776E0DE
:10527000CE0101960E945399BE01695F7F4FCE0116
:1052800001960E9401986DE776E00E94EB97BC01C1
:105290008DEA9FE00E94AC9BCE0101960E94E798A8
:1052A0006DE77BE0CE0101960E945399BE016F5FCE
:1052B0007F4FCE0107960E94D097082FCE0101960E
:1052C0000E94E798002371F064E876E083EE92E1B3
:1052D0000E9467960E94FB1D882321F069EB75E010
:1052E000111102C062EB75E0CE0101960E94419956
:1052F00044E650E070E060E0CE0101960E9457590C
:10530000CE0101960E94E7986EED7BE083EE92E17C
:105310000E946796CE0107960E94E798A0C2093FB7
:105320002FEF120709F00CC168EA75E0CE01019673
:105330000E94419944E650E06FEF7FEFCE01019665
:105340000E94DD5ACE0101960E94E7986AE975E055
:10535000CE0101960E94419944E650E070E060E081
:10536000CE0101960E945759CE0101960E94E798FE
:1053700086ED9DE00E940A8A4CE251E064E070E014
:10538000CE0101960E9407A580910E0D8823D1F0D1
:105390006AE776E0CE0107960E945399BE016F5FDF
:1053A0007F4FCE0107960E9401986DE776E00E943C
:1053B000EB97BC018DEA9FE00E94AC9BCE01079663
:1053C0000E94E79870E060E0CE0101960E94BF97CE
:1053D000082E000C990BC0970A9708F096C06AE84F
:1053E00076E0CE0107960E945399BE016F5F7F4F12
:1053F000CE0107960E940198BC0183EE92E10E94C3
:105400009798CE0107960E94E79889EF9FEF9093B7
:105410000D0C80930C0C0E94FB1D182F6CE875E09E
:10542000CE0107960E94419944E650E070E060E0AA
:10543000CE0107960E945759CE0107960E94E79821
:1054400086ED9DE00E940A8A48E552E065E070E042
:10545000CE0107960E9407A5BE01695F7F4FCE016E
:1054600001960E94AE98CE0107960E94E79880911F
:105470000E0D8823D1F06AE776E0CE0107960E94F0
:105480005399BE016F5F7F4FCE0107960E9401982E
:105490006DE776E00E94EB97BC018DEA9FE00E94E9
:1054A000AC9BCE0107960E94E79870E060E0CE01C9
:1054B00001960E94BF97082E000C990BC0970A977F
:1054C00020F56FE876E0CE0107960E945399BE0161
:1054D0006F5F7F4FCE0107960E940198BC0183EE5B
:1054E00092E10E949798CE0107960E94E79889EF73
:1054F0009FEF90930D0C80930C0C0E94FB1D882352
:1055000021F06FE775E0111102C068E775E0CE0188
:1055100007960E94419944E650E070E060E0CE01B9
:1055200007960E945759CE0107960E94E7986EEDA4
:105530007BE083EE92E10E946796CE010196ECCE6D
:105540006EE675E0CE0101960E94419944E650E076
:105550006FEF7FEFCE0101960E94DD5ACE010196DA
:105560000E94E7986EED7BE083EE92E10E946796E1
:10557000053F8FEF180709F044C064E976E083EE39
:1055800092E10E94679664E675E0CE0101960E9462
:10559000419944E650E06FEF7FEFCE0101960E9403
:1055A0005759CE0101960E94E7988091E712909199
:1055B000E812892B09F453C10E94FB1D882309F4CA
:1055C00059C168EC70E080E090E00E943AA164EE7E
:1055D00074E0CE0101960E94419944EF51E06FEFD3
:1055E0007FEFCE0101960E945759CE0101960E948D
:1055F000E79810930D0C00930C0CC8010E9499754C
:105600002EC1063F2FEF120749F465E176E083EEE5
:1056100092E10E9467966AE575E0B7CF013F8FEF90
:10562000180749F46EE176E083EE92E10E946796F6
:105630006BE475E0AACF023F2FEF120749F468E947
:1056400076E083EE92E10E9467966BE375E09DCF72
:10565000033F8FEF180709F04DC06FE275E0CE01F0
:1056600001960E94419944E650E06FEF7FEFCE0132
:1056700001960E94DD5ACE0101960E94E79861E2F0
:1056800075E0CE0101960E94419944E650E06FEF2B
:105690007FEFCE0101960E945759CE0101960E94DC
:1056A000E79844EF51E062E070E0CE0101960E947D
:1056B00007A5BE016F5F7F4F83EE92E10E94AE9817
:1056C000CE0101960E94E79864EA76E0CE01019649
:1056D0000E94539963EE72E1CE0101960E940198F7
:1056E000BC0183EE92E10E949798CE0101960E9440
:1056F000E7985BCF0230110509F094C065E175E0D1
:10570000CE0101960E94419944E650E06FEF7FEF91
:10571000CE0101960E94DD5ACE0101960E94E798C3
:1057200065E075E0CE0101960E94419944E650E0A3
:105730006FEF7FEFCE0101960E945759CE0101967F
:105740000E94E79844EF51E066E070E0CE010196D8
:105750000E9407A5BE016F5F7F4F83EE92E10E941A
:10576000AE98CE0101960E94E7988091E712909141
:10577000E8120597B0F070E060E083EE92E10E94DD
:10578000BF97082E000C990BC0970A9750F483EE30
:1057900092E10E94E496613523EC72078105910540
:1057A000CCF467EF74E0CE0101960E94419948EE77
:1057B00053E06FEF7FEFCE0101960E945759CE0163
:1057C00001960E94E7986EED7BE083EE92E10E94E5
:1057D0006796EBCE0E9425B620E030E048EC52E41C
:1057E0000E949DB8AB01BC0122E0CE0107960E9449
:1057F000EF9865E076E0CE0101960E945399BE01D4
:10580000695F7F4FCE0101960E940198BC0183EE33
:1058100092E10E949798CE0101960E94E798CE01EE
:105820000796C1CE6EEE74E0CE0101960E944199BA
:1058300044E650E06FEF7FEFCE0101960E9457598A
:10584000CE0101960E94E7986EED7BE083EE92E137
:105850000E9467960B3E8FEF180709F0A6CE2C9694
:105860000FB6F894DEBF0FBECDBFDF91CF911F9171
:105870000F91089568EC70E080E090E00E943AA1FA
:1058800068ED74E0CE0101960E94419944EF51E029
:105890006FEF7FEFCE0101960E9457594ECEBF9217
:1058A000CF92DF92EF92FF920F931F93CF93DF93EC
:1058B000CDB7DEB762970FB6F894DEBF0FBECDBF8F
:1058C0008C016B0162E67AE0CE010D960E9453993D
:1058D00066ED74E0C8010E94419976012FEFE21A4B
:1058E000F20AB701CE0101960E949E96BE016F5F3B
:1058F0007F4FCE0107960E944A996FEA78E0CE0169
:1059000007960E94EB97BC01C8010E946B98CE01DC
:1059100007960E94E798CE0101960E94E7988AE0D8
:10592000B82EBE9CC001BF9C900D1124FC01E15417
:10593000FE4E7F018081082E000C990B0E94B8BD9D
:10594000892B09F4B2C0B701CE0101960E94539988
:10595000BE016F5F7F4FCE0107960E944A9961E9B1
:1059600079E0CE0107960E94EB97BC01C8010E9426
:105970006B98CE0107960E94E798CE0101960E948F
:10598000E798BC9CC001BD9C900D11249C01215442
:105990003E4E7901F9016685062E000C770BCE018B
:1059A00001960E949E96BE016F5F7F4FCE010796C3
:1059B0000E944A996BEA76E0CE0107960E94EB9727
:1059C000BE01635F7F4F0E940198BC01C8010E9425
:1059D0006B98CE0107960E94E798CE0101960E942F
:1059E000E7986FEC74E0C8010E941498F70167858E
:1059F000062E000C770BCE0101960E949E96BE01EA
:105A00006F5F7F4FCE0107960E944A99BE01635F88
:105A10007F4FCE0107960E940198BC01C8010E94E9
:105A20006B98CE0107960E94E798CE0101960E94DE
:105A3000E79869EC74E0C8010E941498F701608946
:105A40007189CE0101960E949E96BE016F5F7F4FC5
:105A5000CE0107960E944A99BE01635F7F4FCE0137
:105A600007960E940198BC01C8010E946B98CE0164
:105A700007960E94E798CE0101960E94E79864EC91
:105A800074E0C8010E941498F70162897389CE01FD
:105A900001960E949E96BE016F5F7F4FC8010E94D3
:105AA0006B98CE0101960E94E798CE010D960E9458
:105AB000E798C80162960FB6F894DEBF0FBECDBF5F
:105AC000DF91CF911F910F91FF90EF90DF90CF90DA
:105AD000BF9008952F923F924F925F926F927F9264
:105AE0008F929F92AF92BF92CF92DF92EF92FF92EE
:105AF0000F931F93CF93DF93CDB7DEB768970FB6A1
:105B0000F894DEBF0FBECDBF2B013C010E94D6A78B
:105B10006D877E878F87988B83E79EE00E94FF8E3C
:105B200062E370E080E090E00E943AA161E0809141
:105B300092040E94899D60E0809190040E94899D5A
:105B400064E670E080E090E00E943AA160918C04ED
:105B500070918D0480918E0490918F040E94631542
:105B60000E9480157B018C010E94E89D4B015C0125
:105B700060E570E080E090E00E943AA16DEA76E096
:105B800085EC92E10E94679620E030E04AE754E419
:105B9000C301B2010E9484B66D8B7E8B8F8B988F70
:105BA000412C512C320160E070E0CB010E9425B6FF
:105BB0002D893E894F89588D0E941EB687FF87C167
:105BC0000E94D6A72D853E854F855889621B730B91
:105BD000840B950B0E9423B620E030E04AE754E4A2
:105BE0000E949DB8AB01BC0123E0CE0101960E944A
:105BF000EF98BE016F5F7F4F8FEB92E10E94AE98EE
:105C0000CE0101960E94E7980E948015D62EC72EDD
:105C1000382E292E0E94E89D698B7A8B8B8B9C8B6A
:105C2000DC01CB0188199909AA09BB094C015D0166
:105C300091ED891697E09906A104B104BCF020E02B
:105C400030E0A9016D2D7C2D832D922D0E94A6B9E7
:105C5000181684F426EA3BE944EC5BE36D2D7C2DB9
:105C6000832D922D0E941EB687FF10C0812C912C8F
:105C700054012EC026EA3BE944EC5BEB6D2D7C2DF4
:105C8000832D922D0E94A6B9181684F3C501B40184
:105C900028EE33E040E050E00E945BB7CA01B90152
:105CA0000E9425B64B015C019701A8016D2D7C2D4A
:105CB000832D922D0E94BEB720E030E04AE754E4E5
:105CC0000E9484B6A50194010E949DB84B015C011D
:105CD0006FEB72E1CE0101960E944A9964ED76E085
:105CE000CE0101960E94EB97BC018FEB92E10E94DE
:105CF0009798CE0101960E94E79823E04D2D5C2DE8
:105D0000632D722DCE0101960E94EF98BE016F5F48
:105D10007F4FCE0107960E944A996BEC76E0CE0148
:105D200007960E94EB97BC0189EB92E10E9497983D
:105D3000CE0107960E94E798CE0101960E94E7984F
:105D400022E0B501A401CE0107960E94EF9863ED11
:105D50007AE0CE0101960E9453996FEB72E1CE0179
:105D600001960E9401986EEC76E00E94EB9769EB39
:105D700072E10E9401986BE17BE00E94EB97BE010B
:105D8000695F7F4F0E94019862ED76E00E94EB9779
:105D9000BC0185EC92E10E946B98CE0101960E94B5
:105DA000E798CE0107960E94E79820E030E0A9012D
:105DB000C501B4010E94A6B987FD06C062E67AE07B
:105DC00089EB92E10E94619822E0B501A401CE0125
:105DD00001960E94EF98BE016F5F7F4FCE0107963C
:105DE0000E944A9962ED76E0CE0107960E94EB97F9
:105DF000BC0189EB92E10E946B98CE0107960E944C
:105E0000E798CE0101960E94E79865EC72E1CE0119
:105E100001960E944A99CE0101960E94E158CE0156
:105E200001960E94E798C301B20125E030E040E00E
:105E300050E00E945BB7672B682B692B21F56DEA58
:105E400074E0CE0101960E94419945E050E070E077
:105E500060E0CE0101960E94DD5ACE0101960E94BB
:105E6000E79869EB72E1CE0101960E944A9945E0FC
:105E700050E06FEF7FEFCE0101960E945759CE019F
:105E800001960E94E7986EED7BE085EC92E10E941E
:105E9000679662E370E080E090E00E943AA10E9481
:105EA000D6A72D853E854F855889621B730B840BC1
:105EB000950B3FEF431A530A630A730A89889A883D
:105EC000AB88BC88ED2CFC2C032D122D6FCE60E02E
:105ED000809192040E94899D68960FB6F894DEBF67
:105EE0000FBECDBFDF91CF911F910F91FF90EF902B
:105EF000DF90CF90BF90AF909F908F907F906F90EA
:105F00005F904F903F902F9008958F929F92AF9205
:105F1000BF92CF92DF92EF92FF920F931F93CF9396
:105F2000DF93CDB7DEB7EA970FB6F894DEBF0FBEAA
:105F3000CDBFF82E6EED7BE0CE01C5960E94539941
:105F40008E010B5E1F4F6F2DC8010E940C0D18872C
:105F50000F831D821E82198289E08A8381E08B83F0
:105F60008C831C8A1B8ACE0101960E94C511CE012A
:105F700001960E946810CE0101960E942AA40E810B
:105F800010E00330110509F488C163EA74E0CE0122
:105F9000C5960E9472986EED7BE085EC92E10E94BE
:105FA0006796BE016B5C7F4FCE0183960E944A9933
:105FB0004AE050E070E060E0CE0183960E94DD5A36
:105FC000CE0183960E94E79861E080E00E94318CC8
:105FD00068EF76E0CE01C5960E94679685E4C82EEC
:105FE0008CE0D82EF12CE12CE016F1060CF0F0C07C
:105FF0006E2DCE0101960E945911F6012191319129
:10600000419151916F010E94BFB74B015C01FFEFBD
:10601000EF1AFF0A20E030E04CEF52EC0E941EB66F
:1060200087FF33C0B701CE0189960E949E9667E430
:1060300078E0CE0183960E945399BE01675D7F4F41
:10604000CE0183960E94019866ED76E00E94EB9760
:10605000BC0185EC92E10E946B98CE0183960E9470
:10606000E798CE0189960E94E7980130110509F062
:1060700055C081E0E816F10409F0B6CF65EC72E195
:10608000CE01C5960E949798AFCF22E0B501A4013A
:10609000CE018F960E94EF98B701CE0189960E949B
:1060A0009E9667E478E0CE0183960E945399BE01E4
:1060B000675D7F4FCE0183960E9401986CE679E080
:1060C0000E94EB97BE01615D7F4F0E940198BC0169
:1060D00089EB92E10E949798CE0183960E94E798FF
:1060E000CE0189960E94E798CE018F960E94E7988C
:1060F00069EB72E1CE0183960E944A9962E67AE0EA
:10610000CE0183960E94EB97BC0185EC92E10E9440
:106110006B98CE0183960E94E798A7CF02301105B5
:1061200011F522E0B501A401CE0183960E94EF98FB
:10613000BE016D5D7F4FCE0189960E944A9962E64D
:106140007AE0CE0189960E94EB97BC01CE01C596FC
:106150000E946B98CE0189960E94E798CE018396A3
:106160000E94E79841CF0330110509F43DCF69EB58
:1061700072E1CE0183960E944A9944E150E06FEFAC
:106180007FEFCE0183960E945759CE0183960E94DD
:10619000E79863ED75E0CE0183960E945399CE0196
:1061A00083960E943959CE0183960E94E798809188
:1061B0008904882309F418CF8091E904882309F41D
:1061C00013CF60ED77E080E090E00E943AA10CCF21
:1061D000CE01C5960E94EF9685EC92E10E94EF9663
:1061E0000115110579F560E974E085EC92E10E94F2
:1061F000729865E874E0CE0183960E9441994AE066
:1062000050E06FEF7FEFCE0183960E945759CE0189
:1062100083960E94E798CE01C5960E94E798EA9679
:106220000FB6F894DEBF0FBECDBFDF91CF911F91A7
:106230000F91FF90EF90DF90CF90BF90AF909F9025
:106240008F900895043011050CF5BE016B5C7F4FF3
:10625000CE0183960E944A994AE050E06FEF7FEFAB
:10626000CE0183960E945759CE0183960E94E798EB
:1062700063ED75E0CE0183960E945399CE0183961B
:106280000E943959CE0183960E94E79862EE76E02B
:1062900085EC92E10E946198BECF65EF76E0CE0179
:1062A000C5960E946796BE016B5C7F4FCE018396B8
:1062B0000E944A994AE050E070E060E0CE01839687
:1062C0000E94DD5ACE0183960E94E7986EED7BE036
:1062D00085EC92E10E94679665EC72E1CE01C5966D
:1062E0000E94979810E000E0602FCE0101960E9476
:1062F00059116B017C0122E0BC01A601CE018396FD
:106300000115110509F077C00E94EF98BE016D5D7F
:106310007F4F8CEC93E10E949E9BCE0183960E945E
:10632000E79822E0B701A601CE0183960E94EF987C
:10633000BE016D5D7F4FCE0189960E944A9962E64B
:106340007AE0CE0189960E94EB97BC0185EC92E140
:106350000E946B98CE0189960E94E798CE018396A1
:106360000E94E7980F5F1F4F0330110509F0BCCF63
:10637000CE01C5960E94EF96BE016B5C7F4FCE01A9
:1063800083960E944A994AE050E06FEF7FEFCE017A
:1063900083960E945759CE0183960E94E79863ED39
:1063A00075E0CE0183960E945399CE0183960E9498
:1063B0003959CE0183960E94E79885EC92E10E94BC
:1063C000EF966BEF76E0CE0183960E94539965ECD1
:1063D00072E1CE0183960E94019862EE76E00E94FF
:1063E000EB97BC0185EC92E10E949798CE018396D1
:1063F0000E94E79810CF0E94EF98BE016D5D7F4F1D
:10640000CE0189960E944A9962E67AE0CE01899689
:106410000E94EB97BC01CE01C5960E946B98CE01FD
:1064200089960E94E79879CF8F929F92AF92BF9200
:10643000CF92DF92EF92FF920F931F93CF93DF9350
:10644000CDB7DEB768970FB6F894DEBF0FBECDBFED
:106450006C0180919E1190919F110197C9F06EED92
:106460007BE0C6010E945399C60168960FB6F89466
:10647000DEBF0FBECDBFDF91CF911F910F91FF9077
:10648000EF90DF90CF90BF90AF909F908F90089546
:1064900065E077E0CE010D960E945399BE01635FDF
:1064A0007F4F86ED9DE00E949E9B6CE271E080E054
:1064B00090E00E943AA1CE0143960E943B6F64E6B1
:1064C00070E080E090E00E943AA110E000E085E0FA
:1064D000A82EB12C9AE0892E912C60E177E0CE01B4
:1064E00001960E945399BE016F5F7F4FCE01439684
:1064F0000E94A4977C01CE0101960E94E798A70113
:106500004F5F5F4FBE016D5E7F4FCE0101960E94CF
:10651000275ABE016F5F7F4FCE010D960E94AE9845
:10652000CE0101960E94E79889899A89892B09F101
:1065300070E060E0CE010D960E94BF97082E000C1F
:10654000990BC0970A97A8F462E177E0CE01019613
:106550000E945399BE016F5F7F4FCE010D960E943E
:10656000D097E82ECE0101960E94E798FF24F3947D
:10657000E110F12C64EB74E0CE0101960E94419988
:1065800044E150E06FEF7FEFCE0101960E94335A55
:10659000CE0101960E94E7980F5F1F4F62E370E003
:1065A00080E090E00E943AA1C801B5010E9435BB8D
:1065B0000197C1F4CE0101960E94EE6D8D819E81FE
:1065C000892B09F46AC0BE016F5F7F4F83EE92E1B1
:1065D0000E9497980E94C44CFF24F394CE01019628
:1065E0000E94E798CE0101960E943B6FBE016F5F4B
:1065F0007F4FCE0143960E94AE98CE0101960E9435
:10660000E79862E370E080E090E00E943AA10436EF
:10661000110519F0FF2009F460CF80910E0D882339
:10662000F1F066ED75E0CE0101960E945399BE012E
:10663000635F7F4FCE0101960E940198BC01CE019D
:1066400007960E944A99CE0107960E94E158CE0112
:1066500007960E94E798CE0101960E94E7988989E3
:106660009A89892B61F070E060E0CE010D960E945E
:10667000BF97082E000C990BC0970A9738F16AE172
:1066800077E0C6010E945399CE0143960E94E79895
:10669000CE010D960E94E798E7CE043111050CF467
:1066A0009DCFC801B4010E9435BB892B09F096CF5C
:1066B000BE01635F7F4F86ED9DE00E949E9B68EC6C
:1066C00070E080E090E00E943AA188CF62E177E03C
:1066D000CE0101960E945399BE016F5F7F4FCE019C
:1066E0000D960E94D097182FCE0101960E94E79830
:1066F0001111C5CFBE01635F7F4FC6010E9438995B
:10670000C3CF2F923F924F925F926F927F928F9260
:106710009F92AF92BF92CF92DF92EF92FF920F9330
:106720001F93CF93DF93CDB7DEB76D970FB6F89475
:10673000DEBF0FBECDBF61E089E10E94899D61E0AF
:1067400089E10E945B9D0E94B99566E277E08DEA3F
:106750009FE00E94119AF12CE12C17E2812F0E94F8
:10676000168C0E94FD9E811195C162E377E08DEA4F
:106770009FE00E949C9B40E150E0612F8DEA9FE0EA
:106780000E94FA991093D0136EE477E08DEA9FE0AF
:106790000E949C9B40E150E0612F8DEA9FE00E94A7
:1067A000FA992FEFE21AF20A1F5F1034B9F663E884
:1067B00077E0EF2811F069E977E08DEA9FE00E9429
:1067C000119A0E946CA780E40E94208C0EEC14E0C9
:1067D000D8016D918D018CEC93E10E949D12B4E083
:1067E000063D1B07A9F70E9415590E94D4158EE497
:1067F00092E00E9445B78093350D8FE492E00E94AD
:1068000045B78093360D8091350D9091360D181651
:10681000190664F41092CD04019741F41092360DDC
:106820001092350D8EE492E00E94338E6BED7BE08A
:10683000CE0101960E9441994AE050E06FEF7FEF50
:10684000CE0101960E94DD5ACE0101960E94E79882
:1068500040E052EC61E070E08DEA9FE00E94E35975
:106860008091CD04882331F068EE73E080E090E001
:106870000E943AA18DEA9FE00E9445898B8B6FEBC5
:10688000E62E61E1F62E0CE211E0C8010E9445B748
:10689000F70181937F010F5F1F4F0632F2E01F0760
:1068A000A1F78091C011181624F42B892D3609F018
:1068B00021C16EED7BE0CE010D960E94539910929E
:1068C000BF1188E18093C01184E08093C1111092C0
:1068D000C6111092C7116BE17AE0CE010D960E94AD
:1068E000679689EC91E1009739F044E050E0BC01F3
:1068F000CE010D960E94B28E81E08093CD1183E08F
:106900008093CE1182E090E09093D0118093CF11CC
:1069100085E090E09093D2118093D11168E17AE004
:10692000CE010D960E94679683ED91E1009739F0B4
:1069300044E050E0BC01CE010D960E94B28E82E090
:106940008093D71183E08093D81182E090E09093F8
:10695000DA118093D91185E090E09093DC11809357
:10696000DB1165E17AE0CE010D960E9467968DED10
:1069700091E1009739F044E050E0BC01CE010D9662
:106980000E94B28E83E08093E1118093E21182E055
:1069900090E09093E4118093E31185E090E0909370
:1069A000E6118093E51160EA77E0CE010D960E9432
:1069B000679687EE91E1009739F044E050E0BC0122
:1069C000CE010D960E94B28E85EF8093EB1183E08D
:1069D0008093EC1182E090E09093EE118093ED11A2
:1069E00085E090E09093F0118093EF118CE291E0BC
:1069F0000E94D58E80910E0D882311F1CE01019653
:106A00000E94B71CBE016F5F7F4F8DEA9FE00E941E
:106A1000AC9BCE0101960E94E79868E17AE08DEA8E
:106A20009FE00E94BE9B2AE04AE050E060E070E0F8
:106A30008DEA9FE00E94AA998DEA9FE00E94F69954
:106A40006EED79E0CE0107960E944199BE01695F23
:106A50007F4F8DEA9FE00E94AC9B10E000E08091A8
:106A6000C111082E000C990B0817190724F5B8015D
:106A7000CE0101960E944F2CBE016F5F7F4F8DEAC1
:106A80009FE00E94AC9BCE0101960E94E7980F5FA9
:106A90001F4FE5CF843009F087CE68E677E08DEAB6
:106AA0009FE00E949C9B40E150E0612F8DEA9FE0B7
:106AB0000E94FA9979CECE0107960E94E7988091BC
:106AC0000E0D882399F068EF79E08DEA9FE00E942F
:106AD000BE9B2AE04AEF50E060E070E08DEA9FE064
:106AE0000E94AA998DEA9FE00E94F699CE010D9628
:106AF0000E94E7988091C81181118091BF11809305
:106B0000BA110E94D6A76093B6117093B711809303
:106B1000B8119093B9113B8910E0323709F499C547
:106B200058E2252E51E1352E710110E000E0C80138
:106B30000E9445B7D7018D937D010F5F1F4F083825
:106B40001105A9F78091281190912911A0912A117E
:106B5000B0912B1185369105A105B1050CF49BC1AF
:106B60008093C9049093CA04A093CB04B093CC043F
:106B700080912C1190912D11A0912E11B0912F1177
:106B80008093C5049093C604A093C704B093C8042F
:106B90008091301190913111A0913211B091331147
:106BA0008093C1049093C204A093C304B093C4041F
:106BB00064E471E1CE0101960E945399BE016F5FBA
:106BC0007F4F8AEB93E10E94AE98CE0101960E941E
:106BD000E79862EA71E1CE0101960E945399BE01E5
:106BE0006F5F7F4F84EB93E10E94AE98CE010196D8
:106BF0000E94E79823E030E050E040E06AEB73E168
:106C0000CE0107960E94649923E030E050E040E016
:106C100064EB73E1CE0101960E9464992D813E815F
:106C20008B859C852817390709F589819A816F81A1
:106C30007885009759F06115710509F0F1C0232B93
:106C400009F4F1C0DC018C9190E00DC06115710573
:106C500009F4E9C0232B09F4E6C0FB01808190E030
:106C600091958195910911E0892B09F010E0CE01F1
:106C700001960E94E798CE0107960E94E7981111AD
:106C800006C06AEB73E184EB93E10E9497988091D0
:106C9000341190913511A0913611B0913711809334
:106CA000BD049093BE04A093BF04B093C004809130
:106CB000381190913911A0913A11B0913B11809304
:106CC000B9049093BA04A093BB04B093BC04809120
:106CD0003C1190913D11A0913E11B0913F118093D4
:106CE000B5049093B604A093B704B093B804809110
:106CF000401190914111A0914211B09143118093A4
:106D0000B1049093B204A093B304B093B404E0919F
:106D1000A011F091A111FD8FEC8FF093D704E093B7
:106D2000D60480915C1190915D11A0915E11B0919B
:106D30005F118C8B9D8BAE8BBF8B8093DC0490930B
:106D4000DD04A093DE04B093DF0480917211909172
:106D50007311A0917411B0917511888F998FAA8FBA
:106D6000BB8F8093D8049093D904A093DA04B09396
:106D7000DB0440904C1150904D1160904E1170907A
:106D80004F114092AD045092AE046092AF047092E5
:106D9000B0048090501190905111A0905211B09079
:106DA00053118092A9049092AA04A092AB04B092CD
:106DB000AC040091AE111091AF11B801012E000C7E
:106DC000880B990B0E9425B66B017C01AC019B01DD
:106DD0000E940BBB811104C01093110C0093100C86
:106DE000209197043091980490E080E028173907AB
:106DF000E4F0D101D8964D915C91D99757FF0BC023
:106E0000FC01EE0FFF1FE956FB4F40815181D996DF
:106E10005C934E93D8970196B2E02B0E311CE6CFCF
:106E20000E94E2BD20CF11E022CFA3019201C30155
:106E3000B2010E940BBB811109C0A5019401C501DB
:106E4000B4010E940BBB882309F472C30E94380D61
:106E500036E7A32E31E1B32E05E41CE0D501CD9039
:106E6000DD90ED90FD905D01A7019601C701B6018F
:106E70000E940BBB811105C0F801C082D182E28261
:106E8000F3820C5F1F4FFCE00D361F0739F781E0DE
:106E900090E00E948B0D1B891257113009F4D9C361
:106EA0002B892E3609F4D4C3809128119091291191
:106EB000A0912A11B0912B1185369105A105B1053C
:106EC0000CF4C7C380919E1190919F118D7F892BE7
:106ED00041F440E855E260E070E086ED9DE00E94FC
:106EE000E35980919E1190919F11019741F440E0E8
:106EF00052EC61E070E086ED9DE00E94E35964E6AB
:106F000070E080E090E00E943AA180919E11909103
:106F10009F11892B09F0B8C02B892E3671F0809112
:106F2000281190912911A0912A11B0912B11853629
:106F30009105A105B1050CF0A7C06EED7BE0CE0177
:106F400007960E94539968EA77E0CE0101960E9465
:106F5000539964EB73E1CE0101960E940198BC0144
:106F6000CE0107960E949798CE0101960E94E7985D
:106F7000BE01695F7F4F86ED9DE00E949E9B68EB9E
:106F80007BE080E090E00E943AA1BE01695F7F4F04
:106F9000CE0101960E944A99CE0101960E94DF5CC3
:106FA000CE0101960E94E7986CE271E080E090E0EB
:106FB0000E943AA14091B8135091B913425051091F
:106FC00064EB73E1CE0101960E94275ABE016F5F08
:106FD0007F4FCE0107960E94AE98CE0101960E9487
:106FE000E798BE01695F7F4FCE0101960E944A99E2
:106FF000BE01695F7F4FCE0101960E940198BC01DE
:10700000CE0107960E949798CE0101960E94E798BC
:1070100060EB77E0CE0101960E945399BE01695F53
:107020007F4FCE0101960E940198BC01CE010796C8
:107030000E949798CE0101960E94E798BE01695F71
:107040007F4F86ED9DE00E949E9B68EB7BE080E099
:1070500090E00E943AA1BE01695F7F4FCE01019688
:107060000E944A99CE0101960E94DF5CCE010196F2
:107070000E94E7986CE271E080E090E00E943AA103
:10708000CE0107960E94E79864E670E080E090E009
:107090000E943AA1F89482E08093B0008093B100FE
:1070A00094E69093B3001092B200809370007894AD
:1070B00080935610109259108091571060E00E94F2
:1070C000899D65EB7BE0CE0101960E9441994AE0E3
:1070D00050E06FEF7FEFCE0101960E94DD5ACE01A6
:1070E00001960E94E7986EED7BE085EC92E10E94AC
:1070F000679680919E1190919F11892B31F46CE6D7
:1071000076E085EC92E10E94679680919E119091C5
:107110009F11019731F466E676E085EC92E10E94DA
:10712000679680919E1190919F11029731F460E7CC
:1071300076E085EC92E10E9467968091C912909169
:10714000CA12892BC1F064EB73E185EC92E10E94D5
:107150006B9865EC72E1CE0101960E944A994AE073
:1071600050E06FEF7FEFCE0101960E945759CE019C
:1071700001960E94E79880919E1190919F1101972E
:1071800009F05CC0CE0107960E9414328B859C8565
:10719000009709F449C0EF81F8852081222309F482
:1071A00043C0079708F440C062EA7BE085EC92E1B7
:1071B0000E947298BE01695F7F4F85EC92E10E9448
:1071C0006B9865EC72E1CE0101960E944A99CE015E
:1071D00001960E94E158CE0101960E94E79869E964
:1071E0007BE0CE0101960E94419948EC50E06FEFA0
:1071F0007FEFCE0101960E94335ACE0101960E9484
:10720000E798BE01695F7F4FCE0101960E944A99BF
:1072100048EC50E06FEF7FEFCE0101960E94575986
:10722000CE0101960E94E79868EE73E080E090E05E
:107230000E943AA1CE0107960E94E7986DE77BE095
:1072400085EC92E10E94729866ED75E0CE010196A0
:107250000E94539964EB73E1CE0101960E9401985C
:1072600065EC72E10E940198BC0185EC92E10E94FC
:107270009798CE0101960E94E79865EC72E1CE01E5
:1072800001960E944A99CE0101960E94E158CE01D2
:1072900001960E94E7986EED7BE085EC92E10E94FA
:1072A000679664E670E080E090E00E943AA10E9458
:1072B000B99564E670E080E090E00E943AA183E234
:1072C0000E94168C81E090E00E94118C0E94FD9E2D
:1072D00083E090E090930F0C80930E0C8CE40E945E
:1072E00014A86B017C0162E370E080E090E00E94F2
:1072F0003AA1A7019601C701B6010E940BBB8823E2
:10730000B9F086E60E9414A86B017C0162E370E08C
:1073100080E090E00E943AA1A7019601C701B60162
:107320000E940BBB882321F010920F0C10920E0CC0
:1073300080910E0C90910F0C039709F08CC268E6B7
:107340007BE0CE0101960E944199CE0101960E94F8
:10735000DF5CCE0101960E94E79883E08093E912FA
:107360000E94B99580ED0E94EB9F853509F096C289
:107370008AEA0E9408A09093EB128093EA128CEAAA
:107380000E9408A09093ED128093EC128EEA0E9466
:1073900008A09093EF128093EE1280EB0E9408A059
:1073A0009093FB128093FA1282EB0E9408A09093B4
:1073B000FD128093FC1284EB0E9408A09093FF12B0
:1073C0008093FE1286EB0E9408A09093F1128093A6
:1073D000F01288EB0E9408A09093F3128093F212AF
:1073E0008AEB0E9408A09093F5128093F4128CEB24
:1073F0000E9408A09093F7128093F6128EEB0E94E1
:1074000008A09093F9128093F8126FE27BE085EC6C
:1074100092E10E9472980E94DAA10E9425B60E9411
:1074200049B90E9425B620E030E048EC52E40E94C1
:107430009DB8AB01BC0122E0CE0101960E94EF98FD
:10744000BE016F5F7F4FCE0107960E944A9969E0A7
:1074500076E0CE0107960E94EB97BC0185EC92E1A5
:107460000E946B98CE0107960E94E798CE01019684
:107470000E94E79865EC72E1CE0101960E944A995C
:10748000CE0101960E94DF5CCE0101960E94E79832
:1074900069E17BE085EC92E10E9472986091C904F9
:1074A0007091CA048091CB049091CC040E9425B6BF
:1074B00020E030E048EC52E40E949DB8AB01BC01F2
:1074C00022E0CE0101960E94EF98BE016F5F7F4FD0
:1074D000CE0107960E944A9969E076E0CE010796B0
:1074E0000E94EB97BC0185EC92E10E946B98CE0163
:1074F00007960E94E798CE0101960E94E79865ECF6
:1075000072E1CE0101960E944A99CE0101960E9435
:10751000DF5CCE0101960E94E7983B89313609F085
:107520004EC281E00E940B5D81E00E94C562C6C12F
:1075300000915411602F002E000C770B880B990BD3
:107540000E9425B69B01AC010E940BBB81117ECC31
:107550006090551170905611B301072C000C880BE8
:10756000990B0E9425B69B01AC010E940BBB8111B7
:107570006DCC10915711612F012E000C770B880BE9
:10758000990B0E9425B69B01AC010E940BBB811197
:107590005DCC8090581190905911A0905A11B090E4
:1075A0005B11A5019401C501B4010E940BBB8111BF
:1075B0004DCC2C893D894E895F89CA01B9010E9451
:1075C0000BBB811143CC288D398D4A8D5B8DCA014F
:1075D000B9010E940BBB811139CC60919E11709151
:1075E0009F11072E000C880B990B0E9425B69B015A
:1075F000AC010E940BBB811129CCEC8DFD8DBF012C
:10760000FF0F880B990B0E9425B69B01AC010E94CD
:107610000BBB81111BCCA7019601C701B6010E94CB
:107620000BBB811113CC04300CF010CC15300CF0D6
:107630000DCCFBEF6F1671040CF008CC20E030E0AD
:10764000A901C501B4010E941EB687FDFFCB00CC85
:107650001CEF8091C9049091CA04A091CB04B09111
:10766000CC048093281190932911A0932A11B093F0
:107670002B118091C5049091C604A091C704B091CC
:10768000C80480932C1190932D11A0932E11B093C8
:107690002F118091C1049091C204A091C304B091B4
:1076A000C4048093301190933111A0933211B093A0
:1076B00033113B89333751F160E08AEB93E10E944B
:1076C0003E9860E084EB93E10E943E984091BE13A7
:1076D0005091BF134115510549F084E491E10097A1
:1076E00029F0BC018AEB93E10E94B28E4091B8135D
:1076F0005091B9134115510549F082EA91E1009783
:1077000029F0BC0184EB93E10E94B28E8091BD040C
:107710009091BE04A091BF04B091C0048093341135
:1077200090933511A0933611B09337118091B9041D
:107730009091BA04A091BB04B091BC04809338111D
:1077400090933911A0933A11B0933B118091B504F5
:107750009091B604A091B704B091B80480933C1105
:1077600090933D11A0933E11B0933F118091B104CD
:107770009091B204A091B304B091B40480934011ED
:1077800090934111A0934211B093431190E080E097
:107790000E94888EE5E4FCE0A6E7B1E18DE69CE07E
:1077A00041915191619171914D935D936D937D9351
:1077B0008E179F07A9F765EC7BE0CE0101960E942A
:1077C0004199CE0101960E94DF5CCE0101960E9494
:1077D000E79897E9C92E94E0D92E20E6A22E21E160
:1077E000B22EF12CE12C80919704909198048E1583
:1077F0009F054CF1D6018D919D916D01F50181930D
:1078000091935F0180910E0D8823C9F066ED75E0BC
:107810008DEA9FE00E949C9B4AE050E0B7018DEA10
:107820009FE00E944F9B63EA77E08DEA9FE00E9411
:107830009C9BF6013297808191810E94899BFFEF8A
:10784000EF1AFF0AD0CF123008F03CCB90E080E076
:107850000E94888E37CB86E00E9415A1BC0190E083
:1078600080E00E9423B62AE037ED43EA5CE30E9401
:1078700084B623E333E948E853E40E94BEB720E02E
:1078800030E048E453E40E941EB687FF66CD82E0F4
:1078900090E090939604809395045FCD62E47BE042
:1078A000CE0101960E944199CE0101960E94E158B5
:1078B000CE0101960E94E7981092940464E670E06D
:1078C00080E090E00E943AA180910E0C90910F0C04
:1078D000892BA1F461E0809192040E94899D60E06F
:1078E000809190040E94899D60918C0470918D0418
:1078F00080918E0490918F040E94631560E08091C6
:1079000092040E94899D8091CD04882331F068EE15
:1079100073E080E090E00E943AA168E17AE081EDB6
:1079200092E10E94679682E090E090930D0C809324
:107930000C0C8091CD04882309F494C16FED7AE09A
:10794000CE0101960E9441994CE251E06FEF7FEF2A
:10795000CE0101960E945759CE0101960E94E798E8
:1079600060918A0470918B048091D6049091D70421
:107970000E94A45684E1C82ED12CE12CF12C10E0F9
:1079800000E00F5F1F4FC701B6010E943AA160914E
:107990008A0470918B048091D6049091D7040E9440
:1079A000A456033011052CF00A301105DCF4892BA4
:1079B000E1F044E1C40ED11CE11CF11CE2CF8DEAE0
:1079C0009FE00E944589182F64E670E080E090E017
:1079D0000E943AA1113609F4A4CD80E00E940B5D0B
:1079E00080E0A3CD892B09F0EDC18091D604909160
:1079F000D7048B30910509F095C1809123139091A4
:107A00002413A0912513B09126138093080C909312
:107A1000090CA0930A0CB0930B0C80911F1390914A
:107A20002013A0912113B09122138093040C909302
:107A3000050CA093060CB093070C4091080C5091D4
:107A4000090C60910A0C70910B0C21E0CE0101969B
:107A50000E94EF9868EF76E0CE0107960E94539956
:107A6000BE016F5F7F4FCE0107960E940198BC0157
:107A700085EC92E10E949798CE0107960E94E798C4
:107A8000CE0101960E94E7984091040C5091050C9C
:107A90006091060C7091070C21E0CE0101960E94C6
:107AA000EF9867EB77E0CE0107960E945399BE01ED
:107AB0006F5F7F4FCE0107960E940198BC0185EC55
:107AC00092E10E946B98CE0107960E94E798CE0142
:107AD00001960E94E79861E47BE085EC92E10E94C8
:107AE00061986EED7BE0CE0101960E94539944E1CE
:107AF00050E070E060E0CE0101960E94DD5ACE01B8
:107B000001960E94E798C090080CD090090CE09074
:107B10000A0CF0900B0C20E030E0A901C701B6017F
:107B20000E94A6B920E030E040E05FE387FD1AC183
:107B3000C701B6010E94BFB70E9449B9AB01BC01A1
:107B4000CE0101960E947196BE016F5F7F4F8FEB51
:107B500092E10E94AE98CE0101960E94E79860E003
:107B600087E00E94318C6FEB72E18CEC93E10E9414
:107B70009E9B6FED8CEC93E10E94239A6DEB77E076
:107B80008CEC93E10E949C9B6091040C7091050C1D
:107B90008091060C9091070C0E9449B94AE050E090
:107BA0008CEC93E10E944F9B61E47BE08CEC93E1D1
:107BB0000E949C9B64E670E080E090E00E943AA105
:107BC000C090080CD090090CE0900A0CF0900B0CBF
:107BD00020E030E040EF51E4C701B6010E94A6B9B1
:107BE00060ED7AE087FF28C020E030E040ED51E40E
:107BF000C701B6010E94A6B987FDB9C060EC7AE062
:107C0000CE0101960E9441994AE050E06FEF7FEF6C
:107C1000CE0101960E945759CE0101960E94E79825
:107C20008091CD04882331F06CED75E080E090E028
:107C30000E943AA160EB7AE0CE0101960E94419940
:107C40004AE050E06FEF7FEFCE0101960E94575956
:107C5000CE0101960E94E79862E370E080E090E038
:107C60000E943AA161E07BE085EC92E10E9472986B
:107C700066ED75E0CE0101960E94539964EB73E1C5
:107C8000CE0101960E94019865EC72E10E94019874
:107C9000BC0185EC92E10E949798CE0101960E946A
:107CA000E79865EC72E1CE0101960E944A99CE01F7
:107CB00001960E94E158CE0101960E94E7986DEE70
:107CC0007AE085EC92E10E94729865EC72E1CE0157
:107CD00001960E944A99CE0101960E94E158CE0178
:107CE00001960E94E7986EED7BE085EC92E10E94A0
:107CF00067966D960FB6F894DEBF0FBECDBFDF91CD
:107D0000CF911F910F91FF90EF90DF90CF90BF9098
:107D1000AF909F908F907F906F905F904F903F902B
:107D20002F9008958631910509F467CE0C9709F0DC
:107D300084CE8091FB0B9091FC0BA091FD0BB09138
:107D4000FE0B8093080C9093090CA0930A0CB0933F
:107D50000B0C8091F70B9091F80BA091F90BB0915F
:107D6000FA0B63CEC701B6010E94BEB7E5CE20E094
:107D700030E040EB51E4C701B6010E94A6B962EAC7
:107D80007AE087FF59CF63E97AE0CE0101960E943D
:107D900041994AE050E06FEF7FEFCE0101960E94DB
:107DA0005759CE0101960E94E7988091CD0488230F
:107DB00031F06CED75E080E090E00E943AA165E85A
:107DC0007AE03ACF0E9415596EE170E080E090E0D1
:107DD0000E943AA10E9485A16B017C0164E670E0DB
:107DE00080E090E00E943AA168EF76E085EC92E1B5
:107DF0000E94679621E0B701A601CE0101960E947C
:107E0000EF98BE016F5F7F4F85EC92E10E946B9807
:107E1000CE0101960E94E79865EC72E1CE010196D1
:107E20000E944A994AE050E070E060E0CE0101967D
:107E30000E94DD5ACE0101960E94E7988091890444
:107E4000882379F08091E904882359F06FED8CEC58
:107E500093E10E94239A63ED75E08CEC93E10E941C
:107E60009C9B62ED75E085EC92E10E946198C09266
:107E7000080CD092090CE0920A0CF0920B0C20E056
:107E800030E040EF51E4C701B6010E94A6B965E7B2
:107E90007AE087FF28C020E030E040ED51E4C701E0
:107EA000B6010E94A6B987FD3EC065E67AE0CE0124
:107EB00001960E9441994AE050E06FEF7FEFCE01BA
:107EC00001960E945759CE0101960E94E798809131
:107ED000CD04882331F06CED75E080E090E00E94E5
:107EE0003AA165E57AE0CE0101960E9441994AE007
:107EF00050E06FEF7FEFCE0101960E945759CE01FF
:107F000001960E94E7986CE271E080E090E00E94A8
:107F10003AA18091CD04882309F4A4CE68EE73E0E1
:107F200080E090E09DCE20E030E040EB51E4C701DE
:107F3000B6010E94A6B967E47AE087FFD4CF68E370
:107F40007AE0CE0101960E9441994AE050E06FEF3D
:107F50007FEFCE0101960E945759CE0101960E94F3
:107F6000E7988091CD04882331F06CED75E080E0D6
:107F700090E00E943AA16AE27AE0B5CF2F923F9258
:107F80004F925F926F927F928F929F92AF92BF9229
:107F9000CF92DF92EF92FF920F931F93CF93DF93D5
:107FA000CDB7DEB7E6970FB6F894DEBF0FBECDBFF4
:107FB00063EE72E18DED92E10E9497980E945096D7
:107FC00060EC77E0CE0101960E945399BE016F5F8D
:107FD0007F4F8DED92E10E94D097182FCE01019630
:107FE0000E94E798112309F48FC026E030E045E0B5
:107FF00050E063EE72E1CE0101960E946499BE01E9
:108000006F5F7F4F8FEB92E10E94AE98CE01019699
:108010000E94E7988FEB92E10E94E4966B016CE678
:1080200079E0CE0101960E945399BE016F5F7F4FA8
:1080300083EE92E10E949A97AC014F5F5F4F63EE2F
:1080400072E1CE010B960E94275ABE01655F7F4FF9
:108050008FEB92E10E94AE98CE010B960E94E798BA
:10806000CE0101960E94E7988FEB92E10E94E49680
:108070009B01E7E9F4E041E050E0A0919704B09162
:108080009804A417B5075CF0A281B381A217B307C7
:1080900011F4138212824F5F5F4F3296EECFF601DA
:1080A000EE0FFF1FE956FB4F7183608382E090E083
:1080B0000E948B0D63EE72E1CE0101960E944A99F7
:1080C000CE0101960E94DF5CCE0101960E94E798E6
:1080D00090E080E00E94888E1092EE041091EE04F1
:1080E000112311F40C94C24C63EE72E1CE0101969F
:1080F0000E944A99CE0101960E94DF5CCE01019652
:108100000E94E7980C947A4A66EC77E0CE010196DB
:108110000E945399BE016F5F7F4F8DED92E10E94E7
:10812000D097182FCE0101960E94E7981123F1F005
:10813000E7E9F4E081E090E0209197043091980421
:108140002817390774F0863091052CF493838283C5
:1081500001963296F1CF9C012E5F3F4F33832283ED
:10816000F7CF82E090E00E948B0DB2CF6CEC77E00D
:10817000CE0101960E945399BE016F5F7F4F8DED36
:1081800092E10E94D097182FCE0101960E94E798A5
:108190001123D1F08091350D9091360D892B81F40A
:1081A00081E090E09093360D8093350D8EE492E05F
:1081B0000E94338E68EC70E080E090E00E943AA16B
:1081C000F0E0E0E019958ACF63ED77E0CE0101960B
:1081D0000E945399BE016F5F7F4F8DED92E10E9427
:1081E000D097182FCE0101960E94E798112399F19C
:1081F0006BED77E0CE0101960E94539960EC73E13C
:10820000CE0101960E940198BC0185EC92E10E948A
:108210009798CE0101960E94E79866ED75E0CE0131
:1082200001960E94539965EC72E1CE0101960E947D
:108230000198BC01CE010B960E944A99CE010B9683
:108240000E94E158CE010B960E94E798CE0101965C
:108250000E94E79841CF65EE77E0CE0101960E943B
:108260005399BE016F5F7F4F8DED92E10E94D097D1
:10827000182FCE0101960E94E798112369F069E555
:1082800079E085EC92E10E94729864EB73E185ECF1
:1082900092E10E946B98C1CF6CEE77E0CE0101961F
:1082A0000E945399BE016F5F7F4F8DED92E10E9456
:1082B000D097182FCE0101960E94E798112309F15B
:1082C00066E379E085EC92E10E94729865EC72E1D8
:1082D000CE0101960E944A99CE0101960E94E15872
:1082E000CE0101960E94E7980E94380D1092EE048C
:1082F00062EF77E083EE92E10E9467960E94C44CA1
:10830000EDCE66EF77E0CE0101960E945399BE0153
:108310006F5F7F4F8DED92E10E94D097182FCE01B5
:1083200001960E94E798112309F495C06CE679E064
:10833000CE0101960E945399BE016F5F7F4F83EE7D
:1083400092E10E949A97AC014F5F5F4F63EE72E13A
:10835000CE010B960E94275ABE01655F7F4F8FEBBF
:1083600092E10E94AE98CE010B960E94E798CE0152
:1083700001960E94E7988FEB92E10E94E4968B01B0
:1083800069E279E085EC92E10E9472988091BF11D8
:10839000882331F06DE179E085EC92E10E947298DA
:1083A0000115110559F465EC72E1CE0101960E94A8
:1083B0004A99CE0101960E94E15804C7CE01019668
:1083C0000E94B71CCE0101960E94E158CE01019691
:1083D0000E94E798023011050CF47ECE6EED79E034
:1083E000CE010B960E944199BE01655F7F4FCE0181
:1083F00001960E944A99CE0101960E94E158CE0151
:1084000001960E94E798F12CE12C8091C111082E71
:10841000000C990BE816F9068CF4B701CE01019611
:108420000E944F2CCE0101960E94E158CE01019688
:108430000E94E798FFEFEF1AFF0AE7CFCE010B96F5
:108440000E94E7980230110509F446CE8CE291E0D3
:108450000E94D58E41CE6DEF77E0CE0101960E944D
:108460005399BE016F5F7F4F8DED92E10E94D097CF
:10847000182FCE0101960E94E798112309F482C3B8
:1084800063EE72E1CE018F960E944A996CE679E024
:10849000CE0101960E945399BE016F5F7F4FCE01BE
:1084A0008F960E949A97AC014F5F5F4FBE01615D4E
:1084B0007F4FCE0189960E94275ACE0101960E94D5
:1084C000E798BE01615D7F4FCE0101960E944A99F7
:1084D000CE0101960E94DF5CCE0101960E94E798D2
:1084E00061E078E0CE0101960E945399BE016F5F72
:1084F0007F4FCE0189960E94A4978C01CE010196F0
:108500000E94E7986EED7BE0CE0183960E9453991E
:108510006EED7BE0CE014D960E9453991016110628
:108520000CF099C1A8014F5F5F4F8DA59EA548171C
:10853000590790F4BE01675D7F4FCE0101960E94FE
:10854000275ABE016F5F7F4FCE0183960E94AE987F
:10855000CE0101960E94E798980150E040E0BE01EC
:10856000675D7F4FCE0101960E946499BE016F5FE7
:108570007F4FCE014D960E94AE98CE0101960E948B
:10858000E79889A19AA1892B09F418C2CE014D96CA
:108590000E94E4966B0121E0C21AD108860138E1FD
:1085A000C316D10414F007E110E017FF02C00FEF6B
:1085B0001FEFB801CE010B960E949E9663E078E013
:1085C000CE0141960E945399BE01655F7F4FCE0157
:1085D00041960E940198BC01CE0101960E944A99E1
:1085E000CE0101960E94DF5CCE0101960E94E798C1
:1085F000CE0141960E94E798CE010B960E94E79823
:10860000BE016D5D7F4FCE0189960E94979861E013
:1086100078E0CE0101960E945399BE016F5F7F4FB3
:10862000CE0189960E94A4977C01CE0101960E94FA
:10863000E7986EED7BE0CE0183960E9467966EED23
:108640007BE0CE014D960E9467961E141F040CF02D
:1086500010C1A7014F5F5F4F8DA59EA54817590711
:1086600090F4BE01675D7F4FCE0101960E94275AAC
:10867000BE016F5F7F4FCE0183960E94AE98CE0100
:1086800001960E94E798970150E040E0BE01675DC7
:108690007F4FCE0101960E946499BE016F5F7F4FAC
:1086A000CE014D960E94AE98CE0101960E94E798A9
:1086B000A8014F5F5F4F8AE0849F9001859F300D36
:1086C0001124A90141545E4E5A01FE0131963F0129
:1086D000F12CE12C809F9001819F300D1124A90184
:1086E00043535E4E2A012AE2322E89A19AA1892B98
:1086F00009F4E8C0CE014D96E114F10409F0CEC0B2
:10870000D7FCCCC00E94EF96A114B10439F044E02C
:1087100050E0B501CE014D960E94B28EB501CE015A
:1087200041960E94539968E078E0CE0147960E94F6
:108730005399BE016F5E7F4FCE0147960E9401980C
:10874000BC01CE010B960E944A99CE010B960E9465
:10875000DF5CCE010B960E94E798CE0147960E94FF
:10876000E798CE0141960E94E79889A19AA10297C5
:1087700008F48DC061E070E0CE014D960E94BF9775
:10878000082E000C990B803391050CF44C96E32DC8
:10879000E81B8E2FF2018083FFEFEF1AFF0ABE0164
:1087A0006D5D7F4FCE0189960E94979861E078E0D9
:1087B000CE010B960E945399BE01655F7F4FCE019B
:1087C00089960E94A4974C01CE010B960E94E798CF
:1087D0006EED7BE0CE0183960E9467966EED7BE0A6
:1087E000CE014D960E946796181419040CF05CC0D7
:1087F000A4014F5F5F4F8DA59EA54817590790F4C0
:10880000BE01675D7F4FCE010B960E94275ABE01C5
:10881000655F7F4FCE0183960E94AE98CE010B9686
:108820000E94E798940150E040E0BE01675D7F4FF1
:10883000CE010B960E946499BE01655F7F4FCE0109
:108840004D960E94AE98CE010B960E94E79852E09A
:10885000650E711C4ACF6EED7BE0CE0183960E94BF
:108860006796BE01675D7F4FCE014D960E94979837
:1088700088CE6EED7BE0CE0183960E946796BE01A6
:10888000675D7F4FCE014D960E94979811CFCE0124
:108890004D960E94E496F20160837ECF0E94E4969A
:1088A000F3017183608378CF6EED7BE0CE01839618
:1088B0000E946796BE01675D7F4FCE014D960E9474
:1088C0009798C5CFD7FE8BC061E078E0CE010B96BC
:1088D0000E945399BE01655F7F4FCE0183960E942F
:1088E000A4978C01CE010B960E94E79817FF66C0F3
:1088F00009811A810931110514F008E110E0101600
:10890000110614F001E010E00093C111B801CE018E
:1089100041960E949E9666E178E0CE0147960E94BD
:108920005399BE016F5E7F4FCE0147960E9401981A
:10893000BC01CE010B960E944A99CE010B960E9473
:10894000DF5CCE010B960E94E798CE0147960E940D
:10895000E798CE0141960E94E798E114F10451F1A5
:108960008B819C8197FF02C090E080E09093C311BF
:108970008093C21121E0E216F104E1F08D819E8125
:10898000081719070CF4C8011816190614F081E02D
:1089900090E081508093C61132E0E316F10451F06B
:1089A0008F8198851816190614F081E090E08150A7
:1089B0008093C7118CE291E00E945E8ECE014D96AD
:1089C0000E94E798CE0183960E94E798CE0189968F
:1089D0000E94E798CE018F960E94E7987FCB809106
:1089E000C011082E000C990B081719070CF083C052
:1089F000B701CE0141960E949E9660E278E0CE01DA
:108A000047960E945399BE016F5E7F4FCE014796F5
:108A10000E940198BC01CE010B960E944A99CE019A
:108A20000B960E94DF5CCE010B960E94E798CE0168
:108A300047960E94E798CE0141960E94E7988AE007
:108A4000809FF001819FF00D1124E154FE4E81E0E2
:108A5000878783E090E0918B808B938B828BE114EE
:108A6000F10409F4ABCF8B819C818038910514F01F
:108A70008FE790E080384FEF940714F480E89FEF81
:108A8000878751E0E516F10409F498CF8AE0809FCA
:108A9000F001819FF00D1124E154FE4E8D819E81E5
:108AA00097FF02C090E080E0918B808B82E0E81617
:108AB000F10409F483CF8AE0809FF001819FF00DDB
:108AC0001124E154FE4E8F81988597FF02C090E0FB
:108AD00080E0938B828B8091C111082E000C990B42
:108AE000081719071CF00F5F0093C1118CE291E089
:108AF0000E94D58E63CFBE016D5D7F4FCE0147963C
:108B00000E944A996091C011062E000C770BCE018D
:108B10000B960E949E9668E278E0CE0141960E94F4
:108B20005399BE01695E7F4FCE0141960E94019824
:108B300069E378E00E94EB97BE01655F7F4F0E947A
:108B40000198BC01CE0147960E949798CE014196AC
:108B50000E94E798CE010B960E94E798BE01695EDD
:108B60007F4FCE010B960E944A99CE010B960E9430
:108B7000E158CE010B960E94E798CE0147960E94DD
:108B8000E7981CCF6DE378E0CE0101960E945399DF
:108B9000BE016F5F7F4F8DED92E10E94D097182F3D
:108BA000CE0101960E94E7981123C9F16CE679E0A5
:108BB000CE0101960E945399BE016F5F7F4F83EEF5
:108BC00092E10E949A97AC014F5F5F4F63EE72E1B2
:108BD000CE010B960E94275ABE01655F7F4F8FEB37
:108BE00092E10E94AE98CE010B960E94E798CE01CA
:108BF00001960E94E7988FEB92E10E94E49661153E
:108C0000710531F481E0809389040E94E41564CAFF
:108C10006130710509F060CA10928904F6CF62E4F0
:108C200078E0CE0101960E945399BE016F5F7F4F9D
:108C30008DED92E10E94D097182FCE0101960E94EF
:108C4000E798112309F43AC143E050E063EE72E182
:108C5000CE0101960E94275ABE016F5F7F4F8FEBB6
:108C600092E10E94AE98CE0101960E94E7986FEBC8
:108C700072E1CE0101960E944A99CE0101960E94AE
:108C8000DF5CCE0101960E94E7986FEB72E1CE01A6
:108C900001960E944A99CE0101960E945298BC0109
:108CA0008AEB93E10E949798CE0101960E94E79883
:108CB0006FEB72E1CE0101960E944A99CE010196B6
:108CC0000E945298BC0184EB93E10E949798CE01D8
:108CD00001960E94E7984091BE135091BF13411531
:108CE000510549F084E491E1009729F0BC018AEB39
:108CF00093E10E94B28E4091B8135091B91341157F
:108D0000510549F082EA91E1009729F0BC0184EB1A
:108D100093E10E94B28E90E080E00E94888E68EA23
:108D200077E0CE0101960E9453996FEB72E1CE017C
:108D300001960E940198BC01CE0141960E944A9979
:108D4000CE0101960E94E79880919E1190919F110B
:108D5000892B39F4BE016F5E7F4F86ED9DE00E9446
:108D60009E9B68EB7BE080E090E00E943AA18091BE
:108D70009E1190919F11029709F087C06FEB72E1ED
:108D8000CE0147960E944A9966E478E0CE010196AA
:108D90000E945399CE0101960E943FABCE010196ED
:108DA0000E94E79864EF71E080E090E00E943AA1B1
:108DB00069E478E0CE0101960E945399CE010196B4
:108DC0000E943FABCE0101960E94E7986CED75E0E2
:108DD00080E090E00E943AA162E578E0CE01019641
:108DE0000E945399CE0101960E943FABCE0101969D
:108DF0000E94E79864EF71E080E090E00E943AA161
:108E000060E678E0CE0101960E945399CE0101966A
:108E10000E943FABCE0101960E94E79864EF71E09B
:108E200080E090E00E943AA168EA77E0CE010196E6
:108E30000E945399BE01695E7F4FCE0101960E9448
:108E40000198BC01CE010B960E944A99CE01019671
:108E50000E94E798CE010B960E94EF96BE01655FD7
:108E60007F4FCE0101960E944A99CE0101960E9441
:108E70003FABCE0101960E94E798CE010B960E946F
:108E8000E798CE0147960E94E79868EB7BE080E088
:108E900090E00E943AA164E471E1CE0101960E9443
:108EA0005399CE0101960E94DF5CCE0101960E948B
:108EB000E7981092EE04CE0141968ECD6EE678E0F2
:108EC000CE0101960E945399BE016F5F7F4F8DEDD9
:108ED00092E10E94D097182FCE0101960E94E79848
:108EE000112309F487C044E050E063EE72E1CE0143
:108EF00001960E94275ABE016F5F7F4F8FEB92E170
:108F00000E94AE98CE0101960E94E79860EB77E050
:108F1000CE0101960E9453996FEB72E1CE0101964A
:108F20000E940198BC01CE010B960E944A99CE0185
:108F300001960E94E79880919E1190919F11892B34
:108F400069F4BE01655F7F4F86ED9DE00E949E9BA8
:108F500068E873E180E090E00E943AA180919E1160
:108F600090919F11029759F563E778E0CE01019641
:108F70000E9453998091C3129091C412892B21F5BC
:108F80006CE778E0CE0101960E946796BE01655FAE
:108F90007F4FCE0141960E944A99CE0141960E9490
:108FA0003FABCE0141960E94E79860ED77E080E00C
:108FB00090E00E943AA1CE0101960E94E79810929B
:108FC000EE04CE010B9608CDBE016F5F7F4FCE0140
:108FD00041960E944A99CE0141960E943FABCE0134
:108FE00041960E94E79860ED77E080E090E00E9473
:108FF0003AA1CCCF65E878E0CE0101960E94539962
:10900000BE016F5F7F4F8DED92E10E94D097182FC8
:10901000CE0101960E94E798112309F462C063EE25
:1090200072E18FEB92E10E94979881E08093EE04C9
:1090300063EE72E1CE0101960E944A99CE0101963B
:109040000E94DF5CCE0101960E94E79880919E11FC
:1090500090919F11029709F16FEB72E186ED9DE00F
:109060000E949E9B68EB7BE080E090E00E943AA12A
:10907000CE0101960E943B6FBE016F5F7F4F83EE72
:1090800092E10E94AE98CE0101960E94E79860EDB1
:1090900077E080E090E00E943AA180919E1190914B
:1090A0009F11029771F46FEB72E1CE0101960E945D
:1090B0004A99CE0101960E943FABCE0101960E94D3
:1090C000E7988091E7129091E812892B09F404C87F
:1090D00066ED75E0CE0101960E94539963EE72E150
:1090E000A4C869E878E0CE0101960E945399BE01B8
:1090F0006F5F7F4F8DED92E10E94D097182FCE01C8
:1091000001960E94E798112309F462C080919E1194
:1091100090919F11019711F00C946C40CE01019633
:109120000E9414328D819E81009709F44BC0E98121
:10913000FA812081222309F445C0079708F442C030
:1091400064E179E0CE010B960E94419948EC50E031
:109150006FEF7FEFCE010B960E94335ACE010B9634
:109160000E94E798BE016F5F7F4FCE010B960E9471
:109170004A9940ED57E06FEF7FEFCE010B960E94CA
:109180005759CE010B960E94E7986FE878E0CE0120
:109190000B960E94539963EE72E1CE010B960E94EA
:1091A0000198BC01CE0141960E944A99CE01419698
:1091B0000E94E158CE0141960E94E798CE010B969D
:1091C0000E94E798CE0101960E94E7980C946C40AB
:1091D0006DE978E0CE0101960E945399BE016F5F60
:1091E0007F4F8DED92E10E94D097182FCE0101960E
:1091F0000E94E798112361F125E030E044E050E05F
:1092000063EE72E1CE0101960E946499BE016F5F28
:109210007F4F8FEB92E10E94AE98CE0101960E94A3
:10922000E79863EE72E1CE0101960E944A99CE0161
:1092300001960E94DF5CCE0101960E94E7988FEBB9
:1092400092E10E94E496CB010E94AC270C946C4002
:1092500062EA78E0CE0101960E945399BE016F5FE9
:109260007F4F8DED92E10E94D097182FCE0101968D
:109270000E94E798112361F127E030E046E050E0DA
:1092800063EE72E1CE0101960E946499BE016F5FA8
:109290007F4F8FEB92E10E94AE98CE0101960E9423
:1092A000E7988FEB92E10E94E496672B69F41092A5
:1092B0000E0D63EE72E1CE0101960E944A99CE0135
:1092C00001960E94DF5C7ECF81E080930E0DF1CF8E
:1092D00069EA78E0CE0101960E945399BE016F5F62
:1092E0007F4F8DED92E10E94D097182FCE0101960D
:1092F0000E94E798112309F4F7C18091430C9091E3
:10930000440C1816190614F00C946E4080918704D2
:1093100090918804909386048093850488E592E078
:1093200090938804809387048DEA9FE00E940A8AC4
:10933000198A1A8A1B8A1C8A66246394712C2E014E
:1093400091E1490E511CFE017596FEABEDAB80918B
:10935000430C9091440C861597050CF4BBC1009109
:10936000870410918804093DFFE01F070CF0B2C18B
:1093700072016801C418D508C6018E0D9F1D0E9498
:1093800045B7F70181937F012DA93EA9E217F307A5
:1093900099F789889A88AB88BC88A5019401C50192
:1093A000B4010E940BBB81119DC0C801049690932B
:1093B0008804809387048FE1E82E8CE0F82E0B510F
:1093C0001C40C8018E0D9F1D0E9445B7F701819377
:1093D0007F0123E43CE02E173F0799F723E0B50116
:1093E000A401CE0101960E94EF98BE016F5F7F4FEE
:1093F000CE010B960E944A9966E979E0CE010B9660
:109400000E94EB97BC0185EC92E10E949798CE01F7
:109410000B960E94E798CE0101960E94E7986FE1B3
:109420007CE0CE0101960E945399BE016F5F7F4F91
:109430008FEB92E10E94AE98CE0101960E94E798D0
:109440006DEA78E0CE0101960E945399BE016F5FEC
:109450007F4F8FEB92E10E94D097182FCE0101969B
:109460000E94E798112309F49EC06DEA78E0CE01CE
:1094700001960E945399A090C312B090C412A114F7
:10948000B10409F48CC08D809E808114910409F48C
:1094900086C0E090B411F090B511E818F908009179
:1094A000BF121091C01229803A80E114F104E1F555
:1094B00069817A81C8010E940FBE8C01009709F46E
:1094C0006EC06091B0117091B1114091B411509182
:1094D000B5110E94C7BD8091B4119091B511080FCC
:1094E000191FE6CF8091850490918604909388049B
:1094F00080938704812FE6960FB6F894DEBF0FBEE7
:10950000CDBFDF91CF911F910F91FF90EF90DF9032
:10951000CF90BF90AF909F908F907F906F905F9013
:109520004F903F902F9008956501C801F7FE62C0EB
:10953000680169817A81C8010E940FBE4C010097C1
:1095400051F15C01A01AB10AA501B801C6010E943F
:10955000C7BDCA0CDB1C6091B0117091B111409174
:10956000B4115091B511C6010E94C7BD8091B411CC
:109570009091B511C80ED91E0D811E81080D191DBF
:109580008091C3129091C4128E0D9F1D9093C412AE
:109590008093C312CECFB801C6010E94EBBDCE01AD
:1095A00001960E94E7986FEB72E185EC92E10E94D0
:1095B0006B9865EC72E1CE0101960E944A99CE014A
:1095C00001960E94E158CE0101960E94E798809191
:1095D00087049091880484969093880480938704EC
:1095E00064E170E080E090E00E943AA1FFEF6F1A22
:1095F0007F0AADCEB1010E940FBE009729F0880D01
:10960000991DCE0CDF1CF6CFAC14BD0441F2809145
:10961000C1129091C2128C159D0588F4B6016F5F3E
:109620007F4FC8010E94C0BC009709F4B8CF909347
:10963000C0128093BF12D092C212C092C112409148
:10964000C3125091C4124150510957FDA8CFBE0119
:109650006F5F7F4F8FEB92E10E944C978C0197FDDB
:109660009ECF2D813E81280F391F8091BF1290918E
:10967000C012820F931F4091C3125091C412421B1B
:10968000530BBC018E0D9F1D0E94D0BD8091C31253
:109690009091C4128E0D9F1D9093C4128093C3129B
:1096A0002091BF123091C012820F931FFC011082D3
:1096B0008091BF129091C0126091B0117091B11160
:1096C0004091B4115091B511800F911F0E94C7BDF8
:1096D000A801B9CF80918504909186049093880465
:1096E000809387040C946E4061EB78E0CE01019684
:1096F0000E945399BE016F5F7F4F8DED92E10E94F2
:10970000D097182FCE0101960E94E7981123D9F126
:1097100026E030E045E050E063EE72E1CE010196D4
:109720000E946499BE016F5F7F4F8FEB92E10E94B0
:10973000AE98CE0101960E94E7988FEB92E10E94CD
:10974000E496672B29F410921E0C88E592E0C6CFB0
:1097500081E080931E0C1092440C1092430C1092E6
:109760001A0C10921B0C10921C0C10921D0C0E94D3
:10977000D6A76093160C7093170C8093180C9093D7
:10978000190C0C946E4067EB78E0CE0101960E94B4
:109790005399BE016F5F7F4F8DED92E10E94D0978C
:1097A000182FCE0101960E94E798112309F478C082
:1097B0008091E7129091E812079710F40C946E4094
:1097C00046E050E063EE72E1CE0101960E94275A16
:1097D000BE016F5F7F4F8FEB92E10E94AE98CE018A
:1097E00001960E94E7988FEB92E10E94D9966093D0
:1097F000EA047093EB048093EC049093ED0464E02E
:1098000079E085EC92E10E9472984091EA045091CF
:10981000EB046091EC047091ED0421E0CE0101961F
:109820000E94EF98BE016F5F7F4FCE010B960E94A2
:109830004A9964ED76E0CE010B960E94EB97BC014D
:1098400085EC92E10E946B98CE010B960E94E798FE
:10985000CE0101960E94E79865EC72E1CE01019677
:109860000E944A99CE0101960E94E158CE010196CC
:109870000E94E7980E94D6A728EE33E040E050E02F
:109880000E948DB7CA01B9010E9423B66093090DE9
:1098900070930A0D80930B0D90930C0D0C946E40F9
:1098A0006EEB78E0CE0101960E945399BE016F5F86
:1098B0007F4F8DED92E10E94D097182FCE01019637
:1098C0000E94E798112309F456C08091E712909105
:1098D000E812079710F40C946E4046E050E063EEF7
:1098E00072E1CE0101960E94275ABE016F5F7F4F41
:1098F0008FEB92E10E94AE98CE0101960E94E7980C
:109900008FEB92E10E94D996609381047093820458
:10991000809383049093840464EF78E085EC92E173
:109920000E94729840918104509182046091830456
:109930007091840421E0CE0101960E94EF98BE014F
:109940006F5F7F4FCE010B960E944A9964ED76E0DF
:10995000CE010B960E94EB97BC0185EC92E10E9430
:109960006B98CE010B960E94E798CE0101960E945B
:10997000E7980C94D3410E94FB1D182F81110C9481
:109980006E40B8CD11E0B6CDAF92BF92CF92DF92CC
:10999000EF92FF920F931F93CF93DF93CDB7DEB774
:1099A000A4970FB6F894DEBF0FBECDBF8091F60B23
:1099B000882399F01092F60BA4960FB6F894DEBFA8
:1099C0000FBECDBFDF91CF911F910F91FF90EF9010
:1099D000DF90CF90BF90AF9008958091E712909163
:1099E000E812049708F040C06DE878E0CE010196D7
:1099F0000E945399BE016F5F7F4F8DED92E10E94EF
:109A0000D097182FCE0101960E94E798112361F19B
:109A100061E070E083EE92E10E94BF9780330CF426
:109A2000845E6AE270E0681B710987FD7395CE0160
:109A300001960E949E96BE016F5F7F4F83EE92E17A
:109A40000E94AE98CE0101960E94E79863EE72E103
:109A500081ED92E10E94979883EE92E10E94E49654
:109A6000CB010E949975A8CF6EEE77E0CE010196EA
:109A70000E945399BE016F5F7F4F8DED92E10E946E
:109A8000D097182FCE0101960E94E798112309F470
:109A9000AFC365EC78E0CE0101960E945399CE01E8
:109AA00001960E94E158CE0101960E94E79861ED6F
:109AB00078E0CE0107960E94539964EB73E1CE01E2
:109AC00007960E940198BC01CE0101960E944A9916
:109AD000CE0101960E94E158CE0101960E94E798BE
:109AE000CE0107960E94E7986091C9047091CA045C
:109AF0008091CB049091CC040E9425B620E030E008
:109B000048EC52E40E949DB8AB01BC0122E0CE01BA
:109B100007960E94EF9867EE78E0CE010D960E94BE
:109B20005399BE01695F7F4FCE010D960E94019847
:109B300069E076E00E94EB97BC01CE0101960E949D
:109B40004A99CE0101960E94E158CE0101960E94E9
:109B5000E798CE010D960E94E798CE0107960E94E5
:109B6000E7984091C5045091C6046091C704709174
:109B7000C80424E0CE0107960E94EF986CEF78E0CD
:109B8000CE010D960E945399BE01695F7F4FCE01B1
:109B90000D960E940198BC01CE0101960E944A993F
:109BA000CE0101960E94E158CE0101960E94E798ED
:109BB000CE010D960E94E798CE0107960E94E79885
:109BC0004091B9045091BA046091BB047091BC04F7
:109BD00022E0CE0107960E94EF984091B104509187
:109BE000B2046091B3047091B40423E0CE010D96E9
:109BF0000E94EF984091BD045091BE046091BF0453
:109C00007091C00422E0CE0143960E94EF984091EB
:109C1000B5045091B6046091B7047091B80423E084
:109C2000CE0149960E94EF9869E179E0CE014F9606
:109C30000E945399BE01675E7F4FCE014F960E94EE
:109C400001986EE279E00E94EB97BE016D5E7F4F56
:109C50000E94019861E379E00E94EB97BE01635F87
:109C60007F4F0E9401986EE279E00E94EB97BE015F
:109C7000695F7F4F0E94019867E379E00E94EB974C
:109C8000BC01CE0101960E944A99CE0101960E9424
:109C9000E158CE0101960E94E798CE014F960E94AE
:109CA000E798CE0149960E94E798CE0143960E941C
:109CB000E798CE010D960E94E798CE0107960E9484
:109CC000E7986AE477E0CE0149960E944199F090C6
:109CD00057110F2D0F2C000C110B0115110509F058
:109CE0007EC1209158113091591140915A115091D3
:109CF0005B1160E070E080EA90E40E949DB8AB01E7
:109D0000BC0122E0CE0101960E94EF986EE276E05F
:109D1000CE0107960E945399BE016F5F7F4FCE011F
:109D200007960E94019862E07BE00E94EB97BC01DD
:109D3000CE0149960E946B98CE0107960E94E79843
:109D4000CE0101960E94E798C8010297029738F564
:109D50008F2D9AE08902B0011124CE0101960E9454
:109D60009E966CE379E0CE0107960E945399BE015E
:109D70006F5F7F4FCE0107960E9401986BEF7AE0EC
:109D80000E94EB97BC01CE0149960E946B98CE01D0
:109D900007960E94E798CE0101960E94E7986AE232
:109DA00077E00430110519F034F062E277E0CE017B
:109DB00049960E941498BE01675E7F4FCE010196BE
:109DC0000E944A99CE0101960E94E158CE01019667
:109DD0000E94E79868E479E0CE0149960E94679670
:109DE00080915411609155117091561183300CF08F
:109DF0008DC3CE0101960E949E9663E479E0CE0168
:109E000007960E945399BE016F5F7F4FCE01079660
:109E10000E9401986CE37AE00E94EB97BC01CE01AE
:109E200049960E946B98CE0107960E94E798CE0152
:109E300001960E94E798BE01675E7F4FCE010196B2
:109E40000E944A99CE0101960E94E158CE010196E6
:109E50000E94E79840915C1150915D1160915E11F4
:109E600070915F1122E0CE0107960E94EF9868E59D
:109E700079E0CE010D960E945399BE01695F7F4F34
:109E8000CE010D960E9401986EE679E00E94EB9754
:109E9000BC01CE0101960E944A99CE0101960E9412
:109EA000E158CE0101960E94E798CE010D960E94DE
:109EB000E798CE0107960E94E79840917211509161
:109EC0007311609174117091751122E0CE010796A3
:109ED0000E94EF9865E779E0CE010D960E945399B4
:109EE000BE01695F7F4FCE010D960E9401986BE124
:109EF00076E00E94EB97BC01CE0101960E944A9940
:109F0000CE0101960E94E158CE0101960E94E79889
:109F1000CE010D960E94E798CE0107960E94E79821
:109F200087E9E82E84E0F82E01E010E099E1C92EDF
:109F3000E2E0EE0EF11C8091970490919804801756
:109F400091070CF457C0F701A080B180B501CE0194
:109F500007960E949E96B801CE010D960E949E968D
:109F600068E879E0CE0143960E945399BE01635F91
:109F70007F4FCE0143960E94019860E979E00E94EC
:109F8000EB97BE01695F7F4F0E94019863E979E01A
:109F90000E94EB97CA9CB001CB9C700D1124685FA6
:109FA0007D4F0E94EB97BC01CE0101960E944A9919
:109FB000CE0101960E94E158CE0101960E94E798D9
:109FC000CE0143960E94E798CE010D960E94E79835
:109FD000CE0107960E94E7980F5F1F4FA9CF01306F
:109FE000110509F0B1CE6CE377E0CE0149960E94ED
:109FF0001498AACE80919E1190919F11892B71F493
:10A0000069E979E0CE0101960E945399CE0101964B
:10A010000E94E158CE0101960E94E79880919E111E
:10A0200090919F11019771F468EA79E0CE01019651
:10A030000E945399CE0101960E94E158CE010196EB
:10A040000E94E79880919E1190919F11029771F460
:10A0500062EB79E0CE0101960E945399CE01019600
:10A060000E94E158CE0101960E94E7986091D604C3
:10A070007091D704CE0107960E949E9664EC79E019
:10A08000CE010D960E945399BE01695F7F4FCE01AC
:10A090000D960E940198BC01CE0101960E944A993A
:10A0A000CE0101960E94E158CE0101960E94E798E8
:10A0B000CE010D960E94E798CE0107960E94E79880
:10A0C0004091EA045091EB046091EC047091ED042E
:10A0D00022E0CE0107960E94EF9861EE79E0CE0172
:10A0E0000D960E945399BE01695F7F4FCE010D9678
:10A0F0000E94019864ED76E00E94EB97BC01CE01CE
:10A1000001960E944A99CE0101960E94E158CE0123
:10A1100001960E94E798CE010D960E94E798CE0125
:10A1200007960E94E79840918104509182046091C3
:10A1300083047091840422E0CE0107960E94EF9878
:10A1400061EF79E0CE010D960E945399BE01695FDF
:10A150007F4FCE010D960E94019864ED76E00E943B
:10A16000EB97BC01CE0101960E944A99CE0101965F
:10A170000E94E158CE0101960E94E798CE010D960B
:10A180000E94E798CE0107960E94E7986EE177E07B
:10A19000CE0101960E944199CE0101960E94FE587F
:10A1A000CE0101960E94E7986091100C7091110CFD
:10A1B000CE0101960E949E96CE0101960E94FE5805
:10A1C000CE0101960E94E7986FEF76E0CE010196EE
:10A1D0000E944199CE0101960E94E158CE0101965C
:10A1E0000E94E7981092EE04CE0149960E94E798EB
:10A1F0008091E7129091E8128330910508F083C1B5
:10A200008130910509F061C070E060E083EE92E179
:10A210000E94BF97D82E8D2DDD0C990B0E94A1BDF9
:10A22000892BB1F00E94D4150E94155962E67AE09C
:10A23000CE0101960E9453994AE050E070E060E040
:10A24000CE0101960E94335ACE0101960E94E798F2
:10A2500063EE72E1CE0107960E944A9970E060E0D9
:10A26000CE0107960E94BF97823409F405C10CF015
:10A2700097C0803309F429C10CF081C0833209F4FE
:10A2800012C18A3209F418C1BE01695F7F4F81EDA6
:10A2900092E10E94979870E060E081ED92E10E9467
:10A2A000BF97082E000C990BC0970A9738F481EDE0
:10A2B00092E10E94E496CB010E94997564E670E0F9
:10A2C00080E090E00E943AA1B1C0029709F0A3CFCC
:10A2D0006DE878E0CE0101960E945399BE016F5F50
:10A2E0007F4F8DED92E10E94D097182FCE010196FD
:10A2F0000E94E798112309F48ECF61E070E083EEAD
:10A3000092E10E94BF97682FCE0101960E941F998B
:10A31000BE016F5F7F4F81ED92E10E94AE98CE014A
:10A3200001960E94E79870E060E083EE92E10E945F
:10A33000BF97D82E80910E0D882309F46CCF61E071
:10A340007AE0CE0101960E94539963EE72E1CE014C
:10A3500001960E94019862E67AE00E94EB97BC01A8
:10A360008DEA9FE00E949E9BCE0101960E94E79895
:10A3700061ED72E18DEA9FE00E94AC9B4CCF81338E
:10A3800009F4B2C0813409F07FCF6EE07AE083EE49
:10A3900092E10E94679680910C0C90910D0C44C044
:10A3A000813699F30CF061C0833409F470C08434B1
:10A3B00009F06ACF8091D5129091D612892BB1F114
:10A3C00061E070E0CE0107960E94BF97182F809140
:10A3D0000E0D882361F067E07AE08DEA9FE00E942D
:10A3E0009C9B61ED72E18DEA9FE00E94AC9B103373
:10A3F0000CF4145E6AE270E0611B710917FD73953D
:10A40000CE0101960E949E96BE016F5F7F4F81ED47
:10A4100092E10E94AE98CE0101960E94E79881EDEC
:10A4200092E10E94E496CB010E949975CE010796B5
:10A430000E94E7980E94D6A76093050D7093060DC1
:10A440008093070D9093080D0E94D6A76093050D89
:10A450007093060D8093070D9093080D6EED7BE0D1
:10A4600083EE92E10E946796A7CA833681F024F0BA
:10A47000843609F49FCF08CF61E17AE083EE92E160
:10A480000E94679610920D0D8CEF9FEFCDCF64E187
:10A490007AE083EE92E10E94679681E080930D0D51
:10A4A0008DEF9FEFC1CF67E17AE083EE92E10E94EA
:10A4B00067968EEF9FEFB8CF6AE17AE083EE92E184
:10A4C0000E9467968FEF9FEFAFCF68E177E081ED55
:10A4D00092E10E94679668E177E083EE92E10E9444
:10A4E000679690E080E0A0CF6BE17AE081ED92E1A9
:10A4F0000E9467966BE17AE083EE92E10E94679694
:10A5000081E090E091CF0E94BE3F9ECFCE010196A8
:10A510000E949E966DE17AE0CE0107960E945399C3
:10A52000BE016F5F7F4FCE0107960E94019876CCE7
:10A53000CF92DF92EF92FF920F931F93CF93DF930F
:10A54000CDB7DEB7E0970FB6F894DEBF0FBECDBF34
:10A550008E01015E1F4F8130910509F0B7C066E2A0
:10A560007AE0CE0101960E94539969E27AE0CE0129
:10A5700007960E9453996CE27AE0CE010D960E94F4
:10A58000539961EF76E0C8010E94419944E650E09A
:10A590006FEF7FEFC8010E94DD5AC8010E94E79863
:10A5A00066EE76E083EE92E10E9472986091D604A6
:10A5B0007091D704CE0185960E949E9663EE72E15B
:10A5C000C8010E944A99BE016B5D7F4FC8010E947D
:10A5D0000198BC01CE018B960E944A9940ED57E04C
:10A5E0006FEF7FEFCE018B960E945759CE018B966D
:10A5F0000E94E798C8010E94E798CE0185960E94C4
:10A60000E79867ED76E0C8010E94419944E650E082
:10A610006FEF7FEFC8010E94DD5AC8010E94E798E2
:10A620006DED79E0C8010E94539923E030E0A80164
:10A63000BE016F5F7F4FCE0185960E94DAA5BE01F5
:10A640006B5D7F4F83EE92E10E94AE98CE018596BE
:10A650000E94E798C8010E94E7988091E7129091C4
:10A66000E812892B09F4E3C270E060E083EE92E126
:10A670000E94BF97082E000C990BC0970A9708F00C
:10A68000D6C283EE92E10E94E4966B016FE27AE01B
:10A69000C8010E94539986E08C9DB0018D9D700D7C
:10A6A000112481E090E08C0F9D1F680F791FC80175
:10A6B0000E940198BC0183EE92E10E949798C80124
:10A6C0000E94E7980E94BE3F182FE2C08A3F2FEFFA
:10A6D000920709F023C164E37AE0CE0101960E945B
:10A6E00053996EE37AE0CE0107960E94539966E48F
:10A6F0007AE0CE010D960E9453996EE47AE0CE0185
:10A7000043960E94539968EC76E0C8010E944199F3
:10A7100044E650E06FEF7FEFC8010E94DD5AC801A8
:10A720000E94E79862EC76E083EE92E10E947298D4
:10A7300080915411EE24E394F12CEC0EFD1E96E072
:10A740008902E00CF11C112463EE72E1C8010E9441
:10A750004A99B701C8010E940198BC01CE018596B3
:10A760000E944A9940ED57E06FEF7FEFCE0185964A
:10A770000E945759CE0185960E94E798C8010E9411
:10A78000E79862EB76E0C8010E94419944E650E008
:10A790006FEF7FEFC8010E94DD5AC8010E94E79861
:10A7A00064E57AE0C8010E94539924E030E0A801F2
:10A7B000BE016F5F7F4FCE0185960E94DAA5BE0174
:10A7C0006B5D7F4F83EE92E10E94AE98CE0185963D
:10A7D0000E94E798C8010E94E7988091E712909143
:10A7E000E812892B09F498C070E060E083EE92E1F2
:10A7F0000E94BF97082E000C990BC0970A9708F08B
:10A800008BC083EE92E10E94E4966230710581056F
:10A8100091050CF46EC066EA76E0C8010E94419989
:10A8200044E650E06FEF7FEFC8010E945759C8011E
:10A830000E94E79844EF51E063E070E0CE01859616
:10A840000E9407A56AE57AE0C8010E94539963EE69
:10A8500072E1C8010E94019861E67AE00E94EB97DC
:10A86000BE016B5D7F4F0E940198BC0183EE92E1B7
:10A870000E949798C8010E94E798CE0185960E9491
:10A88000E7980E94BE3F182FCE0143960E94E7989A
:10A89000CE010D960E94E798CE0107960E94E79898
:10A8A000CE0101960E94E79860E276E0111102C0A5
:10A8B00061E176E0CE0101960E94419948EC50E0BA
:10A8C0006FEF7FEFCE0101960E945759CE0101969E
:10A8D0000E94E798E0960FB6F894DEBF0FBECDBF9A
:10A8E000DF91CF911F910F91FF90EF90DF90CF906C
:10A8F00008956AE57AE0C8010E94539963EE72E117
:10A90000C8010E940198BC0183EE92E10E949798D1
:10A91000C8010E94E798B5CF10E0B6CF0F9609F0B6
:10A92000ECC0CE0101967C016EED7BE0C7010E9478
:10A93000539996E0E90EF11C0E151F05A9F764E680
:10A940007AE0CE0101960E9467968091571181119D
:10A9500030C0209158113091591140915A115091A5
:10A960005B1160E070E080EA90E40E949DB8AB016A
:10A97000BC0122E0CE0185960E94EF986AE67AE05B
:10A98000C8010E945399BE016B5D7F4FC8010E94B0
:10A9900001986BEF7AE00E94EB97BC01CE01019623
:10A9A0000E946B98C8010E94E798CE0185960E948C
:10A9B000E7986BE976E0CE0107960E9472986FE8FF
:10A9C00076E0CE010D960E94729863E876E0CE01A3
:10A9D00043960E94729867E776E0CE0149960E94FE
:10A9E000729861E776E0C8010E94729862E676E0AC
:10A9F000C8010E94419944E650E06FEF7FEFC80123
:10AA00000E94DD5AC8010E94E7986EED7BE083EE5C
:10AA100092E10E9467968091571161E070E06C0F9F
:10AA20007D1F26E08202600D711D1124C8010E9465
:10AA30004A9940ED57E06FEF7FEFC8010E945759E8
:10AA4000C8010E94E79863E576E0C8010E94419939
:10AA500044E650E06FEF7FEFC8010E94DD5AC80165
:10AA60000E94E79863EE72E1C8010E944A9925E0CE
:10AA700030E0A801BE016F5F7F4FCE0185960E9436
:10AA8000DAA5BE016B5D7F4F83EE92E10E94AE9826
:10AA9000CE0185960E94E798C8010E94E7988091B0
:10AAA000E7129091E812892B31F170E060E083EEBB
:10AAB00092E10E94BF97082E000C990BC0970A974D
:10AAC000D0F467E276E0C8010E94539963EE72E128
:10AAD000C8010E940198BC0183EE92E10E94979800
:10AAE000C8010E94E7980E94BE3F182FCE014996E8
:10AAF0000E94E798C9CE10E0F9CF6DE67AE0CE016A
:10AB000001960E9453996DEA79E0CE0107960E9462
:10AB1000539960E77AE0CE010D960E94539963E461
:10AB200076E0C8010E94419944E650E06FEF7FEF64
:10AB3000C8010E94DD5AC8010E94E7986DE376E0E3
:10AB400083EE92E10E94729880919E1190919F11E4
:10AB500026E0289F7001299FF00C112481E090E0ED
:10AB60008C0F9D1FE80EF91E63EE72E1C8010E9472
:10AB70004A99B701C8010E940198BC01CE0185968F
:10AB80000E944A9940ED57E06FEF7FEFCE01859626
:10AB90000E945759CE0185960E94E798C8010E94ED
:10ABA000E7986DE276E0C8010E94419944E650E0E2
:10ABB0006FEF7FEFC8010E94DD5AC8010E94E7983D
:10ABC00063EE72E1C8010E944A9923E030E0A801D7
:10ABD000BE016F5F7F4FCE0185960E94DAA5BE0150
:10ABE0006B5D7F4F83EE92E10E94AE98CE01859619
:10ABF0000E94E798C8010E94E7988091E71290911F
:10AC0000E812892BA1F070E060E083EE92E10E94EF
:10AC1000BF97082E000C990BC0970A9740F483EE5B
:10AC200092E10E94E496CB010E94AC274DCD10E04A
:10AC30002FCECF92DF92EF92FF92CF93C091571118
:10AC4000C4304CF4C1300CF04BC0CC2359F160E05F
:10AC500070E0CB013FC0C430D1F70E94351720E02F
:10AC600030E040EA50E40E9484B620E030EC4FE748
:10AC700054E40E949DB820E030E040EA50E40E9495
:10AC80009DB820E030E040E851E40E9484B620E026
:10AC900030E040E850E40E94BFB720E030E04AE7EF
:10ACA00054E416C00E94351720E030E040EA50E43A
:10ACB0000E9484B620E030EC4FE754E40E949DB837
:10ACC000209158113091591140915A1150915B11B6
:10ACD0000E949DB8CF91FF90EF90DF90CF900895A4
:10ACE0000E9435172AE137E64CE950E40E9484B609
:10ACF000209158113091591140915A1150915B1186
:10AD00000E94BEB76B017C01EC2FEE0FFF0BE55AE2
:10AD1000FA4F60817181072E000C880B990B0E94FD
:10AD200025B69B01AC01C701B601D2CF8091890441
:10AD3000882349F08091E904882329F060E08CECB5
:10AD400093E10C949D1208958F929F92AF92BF92BF
:10AD5000CF92DF92EF92FF920F931F93CF93DF93E7
:10AD60008C01862F0B30110509F092C090912C13A5
:10AD7000992309F0F89462E10E949FA3EC0180916D
:10AD80002C13882309F07894209701F180E090EC4F
:10AD9000A9E7B4EC80931F1390932013A093211381
:10ADA000B09322138093231390932413A09325131D
:10ADB000B0932613CE3F8FEFD80709F49DC0CF3F45
:10ADC000DC0709F4EBC1CCEFDFEF24C1C0912713FE
:10ADD000E09028136E2D70E090E080E00E9425B690
:10ADE0002DEC3CEC4CEC5DE30E9484B64B015C0125
:10ADF0006C2F70E090E080E00E9425B69B01AC01D2
:10AE0000C501B4010E94BFB760931F137093201354
:10AE10008093211390932213D0912913F0902A1339
:10AE20006D2F6F7770E090E080E00E9425B64B01B7
:10AE30005C016F2D70E090E080E00E9425B62DEC63
:10AE40003CEC4CEC5DE30E9484B69B01AC01C50177
:10AE5000B4010E94BFB7D7FD19C06093231370934C
:10AE600024138093251390932613CE0DCD0FCF0D71
:10AE700081E090E020912B13C21302C090E080E0AB
:10AE8000892B09F487C0CFEFDFEF88C19058E5CF59
:10AE9000CFEFDFEF0631110509F0BCC090912C1304
:10AEA000992309F0F89461E00E949FA3EC0180913E
:10AEB0002C13882309F07894209709F180E090EC16
:10AEC000A9E7B4EC80931F1390932013A093211350
:10AED000B09322138093231390932413A0932513EC
:10AEE000B0932613CF3FDC0709F458C1209709F42B
:10AEF00051C0229609F067CFCEEFDFEF8BC0C09133
:10AF00002813D09127136091271370912813762767
:10AF10006727762790E080E00E9423B62DEC3CEC7A
:10AF20004CEC5DE30E9484B660931F137093201372
:10AF30008093211390932213E0902A13F090291309
:10AF40006F2D6F77762F6E2D90E080E00E9423B6F4
:10AF50002DEC3CEC4CEC5DE30E9484B6F7FC18C091
:10AF600060932313709324138093251390932613D7
:10AF70008C2F8D0F8E0D8F0DC1E0D0E090912B1393
:10AF8000891302C0D0E0C0E0D195C195D109AACF04
:10AF90009058E6CFC0901F13D0902013E09021135B
:10AFA000F090221320E030E048EC52E4C701B601F3
:10AFB0000E94A6B9D0E0C0E0181614F4CBEFDFEF82
:10AFC00020E030E0A901C701B6010E941EB687FF4C
:10AFD00002C0CAEFDFEFC0902313D0902413E0909B
:10AFE0002513F090261320E030E048EC52ECC70126
:10AFF000B6010E941EB687FF02C0C9EFDFEF20E056
:10B0000030E040EF52E4C701B6010E94A6B918161D
:10B010000CF4BFC00C30110509F0C0C08CE50E94D3
:10B02000168C90E080E00E94118C0E94FD9E65E0ED
:10B030008CE50E94159F1092340D8093330DC82F1C
:10B04000D0E0209709F4A8C0C530D1050CF4B6C0F3
:10B0500007EF1BE00E941D8FF80180870F5F1F4FD5
:10B06000C801875F9B408C179D07A4F3C091FF0B1D
:10B070000091000C602F70E090E080E00E9425B607
:10B080002DEC3CEC4CEC5DE30E9484B66B017C0142
:10B090006C2F70E090E080E00E9425B69B01AC012F
:10B0A000C701B6010E94BFB76B017C01C092F70BCC
:10B0B000D092F80BE092F90BF092FA0BD091010CC0
:10B0C0001091020C6D2F6F7770E090E080E00E948D
:10B0D00025B64B015C01612F70E090E080E00E949A
:10B0E00025B62DEC3CEC4CEC5DE30E9484B69B0154
:10B0F000AC01C501B4010E94BFB7D7FD5DC060932C
:10B10000FB0B7093FC0B8093FD0B9093FE0BC00F19
:10B11000CD0FC10F8091030CC813B5CE20E030E0F5
:10B1200048EC52E4C701B6010E94A6B9D0E0C0E0E5
:10B13000181614F4CBEFDFEF20E030E040EA50E4E3
:10B14000C701B6010E941EB687FF02C0CAEFDFEF3B
:10B15000C090FB0BD090FC0BE090FD0BF090FE0B31
:10B1600020E030E040EF51ECC701B6010E941EB66E
:10B1700087FF02C0C9EFDFEF20E030E040EF52E48C
:10B18000C701B6010E94A6B9181644F4C8EFDFEF54
:10B1900005C0C8EFDFEF3ECFCEEFDFEFCE01DF918E
:10B1A000CF911F910F91FF90EF90DF90CF90BF90C4
:10B1B000AF909F908F9008959058A1CFCDEFDFEF83
:10B1C000EDCFCF93DF93FC0124813581232B99F0C0
:10B1D000EC01BC0186ED9DE00E94AC9B6EE170E04D
:10B1E00080E090E00E943AA1BE018DEA9FE0DF91ED
:10B1F000CF910C94AC9BDF91CF910895CF93DF93C7
:10B20000FC0124813581232B69F0EC01BC018DEA1E
:10B210009FE00E949E9BBE0186ED9DE0DF91CF9155
:10B220000C949E9BDF91CF9108958091890488238F
:10B23000F9F08091E9048823D9F081E00E94208C04
:10B240008BE39FE10197F1F760E080E00E94318C91
:10B250006CE17DE08CEC93E10E94BE9B61E080E0BC
:10B260000E94318C6CE07DE08CEC93E10C94BE9BF1
:10B270000895CF93DF93209189042223A9F0209190
:10B28000E904222389F0EC016FED8CEC93E10E943C
:10B29000239A8C819D81892B39F0BE018CEC93E13E
:10B2A000DF91CF910C949E9BDF91CF910895EF9207
:10B2B000FF920F931F93CF93DF9320918904222352
:10B2C00009F461C02091E904222309F45CC08A01D9
:10B2D000EB017C01209719F1C095D09561E08C2F8E
:10B2E0000E94318CB7018CEC93E10E949E9B6BEF26
:10B2F0007CE08CEC93E10E94BE9BF701848161E0CD
:10B300008C0F0E94318CB801110F880B990BDF91C3
:10B31000CF911F910F91FF90EF900C943AA10E9452
:10B32000D6A7AB01BC018091C10C9091C20CA09139
:10B33000C30CB091C40C8C599F4FAF4FBF4F8417B3
:10B340009507A607B707F8F461E080E00E94318C0A
:10B35000B7018CEC93E10E949E9B6AEE7CE08CEC42
:10B3600093E10E94BE9B61E0F70184810E94318CD1
:10B370000E94D6A76093C10C7093C20C8093C30C3B
:10B380009093C40CC0CFDF91CF911F910F91FF908C
:10B39000EF900895FF920F931F93CF93DF93EC01EB
:10B3A000F62E08811981C8010E9445B7F81621F0D0
:10B3B0006F2DC8010E944DB7CE01DF91CF911F9133
:10B3C0000F91FF900895CF93DF93EC019A01AB01A9
:10B3D000E889F98982E08083211581EE38074105EB
:10B3E000510581F160E079E08DE390E00E948DB736
:10B3F00021503109410951095695479537952795AF
:10B40000EC85FD851082EE85FF852083188EEC8902
:10B41000FD8986E08083EA89FB8980818061808361
:10B42000EA89FB89808188608083EA89FB89808141
:10B4300080688083EA89FB8980818F7D8083DF91AA
:10B44000CF910895E889F989108220E1D9CFCF936F
:10B45000DF93EC01FB01248135810E946499CE01C8
:10B46000DF91CF910895CF92DF92EF92FF920F93E9
:10B470001F93CF93DF93CDB7DEB762970FB6F894E3
:10B48000DEBF0FBECDBF20918904222309F446C040
:10B490002091E904222309F441C08A016B017C0157
:10B4A0000E94D6A7AB01BC018091BD0C9091BE0C4F
:10B4B000A091BF0CB091C00C8C599F4FAF4FBF4FA4
:10B4C00084179507A607B70748F560E0CD20C0941C
:10B4D000A1F580E00E94318CD12CB7018CEC93E176
:10B4E0000E949E9B69ED7CE08CEC93E10E94BE9BE8
:10B4F000F701848160E08D0D0E94318C0E94D6A7F7
:10B500006093BD0C7093BE0C8093BF0C9093C00CE5
:10B51000B801110F880B990B0E943AA162960FB6E1
:10B52000F894DEBF0FBECDBFDF91CF911F910F9179
:10B53000FF90EF90DF90CF90089580E00E94318CD3
:10B540000E94D6A728EE33E040E050E00E945BB7AF
:10B55000CA01B90120E831E541E050E00E945BB743
:10B56000AB01BC01CE0101960E947196BE016F5FD6
:10B570007F4FCE0107960E944A9966E979E0CE0195
:10B5800007960E94EB97BC01CE010D960E944A9946
:10B59000CE0107960E94E798CE0101960E94E79897
:10B5A000BE01635F7F4F8CEC93E10E949E9BD98824
:10B5B000CE010D960E94E79890CFBF92CF92DF9276
:10B5C000EF92FF920F931F93CF93DF93CDB7DEB728
:10B5D00062970FB6F894DEBF0FBECDBF6C018B0132
:10B5E0007A0180918904882369F18091E904882394
:10B5F00049F177FF37C00095109560E0802F0E94D9
:10B60000318CB6018CEC93E10E949E9B68EC7CE04F
:10B610008CEC93E10E94BE9BF601848160E0800F78
:10B620000E94318C0E94D6A76093BD0C7093BE0C13
:10B630008093BF0C9093C00CB701FF0C880B990B43
:10B640000E943AA162960FB6F894DEBF0FBECDBF3E
:10B65000DF91CF911F910F91FF90EF90DF90CF90EE
:10B66000BF90089560E080E00E94318C0E94D6A7D0
:10B6700028EE33E040E050E00E945BB7CA01B90118
:10B6800020E831E541E050E00E945BB7AB01BC012E
:10B69000CE0101960E947196BE016F5F7F4FCE0171
:10B6A00007960E944A9966E979E0CE0107960E94C2
:10B6B000EB97BC01CE010D960E944A99CE010796E8
:10B6C0000E94E798CE0101960E94E798BE01635F51
:10B6D0007F4F8CEC93E10E949E9BB98860E08B2D9C
:10B6E0000E94318C0115110531F40B2DCE010D9600
:10B6F0000E94E79886CF60E0802F0E94318CF6CFC1
:10B70000CF93DF93EC01483085E058076105710560
:10B7100009F448C008F099C0493481E05807610530
:10B72000710509F4B2C008F040C0443481E0580704
:10B730006105710509F476C000F5413481E05807D0
:10B740006105710509F456C048F440345140610563
:10B75000710509F4E4C06EED7BE0E3C0423481E0A2
:10B7600058076105710509F409C143345140610569
:10B77000710589F765E17AE0D4C0463481E0580765
:10B780006105710509F40CC108F49FC0473481E0DC
:10B7900058076105710509F455C0483451406105E9
:10B7A0007105C9F666E77AE0BCC0423085E058070B
:10B7B0006105710509F4E2C000F5443781E05807DE
:10B7C0006105710509F4F2C040F44237514061054A
:10B7D000710509F66BEF7AE0A4C0411585E05807C2
:10B7E0006105710509F49BC0413055406105710543
:10B7F00009F0B1CF6BE17AE094C0453085E058079D
:10B800006105710509F461C080F4433085E0580793
:10B810006105710509F4AECF4430554061057105ED
:10B8200009F099CF62E17AE07CC0463085E05807A4
:10B830006105710509F4B4C04730554061057105D3
:10B8400009F089CF64E77AE06CC04D3B82E4580789
:10B850008FEF6807710509F4AFC008F048C04F3E8C
:10B8600080E158078FEF6807710561F3F8F4423300
:10B8700085E058076105710509F4ACCF48F44930FB
:10B8800055406105710509F066CF68E77AE049C067
:10B89000443385E058076105710509F487C04D3FC1
:10B8A00052406F4F710509F495CF55CF4D3D82E25F
:10B8B00058078FEF6807710509F478C048F4473ED0
:10B8C00058416F4F710509F046CF6FE07AE029C00B
:10B8D0004F3C80E358078FEF6807710509F4A2CF4A
:10B8E000473C58436F4F710509F45CCF34CF47395B
:10B8F00088E658078FEF6807710509F47BCF48F594
:10B900004D3A82E558078FEF6807710509F451C079
:10B9100078F4453B5A446F4F710509F01CCF68E13C
:10B9200077E0CE010E945399CE01DF91CF91089527
:10B93000453A8AE558078FEF6807710509F4A5CFE6
:10B940004D3952466F4F710509F005CF63ED75E033
:10B95000E8CF473588EA58078FEF6807710519F176
:10B9600080F445388AE758078FEF68077105C1F002
:10B97000473658496F4F710509F0EDCE68E17AE01E
:10B98000D0CF4F3480EB58078FEF6807710509F46B
:10B99000F1CE4D33524C6F4F710509F41BCFDBCE06
:10B9A00067EB7BE0BECF6DE878E0BBCF6DE77BE077
:10B9B000B8CF66ED75E0B5CF6AE77AE0B2CF0F9306
:10B9C0001F93CF93DF9300D000D0CDB7DEB7209187
:10B9D0000E0D2223A9F08C0166ED75E0CE010196D3
:10B9E0000E945399B801CE0101960E940198BC01B2
:10B9F0008DEA9FE00E94AC9BCE0101960E94E798E1
:10BA000026960FB6F894DEBF0FBECDBFDF91CF9163
:10BA10001F910F9108954F925F926F927F929F9224
:10BA2000AF92BF92CF92DF92EF92FF920F931F934C
:10BA3000CF93DF93CDB7DEB7A9970FB6F894DEBFEB
:10BA40000FBECDBF982E882351F080910E0D882314
:10BA500031F06EED7BE08DEA9FE00E94119A0E942A
:10BA6000B99560E08DE20E94009F60E18DE20E9446
:10BA7000009F68E08DE20E94009F40902F1350903D
:10BA800030136090311370903213498E5A8E6B8E42
:10BA90007C8EC0903313D0903413E0903513F09027
:10BAA0003613CD8EDE8EEF8EF8A2809137139091F3
:10BAB0003813A0913913B0913A138EA39FA3A8A76E
:10BAC000B9A789A39AA3ABA3BCA39920C9F180917C
:10BAD0000E0D8823A9F166EF74E1CE0101960E9454
:10BAE0004199CE0101960E94DF5CCE0101960E9431
:10BAF000E7988E01075E1F4F5E0195E2A90EB11C0B
:10BB0000D8016D917D918D919D918D0146E00E94AE
:10BB10005E9A62E67AE08DEA9FE00E949C9BA01606
:10BB2000B10671F76EED7BE0CE0101960E9453994C
:10BB3000CE0101960E94DF5CCE0101960E94E7983B
:10BB400023E938E144E85FE3C301B2010E9484B60F
:10BB50002B013C014D865E866F86788A22E430E6B2
:10BB600045E85FE3C701B6010E9484B66B017C0122
:10BB7000C98ADA8AEB8AFC8A25E83BEE41E95FE371
:10BB80006EA17FA188A599A50E9484B66D8B7E8B3E
:10BB90008F8B988F40922F135092301360923113F5
:10BBA00070923213C0923313D0923413E092351353
:10BBB000F0923613609337137093381380933913D0
:10BBC00090933A13992009F4A0C080910E0D882318
:10BBD00009F49BC069EE74E1CE0101960E9441997F
:10BBE000CE0101960E94DF5CCE0101960E94E7988B
:10BBF0008E01035F1F4F6E01B9E1CB0ED11C78019E
:10BC0000F80161917191819191918F0142E00E94BF
:10BC10005E9A62E67AE08DEA9FE00E949C9BC016E5
:10BC2000D10671F76EED7BE0CE0101960E9453992B
:10BC3000CE0101960E94DF5CCE0101960E94E7983A
:10BC40004BE353E166E070E082E30E942DA0A090F8
:10BC50003B13B0903C13C0903D13D0903E13009125
:10BC60003F13109140136CED74E18DEA9FE00E9448
:10BC7000BE9B4AE050E0B5018DEA9FE00E944F9BD9
:10BC800062E67AE08DEA9FE00E949C9B4AE050E0E9
:10BC9000B6018DEA9FE00E944F9B62E67AE08DEA52
:10BCA0009FE00E949C9B4AE050E0B8018DEA9FE033
:10BCB0000E944F9B6EED7BE08DEA9FE00E94119AFF
:10BCC000CE0101960E94ACA063ED74E18DEA9FE085
:10BCD0000E94BE9B8E010F5F1F4FD8016D917D9119
:10BCE0008D919D918D014AE00E945E9A62E67AE014
:10BCF0008DEA9FE00E949C9B0E151F0571F76EED6B
:10BD00007BE08DEA9FE00E94119A61E08DE10E9444
:10BD1000009F9920B1F080910E0D882391F06FEB78
:10BD200074E18DEA9FE00E94BE9BAE014B5D5F4FC8
:10BD300061E070E08DE10E942DA08DA190E00E9455
:10BD4000899B62E08EE10E94009F63E08FE10E9488
:10BD5000009F64E080E20E94009F992009F450C097
:10BD600080910E0D882309F44BC063EA74E18DEADB
:10BD70009FE00E94BE9BAE014B5D5F4F61E070E0B3
:10BD80008EE10E942DA0CDA0D12CAE014B5D5F4F66
:10BD900061E070E08FE10E942DA0EDA0F12CAE01DA
:10BDA0004B5D5F4F61E070E080E20E942DA00DA12D
:10BDB00010E04AE050E0B6018DEA9FE00E944F9B00
:10BDC00062E67AE08DEA9FE00E949C9B4AE050E0A8
:10BDD000B7018DEA9FE00E944F9B62E67AE08DEA10
:10BDE0009FE00E949C9B4AE050E0B8018DEA9FE0F2
:10BDF0000E944F9B6EED7BE08DEA9FE00E94119ABE
:10BE000065E081E20E94009F9920B1F080910E0DC3
:10BE1000882391F060E974E18DEA9FE00E94BE9B67
:10BE2000AE014B5D5F4F61E070E081E20E942DA0AA
:10BE30008DA190E00E94899B66E082E20E94009FB3
:10BE40009920B1F080910E0D882391F068E774E19C
:10BE50008DEA9FE00E94BE9BAE014B5D5F4F61E0AB
:10BE600070E082E20E942DA08DA190E00E94899B4B
:10BE700067E083E20E94009F9920B1F080910E0D4F
:10BE8000882391F062E674E18DEA9FE00E94BE9BF8
:10BE9000AE014B5D5F4F61E070E083E20E942DA038
:10BEA0008DA190E00E94899B68E084E20E94009F3F
:10BEB0009920B1F080910E0D882391F06AE474E12D
:10BEC0008DEA9FE00E94BE9BAE014B5D5F4F61E03B
:10BED00070E084E20E942DA08DA190E00E94899BD9
:10BEE00069E085E20E94009F9920B1F080910E0DDB
:10BEF000882391F060E374E18DEA9FE00E94BE9B8D
:10BF0000AE014B5D5F4F61E070E085E20E942DA0C5
:10BF10008DA190E00E94899B6AE086E20E94009FCA
:10BF20009920B1F080910E0D882391F06AE174E1BF
:10BF30008DEA9FE00E94BE9BAE014B5D5F4F61E0CA
:10BF400070E086E20E942DA08DA190E00E94899B66
:10BF50006BE088E20E94009F9920B1F080910E0D65
:10BF6000882391F061E074E18DEA9FE00E94BE9B1E
:10BF7000AE014B5D5F4F61E070E088E20E942DA052
:10BF80008DA190E00E94899B6CE089E20E94009F55
:10BF9000992009F479C080910E0D882309F474C0AA
:10BFA00069EE73E18DEA9FE00E94BE9BAE014B5D9E
:10BFB0005F4F61E070E089E20E942DA08DA190E0CA
:10BFC0000E94899B62ED73E18DEA9FE00E94BE9B17
:10BFD00066E070E087E20E9466A090E00E94899B84
:10BFE0006BEB73E18DEA9FE00E94BE9B65E070E021
:10BFF00087E20E9466A090E00E94899B64EA73E158
:10C000008DEA9FE00E94BE9B64E070E087E20E94A0
:10C0100066A090E00E94899B6BE873E18DEA9FE047
:10C020000E94BE9B62E070E087E20E9466A090E002
:10C030000E94899B62E773E18DEA9FE00E94BE9BAC
:10C0400061E070E087E20E9466A090E00E94899B18
:10C0500069E573E18DEA9FE00E94BE9B70E060E0BD
:10C0600087E20E9466A090E00E94899B68E473E1E9
:10C070008DEA9FE00E94BE9B63E070E087E20E9431
:10C0800066A090E00E94899B41E067E070E087E253
:10C090000E9481A041E063E070E087E20E9481A0FD
:10C0A00041E063E070E08AE20E9481A0992091F073
:10C0B00080910E0D882371F06FE273E18DEA9FE0AD
:10C0C0000E94BE9B63E070E08AE20E9466A090E05E
:10C0D0000E94899B40E063E070E08AE20E9481A0B8
:10C0E000992091F080910E0D882371F065E173E144
:10C0F0008DEA9FE00E94BE9B63E070E08AE20E94AE
:10C1000066A090E00E94899B41E062E070E08AE2D4
:10C110000E9481A0992091F080910E0D882371F0EA
:10C1200069EF72E18DEA9FE00E94BE9B62E070E0E1
:10C130008AE20E9466A090E00E94899B40E062E053
:10C1400070E08AE20E9481A0992091F080910E0D0A
:10C15000882371F06CED72E18DEA9FE00E94BE9B36
:10C1600062E070E08AE20E9466A090E00E94899BF3
:10C1700041E061E070E08AE20E9481A0992091F0A4
:10C1800080910E0D882371F060EC72E18DEA9FE0E2
:10C190000E94BE9B61E070E08AE20E9466A090E08F
:10C1A0000E94899B40E061E070E08AE20E9481A0E9
:10C1B000992091F080910E0D882371F063EA72E16D
:10C1C0008DEA9FE00E94BE9B61E070E08AE20E94DF
:10C1D00066A090E00E94899B41E070E060E08AE206
:10C1E0000E9481A0992091F080910E0D882371F01A
:10C1F00067E872E18DEA9FE00E94BE9B70E060E01C
:10C200008AE20E9466A090E00E94899B40E070E074
:10C2100060E08AE20E9481A0992091F080910E0D49
:10C22000882371F06AE672E18DEA9FE00E94BE9B6E
:10C2300070E060E08AE20E9466A090E00E94899B24
:10C2400041E066E070E087E20E9481A041E065E0A5
:10C2500070E087E20E9481A041E064E070E087E244
:10C260000E9481A040E062E070E087E20E9481A02D
:10C2700040E061E070E087E20E9481A040E070E071
:10C2800060E087E20E9481A0992009F475C0809146
:10C290000E0D882309F470C062E572E18DEA9FE01B
:10C2A0000E94BE9B66E070E08BE20E9466A090E078
:10C2B0000E94899B64E372E18DEA9FE00E94BE9B2D
:10C2C00065E070E08BE20E9466A090E00E94899B8E
:10C2D00066E172E18DEA9FE00E94BE9B64E070E03F
:10C2E0008BE20E9466A090E00E94899B6DEF71E155
:10C2F0008DEA9FE00E94BE9B62E070E08BE20E94AC
:10C3000066A090E00E94899B64EE71E18DEA9FE057
:10C310000E94BE9B61E070E08BE20E9466A090E00C
:10C320000E94899B6BEC71E18DEA9FE00E94BE9BAD
:10C3300070E060E08BE20E9466A090E00E94899B22
:10C3400068EB71E18DEA9FE00E94BE9B63E070E0C4
:10C350008BE20E9466A090E00E94899B63EA71E1F3
:10C360008DEA9FE00E94BE9B64E070E08CE20E9438
:10C3700066A090E00E94899B40E064E070E08CE25F
:10C380000E9481A0AE014B5D5F4F61E070E08CE2E6
:10C390000E942DA06DA1607F66608CE20E94009FCC
:10C3A000992009F45EC080910E0D882309F459C0CC
:10C3B0006FE871E18DEA9FE00E94BE9BAE014B5D8C
:10C3C0005F4F61E070E08CE20E942DA06DA16F7064
:10C3D0006650770B072E000C880B990B0E9425B630
:10C3E0009B01AC0160E070E080E090E40E9471BAD3
:10C3F00020E030E048EC50E40E9484B60E94409B6C
:10C4000068E771E18DEA9FE00E94BE9BAE014B5D43
:10C410005F4F61E070E080E30E942DA06DA14AE0D3
:10C4200050E08DEA9FE00E94FA9960E671E18DEAA2
:10C430009FE00E94BE9B61E070E080E30E9466A0E6
:10C4400090E00E94899B67E471E18DEA9FE00E9481
:10C45000BE9B61E070E08FE20E9466A090E00E94C7
:10C46000899B41E061E070E08FE20E9481A0992009
:10C4700091F080910E0D882371F06FE271E18DEAE9
:10C480009FE00E94BE9B61E070E08EE20E9466A089
:10C4900090E00E94899B41E061E070E08EE20E94A2
:10C4A00081A040E067E070E081E30E9481A09920D4
:10C4B00009F455C080910E0D882309F450C06CE139
:10C4C00071E18DEA9FE00E94BE9B67E070E081E32E
:10C4D0000E9466A090E00E94899B6CE77AE08DEA5A
:10C4E0009FE00E949C9BAE014B5D5F4F61E070E05E
:10C4F00080E00E942DA08DA10E94A4136EED7BE030
:10C500008DEA9FE00E94119A0DE110E06BE477E064
:10C510008DEA9FE00E949C9B40E150E0B8018DEACB
:10C520009FE00E944F9B60E87AE08DEA9FE00E94C6
:10C530009C9BAE014B5D5F4F61E070E0802F0E94DD
:10C540002DA08DA10E94A4136EED7BE08DEA9FE0EB
:10C550000E94119A0F5F1F4F0A331105B9F6A99671
:10C560000FB6F894DEBF0FBECDBFDF91CF911F9104
:10C570000F91FF90EF90DF90CF90BF90AF909F9082
:10C580007F906F905F904F9008951F93CF93DF93AC
:10C59000CDB7DEB7A8970FB6F894DEBF0FBECDBFFC
:10C5A000182F0E94B9958EE10E94168C62E08AE4F1
:10C5B00090E10E94FD0B60E08AE490E10E94FD0B97
:10C5C0000E94FD9E8EE10E94168C61E08AE490E15B
:10C5D0000E94FD0B60E28AE490E10E94FD0B0E9444
:10C5E000FD9E80E290E0909304138093031380E01B
:10C5F00090E8A9E8B4E48093E4049093E504A09360
:10C60000E604B093E70480E090E0A5E7B4E480930B
:10C61000E0049093E104A093E204B093E304BE012C
:10C620006F5F7F4F80E093E10E94C48B112309F478
:10C6300084C062E97CE08DEA9FE00E94BE9B8DEAA7
:10C640009FE00E94F69962E87CE08DEA9FE00E94FC
:10C65000BE9BBE016F5F7F4F8DEA9FE00E94119AE3
:10C6600062E77CE08DEA9FE00E94BE9B6D857E853F
:10C670008F8598890E942A9A62E67CE08DEA9FE085
:10C680000E94BE9B69897A898B899C890E942A9A1B
:10C6900062E57CE08DEA9FE00E94BE9B20E030E0F6
:10C6A00040E251E4698D7A8D8B8D9C8D0E9484B619
:10C6B00042E00E945E9A63E87AE08DEA9FE00E9481
:10C6C000119A62E47CE08DEA9FE00E94BE9B20E02C
:10C6D00030E040E251E46D8D7E8D8F8D98A10E94F7
:10C6E00084B642E00E945E9A63E87AE08DEA9FE0B9
:10C6F0000E94119A62E37CE08DEA9FE00E94BE9B5B
:10C7000020E030E040E251E469A17AA18BA19CA134
:10C710000E9484B642E00E945E9A63E87AE08DEA65
:10C720009FE00E94119A6CE07CE08DEA9FE00E94FD
:10C73000BE9B8DEA9FE00E94F69964EF71E080E075
:10C7400090E00E943AA1A8960FB6F894DEBF0FBE03
:10C75000CDBFDF91CF911F9108954F925F926F925D
:10C760007F928F929F92AF92BF92CF92DF92EF9281
:10C77000FF92CF93DF93CDB7DEB72C970FB6F89427
:10C78000DEBF0FBECDBF0E9415590E94DAA12B015A
:10C790003C010E9485A14B015C016091C90470912C
:10C7A000CA048091CB049091CC040E9425B66B0101
:10C7B0007C010E94DAA10E9425B6A70196010E9481
:10C7C0009DB821E03EED42E45EE30E9471BA9B0118
:10C7D000AC0160E070E080E89FE30E94BEB720E01B
:10C7E0003AE24DE257E40E9484B66B017C01C3013A
:10C7F000B2010E9425B620E030E048EC52E40E94ED
:10C800009DB8AB01BC0122E0CE0101960E94EF98D9
:10C81000BE016F5F7F4F89EB92E10E94AE98CE011F
:10C8200001960E94E79869E076E089EB92E10E9428
:10C83000619869EB72E18FEB92E10E94979865E055
:10C8400076E0CE0101960E94539969EB72E1CE0128
:10C8500001960E940198BC0189EB92E10E94979891
:10C86000CE0101960E94E79868EF76E085EC92E1B0
:10C870000E94679621E0B501A401CE0101960E94B5
:10C88000EF98BE016F5F7F4F85EC92E10E946B983D
:10C89000CE0101960E94E79867E87AE085EC92E184
:10C8A0000E94619821E0B701A601CE0101960E9485
:10C8B000EF98BE016F5F7F4FCE0107960E944A99A5
:10C8C00064E37BE0CE0107960E94EB97BC0185EC08
:10C8D00092E10E946B98CE0107960E94E798CE01E4
:10C8E00001960E94E79869EB72E1CE0101960E94E1
:10C8F0004A9962E67AE0CE0101960E94EB9765ECD8
:10C9000072E10E940198BC0185EC92E10E94979827
:10C91000CE0101960E94E79821E0B501A401CE0165
:10C9200001960E94EF98BE016F5F7F4F8BEC92E102
:10C930000E94AE98CE0101960E94E7986BEC72E1DE
:10C94000CE0101960E944A994AE050E070E060E012
:10C95000CE0101960E94DD5ACE0101960E94E79811
:10C9600065E070E080E090E00E943AA163ED75E040
:10C97000CE0101960E945399CE0101960E94395929
:10C98000CE0101960E94E7986FEB72E1CE0101960D
:10C990000E944A994AE050E06FEF7FEFCE01019686
:10C9A0000E945759CE0101960E94E79820E0B701F6
:10C9B000A601CE0101960E94EF98BE016F5F7F4FE6
:10C9C000CE0107960E944A9964E37BE0CE01079668
:10C9D0000E94EB97BC018BEC92E10E949798CE01EC
:10C9E00007960E94E798CE0101960E94E7986BECAB
:10C9F00072E1CE0101960E944A994AE050E064EF4C
:10CA00007FEFCE0101960E945759CE0101960E94F8
:10CA1000E79865E070E080E090E00E943AA18091A4
:10CA20000D0D882331F068E572E080E090E00E940F
:10CA30003AA12C960FB6F894DEBF0FBECDBFDF91A2
:10CA4000CF91FF90EF90DF90CF90BF90AF909F90ED
:10CA50008F907F906F905F904F9008952F923F92AC
:10CA60004F925F926F927F928F929F92AF92BF92FE
:10CA7000CF92DF92EF92FF920F931F93CF93DF93AA
:10CA8000CDB7DEB7C854D1090FB6F894DEBF0FBEDC
:10CA9000CDBF2B013C012DA73EA74FA758AB28EED9
:10CAA000421623E052066104710434F030E9432E4B
:10CAB00055245394612C712CCDA4DEA4EFA4F8A8C6
:10CAC00020E1C21627E2D206E104F10454F020E18D
:10CAD000C22E27E2D22EE12CF12CCDA6DEA6EFA6A7
:10CAE000F8AA80910D0D882341F0C12CD12C76013C
:10CAF000C394CDA6DEA6EFA6F8AA0E94D6A72596D7
:10CB00006CAF7DAF8EAF9FAF25970E94D6A76DAB60
:10CB10007EAB8FAB98AF25966CAD7DAD8EAD9FADE6
:10CB2000259728EE33E040E050E00E945BB729965D
:10CB30002CAF3DAF4EAF5FAF299721E02DA319A6D3
:10CB40001AA61BA61CA68E01035F1F4FCC24DD2452
:10CB50007601C418D508E608F708C9AADAAAEBAA2C
:10CB6000FCAA6DA97EA98FA998AD2596CCACDDACA9
:10CB7000EEACFFAC25976C197D098E099F09CDA4F9
:10CB8000DEA4EFA4F8A86C157D058E059F050CF0BA
:10CB9000B8C30E9425B620E030E04AE754E40E9482
:10CBA0009DB8AB01BC0123E0C8010E94EF98B80119
:10CBB0008FEB92E10E94AE98C8010E94E798A7010E
:10CBC00096012A303105410551058CF429964CAD6A
:10CBD0005DAD6EAD7FAD2997C8010E947196B80119
:10CBE0008FEB92E10E94AE98C8010E94E798809175
:10CBF0000D0D882309F470C26EED7BE08FEB92E19E
:10CC00000E946796CE0101960E94ACA06EED7BE07B
:10CC100085EC92E10E946796AE014F5F5F4F1A016B
:10CC2000812C912C5401D101CD90DD90ED90FD909F
:10CC30001D01A7019601C701B6010E9484B69B01A0
:10CC4000AC01C501B4010E94BFB74B015C0123E0F8
:10CC5000B701A601C8010E94EF98B801CE01439622
:10CC60000E944A9962E67AE0CE0143960E94EB97D1
:10CC7000BC0185EC92E10E946B98CE0143960E9424
:10CC8000E798C8010E94E7982016310661F6C501B1
:10CC9000B4010E94C7BA4B015C01BDE24B16B1E082
:10CCA0005B066104710434F00E94155960E080E075
:10CCB0000E94318C23E0B501A401CE0143960E946D
:10CCC000EF986DED7BE0C8010E9453996FEB72E124
:10CCD000C8010E9401986DE87AE00E94EB97BE01BE
:10CCE0006D5E7F4F0E94019861E97AE00E94EB97A8
:10CCF000BC0185EC92E10E946B98C8010E94E79804
:10CD0000CE0143960E94E7982AE939E949E55FE3B5
:10CD1000C501B4010E94A6B918160CF0F4C123E3B2
:10CD200033E343E95FE3C501B4010E941EB6880FF7
:10CD3000880BCDA0C822CDA28091100C9091110C2F
:10CD40008130910509F4F4C1029721F0DDA0DD20C6
:10CD500009F4EEC189849A84AB84BC84C980DA80EA
:10CD6000EB80FC80CDA2DEA2EFA2F8A6CD80DE8013
:10CD7000EF80F88420E030E0A901C501B4010E94F1
:10CD80001EB6882309F4C1C12DA13EA14FA158A50B
:10CD9000CA01B9010E9484B669AF7AAF8BAF9CAF6C
:10CDA000A7019601C701B6010E9484B69B01AC01A0
:10CDB00069AD7AAD8BAD9CAD0E94BFB70E94C7BA7A
:10CDC000A50194010E943EB820EE3EE245E652E401
:10CDD0000E9484B669AF7AAF8BAF9CAF20E030E0A1
:10CDE000A901C701B6010E941EB6882309F492C1A9
:10CDF0002DA13EA14FA158A5CA01B9010E9484B638
:10CE000021966CAF7DAF8EAF9FAF2197A5019401A6
:10CE1000C501B4010E9484B69B01AC0121966CADA2
:10CE20007DAD8EAD9FAD21970E94BFB70E94C7BA5E
:10CE3000A70196010E943EB820EE3EE245E652E48C
:10CE40000E9484B621966CAF7DAF8EAF9FAF2197C5
:10CE500020E030E0A9016DA17EA18FA198A50E94DC
:10CE60001EB6882309F45BC1A5019401C501B40174
:10CE70000E9484B64B015C01A7019601C701B6016F
:10CE80000E9484B69B01AC01C501B4010E94BFB7EA
:10CE90000E94C7BA2DA13EA14FA158A50E943EB83D
:10CEA0006B017C016FEB72E1C8010E944A9960EB53
:10CEB00071E1C8010E940198BC0185EC92E10E94D9
:10CEC0009798C8010E94E79865EC72E1C8010E943A
:10CED0004A99C8010E94FE58C8010E94E79821E0C3
:10CEE00049AD5AAD6BAD7CADCE014F960E94EF9827
:10CEF00021E021964CAD5DAD6EAD7FAD2197CE01A9
:10CF000049960E94EF9820EE3EE245E652E4C701C2
:10CF1000B6010E9484B6AB01BC0121E0C8010E94A9
:10CF2000EF98B801CE0143960E944A9962E67AE0F2
:10CF3000CE0143960E94EB97BE01675E7F4F0E9431
:10CF4000019862E67AE00E94EB97BE01615E7F4F36
:10CF50000E940198BC0185EC92E10E949798CE0155
:10CF600043960E94E798C8010E94E798CE0149962F
:10CF70000E94E798CE014F960E94E7986DEA78E00C
:10CF8000C8010E94539965EC72E1C8010E940198A2
:10CF9000BC0189EB92E10E949798C8010E94E79832
:10CFA00069EB72E1C8010E944A99C8010E946D189C
:10CFB000C8010E94E79865EC72E189EB92E10E945A
:10CFC000979865EC72E1C8010E944A99C8010E94D5
:10CFD000E158C8010E94E7982DE2421621E052066E
:10CFE0006104710474F469A57AA58BA59CA525E05C
:10CFF00030E040E050E00E945BB7672B682B692B64
:10D00000A9F56CE075E18FEB92E10E94729864E9FA
:10D010007AE0C8010E94539945E050E067EF7FEF46
:10D02000C8010E94DD5AC8010E94E7986EED7BE0BE
:10D03000C8010E945399C8010E943959C8010E9431
:10D04000E79865EC72E1C8010E944A9945E050E01A
:10D0500070E060E0C8010E945759C8010E94E7983B
:10D060006EED7BE085EC92E10E946796B201C30110
:10D0700077FE04C069A97AA98BA99CA90E943AA14C
:10D0800031E03DA30E94D6A76B017C012DA93EA9EA
:10D090004FA958ADC21AD30AE40AF50AC9A6DAA6FE
:10D0A000EBA6FCA6C414D504E604F70444F4C301BB
:10D0B000B2016C197D098E099F090E943AA10E9454
:10D0C000D6A76DAB7EAB8FAB98AF6EED7BE085ECFA
:10D0D00092E10E94679645CD63ED7AE0C8010E9417
:10D0E00053996FEB72E1C8010E94019866E979E0FB
:10D0F0000E94EB97BC018FEB92E10E949798C801C8
:10D100000E94E7987FCD1DA217CE6BED7FE089ECE2
:10D110009FE35ACE6BED7FE089EC9FE38DCE8BEDE4
:10D12000C82E8FE0D82E89ECE82E8FE3F82EBACEE9
:10D130006BE97AE0C8010E94539965EC72E1C8017D
:10D140000E940198BC0185EC92E10E949798C80169
:10D150000E94E79865EC72E1C8010E944A99C801F3
:10D160000E94E158C8010E94E79865EC72E1C8018D
:10D170000E944A99C8010E946D18C8010E94E79850
:10D1800023E0B501A401CE0143960E94EF986EE81A
:10D190007AE0C8010E945399BE016D5E7F4FC801BD
:10D1A0000E94019861E97AE00E94EB97BC0185EC4E
:10D1B00092E10E949798C8010E94E798CE01439699
:10D1C0000E94E79865EC72E1C8010E944A99C80183
:10D1D0000E946D18C8010E94E7986FEB72E1C801C8
:10D1E0000E944A9965EC72E1C8010E940198BC0155
:10D1F00085EC92E10E949798C8010E94E79868EA3E
:10D200007AE08FEB92E10E94619849855A856B859F
:10D210007C8522E0CE014F960E94EF984D815E8181
:10D220006F81788522E0CE0149960E94EF9849816E
:10D230005A816B817C8122E0C8010E94EF98B8017D
:10D24000CE0143960E944A9962E67AE0CE01439667
:10D250000E94EB97BE01675E7F4F0E94019862E6D5
:10D260007AE00E94EB97BE01615E7F4F0E940198B9
:10D27000BC0189EB92E10E949798CE0143960E94EF
:10D28000E798C8010E94E798CE0149960E94E79866
:10D29000CE014F960E94E7984DE2441641E05406B5
:10D2A0006104710474F469A57AA58BA59CA525E099
:10D2B00030E040E050E00E945BB7672B682B692BA1
:10D2C000F1F46FEB72E1C8010E944A9948E050E026
:10D2D0006FEF7FEFC8010E94335AC8010E94E798A0
:10D2E00069EB72E1C8010E944A994AE050E070E09F
:10D2F00060E0C8010E945759C8010E94E7981DA22A
:10D30000C1CE6FEB72E1CE010D960E944A994AE0C0
:10D3100050E06FEF7FEFCE010D960E94DD5ACE01F7
:10D320000D960E94E798CDA0CC2001F164E075E154
:10D33000CE010D960E94419945E050E070E060E01A
:10D34000CE010D960E94DD5ACE010D960E94E798FF
:10D350006EED7BE0CE010D960E945399CE010D96A5
:10D360000E943959CE010D960E94E79869EB72E14F
:10D37000CE010D960E944A994AE050E06FEF7FEF90
:10D38000CE010D960E945759CE010D960E94E79846
:10D39000C85BDF4F0FB6F894DEBF0FBECDBFDF9185
:10D3A000CF911F910F91FF90EF90DF90CF90BF90A2
:10D3B000AF909F908F907F906F905F904F903F9035
:10D3C0002F9008954F925F926F927F928F929F92CB
:10D3D000AF92BF92CF92DF92EF92FF920F931F9383
:10D3E000CF93DF93CDB7DEB7CA54D1090FB6F89407
:10D3F000DEBF0FBECDBF8C016EED7BE0CE01C796C8
:10D400000E9453996EED7BE0CE01CD960E94539918
:10D41000BE016F5F7F4F80E093E10E942F0CCD88AB
:10D42000DE88EF88F88C20E030E040E251E4C7016C
:10D43000B6010E9484B62B013C01898D9A8DAB8D7B
:10D44000BC8D2B968CAF9DAFAEAFBFAF2B9720E0BE
:10D4500030E040E251E4BC01CD010E9484B64B01B2
:10D460005C0120E030E040E251E46D8D7E8D8F8DD7
:10D4700098A10E9484B627966CAF7DAF8EAF9FAF08
:10D480002797C701B60190582B962CAD3DAD4EADF8
:10D490005FAD2B970E943EB82BED3FE049EC5FE378
:10D4A0000E94BFB72091C5043091C6044091C704C3
:10D4B0005091C8040E94BFB76B017C0120E030E0AE
:10D4C000A9010E941EB687FDCFC2C092B90CD092AE
:10D4D000BA0CE092BB0CF092BC0CC090B90CD0908E
:10D4E000BA0CE090BB0CF090BC0C2BED3FE049EC8B
:10D4F00050E4C701B6010E94A6B9181684F42BEDBA
:10D500003FE049EC50E4C701B6010E94BEB760930A
:10D51000B90C7093BA0C8093BB0C9093BC0C20E0B8
:10D5200030E044E353E46091B90C7091BA0C8091FF
:10D53000BB0C9091BC0C0E9484B62BED3FE049E4FB
:10D5400050E40E949DB86093B50C7093B60C809324
:10D55000B70C9093B80C0E9449B9CE018B960E94EB
:10D560009E9661EB7AE0CE0185960E945399BE01AA
:10D57000655D7F4FCE0185960E9401986BEB7AE046
:10D580000E94EB97BC018BEC92E10E949798CE0130
:10D5900085960E94E798CE018B960E94E798C090EE
:10D5A000B50CD090B60CE090B70CF090B80C20E021
:10D5B00030E044EB52E4C701B6010E941EB61816D3
:10D5C0000CF463C220E030E040E05FE3C701B60145
:10D5D0000E94BFB70E9449B9CE018B960E949E96C9
:10D5E00062EC7AE0CE0185960E945399BE01655D9A
:10D5F0007F4FCE0185960E940198BC01CE01C7964F
:10D600000E949798CE0185960E94E798CE018B964E
:10D610000E94E79862EC79E0CE01CD960E94679671
:10D62000BE01695C7F4FCE0185960E944A994AE00F
:10D6300050E070E060E0CE0185960E94DD5ACE0198
:10D6400085960E94E7980E94D6A7AB01BC01809105
:10D65000BD0C9091BE0CA091BF0CB091C00C8C5928
:10D660009F4FAF4FBF4F84179507A607B70708F026
:10D6700091C26EED7BE0CE0185960E945399CE015A
:10D6800085960E943959CE0185960E94E798BE0181
:10D69000635C7F4F8CEC93E10E949E9B62E67AE094
:10D6A000CE0185960E945399BE01635C7F4FCE01E7
:10D6B00085960E940198BC01CE01C7960E946B9886
:10D6C000CE0185960E94E7980E94D6A7C090C90C0B
:10D6D000D090CA0CE090CB0CF090CC0C6C197D096A
:10D6E0008E099F090E9423B620E030E04AE754E407
:10D6F0000E949DB8AB01BC0123E0CE018B960E9435
:10D70000EF9863ED7AE0CE0185960E945399BE01B1
:10D71000655D7F4FCE0185960E94019866E979E0AC
:10D720000E94EB97BC0189EB92E10E949798CE0191
:10D7300085960E94E798CE018B960E94E79869EB48
:10D7400072E1CE0185960E944A996BEC72E1CE019E
:10D7500085960E940198BE01695C7F4F0E940198E6
:10D76000BC01CE01C7960E949798CE0185960E9473
:10D77000E7986DEB7CE085EC92E10E94729821E0E5
:10D78000B301A201CE0185960E94EF98BE016B5DA8
:10D790007F4F85EC92E10E946B98CE0185960E94A6
:10D7A000E79821E027964CAD5DAD6EAD7FAD279734
:10D7B000CE01C1960E94EF9821E0B501A401CE01EF
:10D7C0008B960E94EF9862E67AE0CE0185960E94E1
:10D7D0005399BE01655D7F4FCE0185960E940198E9
:10D7E00062E67AE00E94EB97BE016F5C7F4F0E9479
:10D7F00001986AEC7AE00E94EB97BC0185EC92E11B
:10D800000E946B98CE0185960E94E798CE018B9678
:10D810000E94E798CE01C1960E94E798A301920169
:10D82000C301B2010E9484B66B017C01A501940181
:10D83000C501B4010E9484B69B01AC01C701B601C9
:10D840000E94BFB76B017C0127962CAD3DAD4EAD5C
:10D850005FAD2797CA01B9010E9484B69B01AC0154
:10D86000C701B6010E94BFB70E94C7BA6093B10C4E
:10D870007093B20C8093B30C9093B40C6EEC7AE07E
:10D8800085EC92E10E9461984091B10C5091B20CEC
:10D890006091B30C7091B40C21E0CE0185960E948A
:10D8A000EF98BE016B5D7F4FCE018B960E944A9927
:10D8B00064E87AE0CE018B960E94EB97BC018BEC7A
:10D8C00092E10E949798CE018B960E94E798CE0134
:10D8D00085960E94E7986BEC72E185EC92E10E94DC
:10D8E0006B98C090B10CD090B20CE090B30CF0905B
:10D8F000B40C20E030E04AE754E4C701B6010E94CE
:10D90000A6B987FD29C020E030E04AE754E4C7010A
:10D91000B6010E949DB8AB01BC0123E0CE01859603
:10D920000E94EF98BE016B5D7F4FCE018B960E94E7
:10D930004A9965E87AE0CE018B960E94EB97BC018C
:10D940008BEC92E10E949798CE018B960E94E7980B
:10D95000CE0185960E94E79820E030E64AE656E43C
:10D960006091B10C7091B20C8091B30C9091B40C99
:10D970000E941EB6BE01695C7F4F87FF2AC1CE019F
:10D9800085960E944A9962ED7AE0CE0185960E94C2
:10D99000EB9765EC72E10E940198BC0185EC92E185
:10D9A0000E949798CE0185960E94E7980330110552
:10D9B000A1F465EC72E1CE0185960E944A99CE01F0
:10D9C00085960E94E158CE0185960E94E7986EEDFB
:10D9D0007BE085EC92E10E94679665ED7AE0CE01EE
:10D9E00085960E9453996BEC72E1CE0185960E9458
:10D9F0000198BC01CE018B960E944A994AE050E002
:10DA00006FEF7FEFCE018B960E945759CE018B9618
:10DA10000E94E798CE0185960E94E7986AE070E040
:10DA200080E090E00E943AA1CE01CD960E94E79856
:10DA3000CE01C7960E94E798C65BDF4F0FB6F894F9
:10DA4000DEBF0FBECDBFDF91CF911F910F91FF9031
:10DA5000EF90DF90CF90BF90AF909F908F907F908E
:10DA60006F905F904F9008952BED3FE049EC50E4AC
:10DA7000C701B6010E94BFB76093B90C7093BA0C8E
:10DA80008093BB0C9093BC0C28CD20E030E044E3A5
:10DA900053E4C701B6010E941EB61816CCF0A701C8
:10DAA000960160E070E884E393E40E94BEB760935F
:10DAB000B50C7093B60C8093B70C9093B80C0E9481
:10DAC00049B9CE018B960E949E9665EC7AE08ACD8C
:10DAD00020E030E047E853E4C701B6010E941EB6DB
:10DAE0001816CCF120E030E044E353E4C701B6015E
:10DAF0000E94BEB720E030E040E05FE30E94BFB785
:10DB00006093B50C7093B60C8093B70C9093B80CDF
:10DB10000E9449B9CE018B960E949E9665EC7AE0F0
:10DB2000CE0185960E945399BE01655D7F4FCE015F
:10DB300085960E940198BC01CE01C7960E949798D5
:10DB4000CE0185960E94E798CE018B960E94E798B9
:10DB500068EC7AE061CDA701960160E070E084EBAB
:10DB600093E40E94BEB720E030E040E05FE30E9413
:10DB7000BFB76093B50C7093B60C8093B70C9093BD
:10DB8000B80C0E9449B9CE018B960E949E9662EC19
:10DB90007AE0C6CF0E94D6A70E9423B66B017C0113
:10DBA0006091BD0C7091BE0C8091BF0C9091C00C27
:10DBB0000E9425B620E030E048EC51E40E94BFB757
:10DBC0009B01AC01C701B6010E941EB687FD51CD75
:10DBD00065CD85EC92E10E94979820CFDF92EF927D
:10DBE000FF920F931F93CF93DF93CDB7DEB762976A
:10DBF0000FB6F894DEBF0FBECDBF8C011092020DA0
:10DC00006EED7BE0CE010D960E945399FF24F394B4
:10DC10008DEA9FE00E9467892091020D181619066F
:10DC20007CF521112DC08DEA9FE00E9445898A3044
:10DC300009F07EC089899A89892B09F481C0F09204
:10DC4000020D6EED7AE0CE0101960E945399BE015D
:10DC5000635F7F4FCE0101960E940198BC01CE0107
:10DC600007960E944A99CE0107960E94DF5CCE017A
:10DC700007960E94E798CE0101960E94E79860C03F
:10DC8000F12CE12CDD24D394222309F460C089898E
:10DC90009A89019709F045C064ED76E0CE010796B8
:10DCA0000E945399BE01695F7F4FCE010D960E947D
:10DCB000D097F12C811115C06BEF77E0CE01019662
:10DCC0000E945399BE016F5F7F4FCE010D960E9457
:10DCD000D097FF24F3948111F12CCE0101960E947C
:10DCE000E798CE0107960E94E798FF20A1F050E048
:10DCF00040E0BE01635F7F4FCE0101960E94275A2C
:10DD0000BE016F5F7F4F81ED92E10E94AE98CE0120
:10DD100001960E94E79864E170E080E090E00E9444
:10DD20003AA1BE01635F7F4FC8010E94389990C03D
:10DD30008D3009F47FCF682FCE010D960E943E985A
:10DD40006AE070E080E090E00E943AA161CF86ED49
:10DD50009DE00E9467891816190614F586ED9DE06E
:10DD60000E9445898A30A9F08D3099F09091020D7A
:10DD700091110FC0682FCE010D960E943E988FEF33
:10DD8000E81AF80A65E070E080E090E00E943AA1AD
:10DD9000DECF89899A89892BA9F3D092020DF2CF1F
:10DDA00064E170E080E090E00E943AA1EF28D1F1B8
:10DDB00089899A89892BB1F180910E0D882361F1AF
:10DDC00066ED75E0CE0101960E945399BE016F5F2A
:10DDD0007F4FCE010D960E94D097F82ECE0101966E
:10DDE0000E94E798F11018C067EE7AE08DEA9FE094
:10DDF0000E949C9BBE01635F7F4FCE0101960E94F3
:10DE00004A99BE016F5F7F4F8DEA9FE00E94AC9BF5
:10DE1000CE0101960E94E79864E170E080E090E016
:10DE20000E943AA189899A892091020D211131CF4E
:10DE3000009709F02ECF64E670E080E090E00E9449
:10DE40003AA10E94D6A76EED7BE0C8010E945399CB
:10DE5000CE010D960E94E798C80162960FB6F8941D
:10DE6000DEBF0FBECDBFDF91CF911F910F91FF900D
:10DE7000EF90DF900895DF92EF92FF920F931F9340
:10DE8000CF93DF93CDB7DEB72C970FB6F894DEBFF4
:10DE90000FBECDBF8C011092020D6EED7BE0CE0166
:10DEA00007960E945399F12CE12CDD24D39486ED42
:10DEB0009DE00E9467891816190694F48091020D5E
:10DEC00081110EC086ED9DE00E9445898A30D1F512
:10DED0008B859C85892B09F443C0D092020D40C0EC
:10DEE00062E370E080E090E00E943AA1EF2851F0F8
:10DEF00086ED9DE00E940A8A64E670E080E090E092
:10DF00000E943AA18091020D811131C08B859C85C0
:10DF1000892B69F56EED7BE0C8010E945399CE0113
:10DF200007960E94E798C8012C960FB6F894DEBFBA
:10DF30000FBECDBFDF91CF911F910F91FF90EF905A
:10DF4000DF9008958D3021F29091020D9111C0CF94
:10DF5000682FCE0107960E943E988FEFE81AF80AC4
:10DF60006FE070E080E090E00E943AA1A0CF809145
:10DF70000E0D882379F0BE01695F7F4FCE010196B7
:10DF80000E944A99CE0101960E94E158CE01019665
:10DF90000E94E798BE01695F7F4FC8010E943899CF
:10DFA000BECF4F925F926F927F928F929F92AF926D
:10DFB000BF92EF92FF920F931F93CF93DF93CDB752
:10DFC000DEB762970FB6F894DEBF0FBECDBF7C01FF
:10DFD0005B0182EF9CE00E94308F892BD9F46EEDBB
:10DFE0007BE0C7010E945399C70162960FB6F8946F
:10DFF000DEBF0FBECDBFDF91CF911F910F91FF907C
:10E00000EF90BF90AF909F908F907F906F905F90B8
:10E010004F9008954091F60C5091F70C6091F80CD8
:10E020007091F90CCE0107960E94805B80910E0DD5
:10E03000882359F16EEE7AE0CE0101960E94539941
:10E04000BE01695F7F4FCE0101960E9401986FEA81
:10E0500078E00E94EB97BC018DEA9FE00E949E9BB6
:10E06000CE0101960E94E7984091F60C5091F70C72
:10E070006091F80C7091F90C20E18DEA9FE00E940C
:10E08000AA998DEA9FE00E94F69970E060E0CE01C7
:10E0900007960E94BF97182F8A3211F01092F60B44
:10E0A0000E94D6A76093050D7093060D8093070D0F
:10E0B0009093080D6EED7BE0CE010D960E94539972
:10E0C000812F110F990BC0970A9708F068C0CE01F5
:10E0D00007960E94E49663307105810591050CF066
:10E0E00084C001E010E082E0982E0A151B0509F4B7
:10E0F0007CC06CE271E080E090E00E943AA19092D6
:10E10000561010925910412C512C320182EE9CE095
:10E110000E94308F892B91F48EE1481651046104DE
:10E12000710449F16EE170E080E090E00E943AA154
:10E130008FEF481A580A680A780AE8CF8EE1481625
:10E14000510461047104B9F04091E60C5091E70C60
:10E150006091E80C7091E90CCE0101960E94805B01
:10E16000BE016F5F7F4FCE010D960E94AE98CE012B
:10E1700001960E94E79889899A89892B39F0BE0116
:10E18000635F7F4FCE0107960E946B980F5F1F4F12
:10E190006EED7BE0CE010D960E946796A6CF6CE2F5
:10E1A00071E080E090E00E943AA182E080935610F6
:10E1B00010925910812C912C540182EE9CE00E9407
:10E1C000308F892B61F58EE188169104A104B1048A
:10E1D00009F043C089899A89892B39F0BE01635FB0
:10E1E0007F4FCE0107960E946B9864E670E080E056
:10E1F00090E00E943AA182E080935610109259104C
:10E20000BE01695F7F4FC7010E943899CE010D960C
:10E210000E94E798CE0107960E94E798E5CE8EE12E
:10E2200088169104A104B104A9F24091E60C509122
:10E23000E70C6091E80C7091E90CCE0101960E9408
:10E24000805BBE016F5F7F4FCE010D960E94AE983E
:10E25000CE0101960E94E798BDCF6EE170E080E0AC
:10E2600090E00E943AA18FEF881A980AA80AB80A8B
:10E27000A4CFAF92BF92CF92DF92EF92FF920F9313
:10E280001F93CF93DF93CDB7DEB72C970FB6F894DB
:10E29000DEBF0FBECDBF7C015B010E9431A9182FEC
:10E2A000811117C06EED7BE0C7010E945399C70131
:10E2B0002C960FB6F894DEBF0FBECDBFDF91CF9185
:10E2C0001F910F91FF90EF90DF90CF90BF90AF9094
:10E2D00008958A3211F01092F60B0E94D6A760932F
:10E2E000050D7093060D8093070D9093080D612F17
:10E2F000CE0107960E941F99812F012E000C990BC9
:10E30000C0970A9768F5CE0107960E94E49663309D
:10E310007105810591050CF070C001E010E00A154F
:10E320001B0509F46AC062E370E080E090E00E949F
:10E330003AA10E9431A9D12CC12C81113BC08FEF91
:10E34000C81AD80A85E1C816D10409F456C06EE18E
:10E3500070E080E090E00E943AA10E9431A9EDCFE8
:10E36000612FCE0101960E941F99BE016F5F7F4F02
:10E37000CE0107960E94AE98CE0101960E94E798C2
:10E3800062E370E080E090E00E943AA10E9431A92F
:10E3900010E000E0811121C00F5F1F4F0F31110508
:10E3A00061F16EE170E080E090E00E943AA10E948D
:10E3B00031A9F0CF682FCE0101960E941F99BE01AE
:10E3C0006F5F7F4FCE0107960E946B98CE0101963A
:10E3D0000E94E7980F5F1F4FA2CF682FCE010196D2
:10E3E0000E941F99BE016F5F7F4FCE0107960E946A
:10E3F0006B98CE0101960E94E798BE01695F7F4F3E
:10E40000C7010E943899CE0107960E94E7984FCF26
:10E410003F924F925F926F927F928F929F92AF92B4
:10E42000BF92CF92DF92EF92FF920F931F93CF9301
:10E43000DF93CDB7DEB7E4970FB6F894DEBF0FBE1B
:10E44000CDBF8091F60B8823D1F01092F60BE496A5
:10E450000FB6F894DEBF0FBECDBFDF91CF911F91F5
:10E460000F91FF90EF90DF90CF90BF90AF909F9073
:10E470008F907F906F905F904F903F90089581E0D4
:10E480008093F60B6EED7BE0CE0185960E9453994A
:10E490006EED7BE0CE018B960E94539910E000E078
:10E4A00082E0382E98EEC92E93E0D92EE12CF12C83
:10E4B000F8013197E031F105B0F48827ED59FD48B6
:10E4C0008F4F0C9449BB4873DF73F473FD7306746C
:10E4D0000F74207429745874697472747B74847412
:10E4E0001F75287531756EED7BE0CE0185960E9413
:10E4F000679680919E1190919F11892B31F46CE663
:10E5000076E0CE0185960E94679680919E1190914B
:10E510009F11019731F466E676E0CE0185960E9460
:10E52000679680919E1190919F11029731F460E758
:10E5300076E0CE0185960E94679689A59AA5892BDB
:10E5400031F064EB73E1CE0185960E946B9865E72C
:10E5500076E0CE0101960E94539960EC73E1CE0102
:10E5600001960E940198BC01CE018B960E9497985B
:10E57000CE0101960E94E79880919E1190919F1183
:10E58000019709F046C0BE016B5D7F4FCE01019639
:10E590000E944A9948EC50E06FEF7FEFCE01019660
:10E5A0000E94DD5ACE0101960E94E798BE01655D8A
:10E5B0007F4FCE0101960E944A9940ED57E06FEFE0
:10E5C0007FEFCE0101960E945759CE0101960E941D
:10E5D000E798CE0101960E9414328D819E810097AA
:10E5E000A1F0E981FA812081222379F0079768F070
:10E5F00065EF7EE0CE0185960E947298BE016F5F46
:10E600007F4FCE018B960E949798CE0101960E9473
:10E61000E798BE016B5D7F4FCE0101960E944A993B
:10E6200048EC50E06FEF7FEFCE0101960E94335A25
:10E63000CE0101960E94E798BE01655D7F4FCE0135
:10E6400001960E944A9948EC50E06FEF7FEFCE01AF
:10E6500001960E945759CE0101960E94E7980E94A8
:10E6600031A9982EB12CA12C911060C28FEFA81A5D
:10E67000B80A95E6A916B10409F4FCC10E9431A9B3
:10E68000982E64E170E080E090E00E943AA1ECCF27
:10E6900069EE7EE0CE0185960E9472980E94D6A710
:10E6A0004B015C010E94D6A7A70196010E948DB77D
:10E6B000CA01B90120E831E541E050E00E948DB780
:10E6C00020E13EE040E050E00E945BB729AB3AAB6E
:10E6D0004BAB5CAB2CE330E040E050E00E945BB71A
:10E6E00029013A01AB01BC01CE0101960E9471964D
:10E6F000B301A201CE0107960E94719649A95AA9B9
:10E700006BA97CA9CE010D960E947196C501B4013A
:10E7100020E03CE546E255E00E948DB7BA01A90130
:10E72000CE0149960E947196BE01675E7F4FCE0171
:10E7300043960E944A9963EF7AE0CE0143960E9485
:10E74000EB97BE01635F7F4F0E94019866EF7AE00E
:10E750000E94EB97BE01695F7F4F0E9401986BECAE
:10E7600076E00E94EB97BE016F5F7F4F0E94019899
:10E7700064ED76E00E94EB97BC01CE014F960E94BB
:10E780004A99CE0143960E94E798CE0149960E948D
:10E79000E798CE010D960E94E798CE0107960E9459
:10E7A000E798CE0101960E94E798BE01615E7F4F17
:10E7B000CE018B960E94AE98CE014F9628CF8091C5
:10E7C0000E0C90910F0C6AED7EE0019711F06CEC4D
:10E7D0007EE0CE0185960E9472986CEB7EE0CE01C1
:10E7E0008B960E94729815CF6CEA7EE0CE018596DA
:10E7F0000E9472986FE97EE0F2CF62E97EE0CE017E
:10E8000085960E94729867E87EE0E9CF6BE77EE02C
:10E81000CE0185960E9472986AE67EE0E0CF8091F4
:10E820000E0C90910F0C6FE57EE0039711F065E5FB
:10E830007EE0CE0185960E9472986AE47EE0CFCF9A
:10E840006DE37EE0CE0185960E9472986EE27EE0D6
:10E85000C6CF63E27EE0CE0185960E9472986091F9
:10E86000551170915611CE0107960E949E966BE647
:10E870007AE0CE0101960E945399BE01695F7F4FF5
:10E88000CE0101960E9401986CE37AE00E94EB971A
:10E89000BC01CE0185960E946B98CE0101960E9424
:10E8A000E798CE0107960E94E79866E17EE097CF51
:10E8B00080910E0C90910F0C65E07EE0029711F0B4
:10E8C00065EF7DE0CE0185960E94729868EE7DE04E
:10E8D00086CF6CED7DE0CE0185960E9472986CEC3F
:10E8E0007DE07DCF61EC7DE0CE0185960E9472983F
:10E8F00067EB7DE074CF6BEA7DE0CE0185960E94E8
:10E9000072986BE97DE06BCFB090571160E97DE0C4
:10E91000CE0185960E94729883E08B1524F192E0D7
:10E92000B9160CF073C0BB2031F181E0B81609F4C0
:10E9300064C060915711062E000C770BCE0107962C
:10E940000E949E966FE279E0CE0101960E94539953
:10E95000BE01695F7F4FCE0101960E940198BC0104
:10E9600085EC92E13FC094E0B912E3CF6DEF7AE01D
:10E9700085EC92E146C08090581190905911A0907A
:10E980005A11B0905B1120E030E048E452E4C50138
:10E99000B4010E941EB687FF02C033243394A50140
:10E9A000940160E070E080EA90E40E949DB8AB01C1
:10E9B000BC01232DCE0107960E94EF9863ED7AE00B
:10E9C000CE0101960E945399BE01695F7F4FCE012F
:10E9D00001960E94019862E07BE00E94EB97BC01E7
:10E9E000CE0185960E946B98CE0101960E94E79811
:10E9F000CE0107960E94E79806C069EF7AE0CE0143
:10EA000085960E94619860E87DE0E9CE8B2D9AE0C2
:10EA10008902B0011124CE0107960E949E966BE6F2
:10EA20007AE0CE0101960E945399BE01695F7F4F43
:10EA3000CE0101960E9401986BEF7AE0CECF63E79A
:10EA40007DE0CE0185960E94729863E67DE0C7CE98
:10EA500067E57DE0CE0185960E94729868E47DE0CE
:10EA6000BECE6CE37DE0CE0185960E9472986CE28A
:10EA70007DE0B5CE6EED7BE083EE92E10E9467967D
:10EA8000CE0101960E94EE6DBE016F5F7F4F83EE57
:10EA900092E10E94AE98CE0101960E94E798809183
:10EAA000E7129091E812892B89F461E070E0CE01C1
:10EAB00001960E943971BE016F5F7F4F83EE92E134
:10EAC0000E94AE98CE0101960E94E7988091E712CD
:10EAD0009091E812892B89F461E070E0CE010196F3
:10EAE0000E94D16FBE016F5F7F4F83EE92E10E9463
:10EAF000AE98CE0101960E94E7988091E71290911E
:10EB0000E812892B51F48091F60B882331F00F5FC6
:10EB10001F4F0131110509F0CBCCCE018B960E941D
:10EB2000E798CE0185960E94E79891CC1092F60B5B
:10EB3000F4CF2F923F924F925F926F927F928F927B
:10EB40009F92AF92BF92CF92DF92EF92FF920F937C
:10EB50001F93CF93DF93CDB7DEB7C554D1090FB65E
:10EB6000F894DEBF0FBECDBF8C01E0900C0CF0908E
:10EB70000D0C80910E0D882349F062E171E18DEA60
:10EB80009FE00E94BE9BC8010E94899BC801059618
:10EB9000059710F40C94BE8880910C0C90910D0C8C
:10EBA00080179107E1F00E9415590E94D4150C3E80
:10EBB0002FEF120724F010930D0C00930C0CB801EA
:10EBC000CE0101960E949E96BE016F5F7F4F81ED40
:10EBD00092E10E94AE98CE0101960E94E7986EEDF8
:10EBE0007BE085EC92E10E94679662E67AE0CE01D6
:10EBF00001960E9453994AE050E06FEF7FEFCE01FB
:10EC000001960E94335ACE0101960E94E798F801BE
:10EC10007C96E632F10510F00C949F888827EC5E14
:10EC2000F9488F4F0C9449BBAF879F880488FC87B5
:10EC3000CF87B9879F88B4879F889F889F889F8840
:10EC40009F885676C1764777CF78D678AA7A5D7B4B
:10EC5000857C5C7E597FAE7FC37FC67F9F8807809F
:10EC60000A80B68173838F83AD841985E5856786B5
:10EC70006F866E870E94E415CB5BDF4F0FB6F8946A
:10EC8000DEBF0FBECDBFDF91CF911F910F91FF90DF
:10EC9000EF90DF90CF90BF90AF909F908F907F903C
:10ECA0006F905F904F903F902F9008950E9415595C
:10ECB00089E390E00E94195620E030E04AE754E4EE
:10ECC0000E9484B6AB01BC0121E0CE0101960E94F6
:10ECD000EF986BEB78E0CE0180960E945399BE01CD
:10ECE0006F5F7F4FCE0180960E94019865E07BE0C8
:10ECF0000E94EB97BC0185EC92E10E949798CE01AF
:10ED000080960E94E798CE0101960E94E79869E0FC
:10ED10007BE08FEB92E10E9467966FEB72E1CE0190
:10ED200001960E944A994AE050E068E070E0CE0106
:10ED300001960E94DD5ACE0101960E94E79865EC8B
:10ED400072E1CE0101960E944A994AE050E06FEFCD
:10ED50007FEFCE0101960E945759CE0101960E9485
:10ED6000E7986FEB72E185EC92E10E946B988091DD
:10ED70000D0D882309F4C8C164E670E080E090E0DE
:10ED80007DC4C0900402D09005020E94155989E309
:10ED900090E00E94195620E030E04AE754E40E94D7
:10EDA00084B60E9449B9CE0101960E949E966BEBF3
:10EDB00078E0CE0180960E945399BE016F5F7F4F2D
:10EDC000CE0180960E94019865E07BE00E94EB975F
:10EDD000BC0185EC92E10E949798CE0180960E943A
:10EDE000E798CE0101960E94E7988091C912909110
:10EDF000CA12A3E0FA2E099710F0F2E0FF2E8091DC
:10EE0000541140E050E0BA018330DCF4C6010E94A6
:10EE100035174B015C016091551170915611072E09
:10EE2000000C880B990B0E9425B6A50194010E9445
:10EE300084B620E030EC4FE754E40E949DB8AB016B
:10EE4000BC012F2DCE0101960E94EF9867E37BE075
:10EE5000CE0180960E945399BE016F5F7F4FCE0115
:10EE600080960E9401986BE176E00E94EB97BC01CE
:10EE700085EC92E10E946B98CE0180960E94E79803
:10EE8000CE0101960E94E79861E17BE042CF80913C
:10EE90000D0D882309F478C183E79EE00E94FF8E60
:10EEA00062E370E080E090E00E943AA161E080912E
:10EEB00092040E94899D60E0809190040E94899D47
:10EEC00064E670E080E090E00E943AA160918C04DA
:10EED00070918D0480918E0490918F040E9463152F
:10EEE0000E948015AB01BC0123E0CE0180960E94F8
:10EEF000EF98BE01605E7F4FCE0101960E944A9955
:10EF000064E37BE0CE0101960E94EB97BC018FEB9E
:10EF100092E10E949798CE0101960E94E798CE0157
:10EF200080960E94E7986FEC76E0CE0101960E94F1
:10EF300053996FEB72E1CE0101960E940198BC01DA
:10EF400085EC92E10E949798CE0101960E94E79885
:10EF50000E9480156B017C010E94E89D4B015C01C1
:10EF60008BE19EE40197F1F70E9480152B013C0193
:10EF70000E94E89D9B01AC01281939094A095B09E7
:10EF800049015A0131ED831637E09306A104B1041B
:10EF9000CCF0A7019601C301B2010E94BEB76B017C
:10EFA0007C0120E030E0A9010E94A6B9181674F493
:10EFB00026EA3BE944EC5BE3C701B6010E941EB6BA
:10EFC00087FF0EC040E050E0BA0126C026EA3BE9C8
:10EFD00044EC5BEBC701B6010E94A6B9181694F386
:10EFE000C501B40128EE33E040E050E00E945BB779
:10EFF000CA01B9010E9425B64B015C0120E030E056
:10F000004AE754E4C701B6010E9484B6A501940101
:10F010000E949DB8AB01BC0122E0CE0180960E9407
:10F02000EF98BE01605E7F4FCE0101960E944A9923
:10F0300062ED76E0CE0101960E94EB97BC0189EB70
:10F0400092E10E949798CE0101960E94E798CE0126
:10F0500080960E94E7986AE17BE0CE0101960E94CB
:10F06000539969EB72E1CE0101960E940198BC01AF
:10F0700085EC92E10E946B98CE0101960E94E79880
:10F0800062E67AE0CE0101960E94539969EB72E143
:10F09000CE0101960E940198BC018FEB92E10E9483
:10F0A0006B98CE0101960E94E7986EEF7EE0CE014C
:10F0B00001960E9441994AE050E070E060E0CE0184
:10F0C00001960E94DD5ACE0101960E94E7986FEBEF
:10F0D00072E1CE0101960E944A9945E050E06FEF3F
:10F0E0007FEFCE0101960E945759CE0101960E94F2
:10F0F000E7986EE17BE085EC92E10E94619860E028
:10F10000809192040E94899D8091C9129091CA12A7
:10F11000009799F14197A8F40230110594F065EC3D
:10F1200072E1CE0101960E944A994AE050E06FEFE9
:10F130007FEFCE0101960E945759CE0101960E94A1
:10F14000E79865EC72E1CE0101960E944A99CE01E2
:10F1500001960E94E158CE0101960E94E79865EC65
:10F1600072E1CE0101960E944A99CE0101960E9459
:10F170006D18CE0101960E94E79864E670E080E089
:10F1800090E00E943AA178CD609181047091820450
:10F1900080918304909184040E946A2DB5CF809160
:10F1A0007B0490917C040E94852FAECF40917D041A
:10F1B00026964FAF269760E0842F0E94899D80910C
:10F1C0000D0D811109C08091BA11EFE0CE2ED12C26
:10F1D000E12CF12C882329F073E0C72ED12CE12CEF
:10F1E000F12C6DE07FE085EC92E10E94729865EC75
:10F1F00072E1CE0101960E944A994AE050E06FEF19
:10F200007FEFCE0101960E94DD5ACE0101960E9449
:10F21000E798312C212C21961FAE219725961FAE01
:10F2200025971CAE1DAE1EAE1FAE62E3662E712C7E
:10F23000812C912C540126968FAD26970E94C59D56
:10F24000092E000CAA0BBB0B880E991EAA1EBB1E12
:10F2500065E070E080E090E00E943AA151E0651A1C
:10F26000710849F74090D8045090D9046090DA04AE
:10F270007090DB04C501B4010E9425B620E030E0A7
:10F2800040EA50E40E9484B620E030E040E85AE3CF
:10F290000E9484B620E030E048E452E40E949DB829
:10F2A000A30192010E94BEB720E030E040E751E4A4
:10F2B0000E9484B64B015C01A30192016AE979E9DD
:10F2C00089E390E40E94BEB79B01AC01C501B40183
:10F2D0000E949DB820E030E0A9010E94BFB720E065
:10F2E00030E040E251E40E9484B64B015C01232DE2
:10F2F000322D21964FAD219725965FAD25970E941F
:10F30000A6B9181644F4382C292C2196AFAE2197B3
:10F310002596BFAE259720E030E0A901B401C501D4
:10F320000E941EB687FF04C0812C912CA12CB12C09
:10F3300022E0A401B501CE0180960E94EF98BE01A3
:10F34000605E7F4FCE0101960E944A9961E37BE0A7
:10F35000CE0101960E94EB97BC018FEB92E10E94D7
:10F360009798CE0101960E94E798CE0180960E9460
:10F37000E7986FEB72E1CE0101960E944A994AE04C
:10F3800050E070E060E0CE0101960E945759CE0136
:10F3900001960E94E7980E94D6A7AB01BC0180911C
:10F3A000C10C9091C20CA091C30CB091C40C8C59AB
:10F3B0009F4FAF4FBF4F84179507A607B70708F0B9
:10F3C000AAC00E9496566CE370E080E090E00E9434
:10F3D0003AA18CAD9DADAEADBFAD0196A11DB11DE5
:10F3E0008CAF9DAFAEAFBFAFC816D906EA06FB061D
:10F3F0000CF01BCF64E670E080E090E00E943AA140
:10F400000E94155964E670E080E090E00E943AA105
:10F4100065E07FE08FEB92E10E9472986FEB72E102
:10F42000CE0101960E944A9944E150E070E060E00C
:10F43000CE0101960E94DD5ACE0101960E94E79806
:10F4400022E0432D522D21966FAD219725967FAD59
:10F450002597CE0180960E94EF98BE01605E7F4F97
:10F46000CE0101960E944A9961E37BE0CE010196AC
:10F470000E94EB97BC018FEB92E10E949798CE011E
:10F4800001960E94E798CE0180960E94E7986FEB64
:10F4900072E1CE0101960E944A9942E350E06FEF7B
:10F4A0007FEFCE0101960E945759CE0101960E942E
:10F4B000E79864E170E080E090E00E943AA10E9449
:10F4C00096566EE170E080E090E00E943AA16EE115
:10F4D00070E080E090E00E943AA166E37BE0CE011C
:10F4E00001960E9453996FEB72E1CE0101960E9442
:10F4F00001986AE37BE00E94EB9765EC72E10E9461
:10F500000198BC0185EC92E10E949798CE0101968A
:10F510000E94E798F9CD0E94D6A70E9423B64B011E
:10F520005C016091C10C7091C20C8091C30C9091F0
:10F53000C40C0E9425B620E030E048EC51E40E9463
:10F54000BFB79B01AC01C501B4010E941EB687FD87
:10F5500038CF39CF80917F049091800499270E9401
:10F5600035172DE038E643E55BE30E9484B66B0176
:10F570007C012091070530910805409109055091C3
:10F580000A050E941EB618160CF47BC06091EF04A9
:10F590007091F0048091F1049091F20420E030E049
:10F5A00048EC52E40E9484B620E030E048EA51E49E
:10F5B0000E9484B62091DC043091DD044091DE0489
:10F5C0005091DF040E949DB86B017C016AE17FE0ED
:10F5D0008FEB92E10E9472986FEB72E1CE0101967F
:10F5E0000E944A9942E350E070E060E0CE0101964B
:10F5F0000E94DD5ACE0101960E94E79822E0B701F1
:10F60000A601CE0101960E94EF9864E47BE0CE0152
:10F6100080960E945399BE016F5F7F4FCE01809606
:10F620000E9401986EE37BE00E94EB97BC0185ECA1
:10F6300092E10E949798CE0180960E94E798CE01B1
:10F6400001960E94E79865EC72E1CE0101960E9456
:10F650004A9942E350E06FEF7FEFCE0101960E949E
:10F660005759CE0101960E94E79880910D0D88238D
:10F6700009F44ACD60E273E080E090E00E943AA194
:10F6800043CD20911B0530911C0540911D055091E3
:10F690001E05C701B6010E94A6B987FF05C0C701B4
:10F6A000B6010E94888D7ACF6091030570910405A0
:10F6B000809105059091060571CF0E9415596EE461
:10F6C0007FE085EC92E10E94729865EC72E1CE01D8
:10F6D00001960E944A994AE050E070E060E0CE0155
:10F6E00001960E94DD5ACE0101960E94E79865E4DA
:10F6F0007FE08FEB92E10E9472986FEB72E1CE0196
:10F7000001960E944A9944E150E06FEF7FEFCE01ED
:10F7100001960E945759CE0101960E94E798809168
:10F72000C50C9091C60C8230910509F041C00E9431
:10F73000A9A6811104C01092C60C1092C50C80912C
:10F74000C50C9091C60C029709F448C069E37FE0AC
:10F7500085EC92E10E94729865EC72E1CE0101960F
:10F760000E944A994AE050E070E060E0CE010196C4
:10F770000E94DD5ACE0101960E94E79865EC72E185
:10F78000CE0101960E944A9962E67AE0CE01019686
:10F790000E94EB976FEB72E10E940198BC0185EC2F
:10F7A00092E10E949798CE0101960E94E7985DCF62
:10F7B000892B61F60E94A9A6882339F082E090E0A7
:10F7C0009093C60C8093C50CBACF0E94A9A6811154
:10F7D000F5CF0E94A9A68111F1CFB1CF8AE090E0C8
:10F7E0000E9410166B017C0120E030E0A9010E940C
:10F7F0001EB6181634F08AE090E00E9410166B01D5
:10F800007C015BE0A52EB12C20E030E042ED53E41A
:10F81000C701B6010E941EB618168CF091E0A91A15
:10F82000B10869F068EC70E080E090E00E943AA1D5
:10F8300083E090E00E9410166B017C01E5CF20E090
:10F8400030E0A901C701B6010E941EB618166CF17E
:10F850006BE27FE085EC92E10E94729865EC72E1C8
:10F86000CE0101960E944A9942E350E06FEF7FEF8C
:10F87000CE0101960E945759CE0101960E94E79849
:10F8800062E27FE08FEB92E10E9472986FEB72E18F
:10F89000CE0101960E944A9942E350E070E060E098
:10F8A000CE0101960E94DD5ADCCE20E030E048EC2B
:10F8B00052E4C701B6010E941EB621E087FF20E096
:10F8C000B701A601CE0101960E94EF9863E47BE0A8
:10F8D000CE0180960E945399BE016F5F7F4FCE018B
:10F8E00080960E94019868E47BE00E94EB97BC013F
:10F8F00085EC92E10E949798CE0180960E94E7984D
:10F90000CE0101960E94E798A9CF0E94D6A72B01AD
:10F910003C0183E79EE00E94FF8E64E670E080E099
:10F9200090E00E943AA140E855E260E070E083E791
:10F930009EE00E94E35964E670E080E090E00E945F
:10F940003AA167E87FE08FEB92E10E9472986FEB3B
:10F9500072E1CE0101960E944A9942E350E06FEFB6
:10F960007FEFCE0101960E94DD5ACE0101960E94E2
:10F97000E7986CE77FE08FEB92E10E9472986FEB63
:10F9800072E1CE0101960E944A9942E350E06FEF86
:10F990007FEFCE0101960E945759CE0101960E9439
:10F9A000E79880910E0C90910F0C8D7F1CAEB12CBE
:10F9B000A12CD12CC12CF12CE12C019709F47AC097
:10F9C000DE019096B9AFA8AFFE017E96FBAFEAAF1D
:10F9D0000E94D6A76419750986099709683B7B4080
:10F9E0008105910508F066C083E79EE00E94678963
:10F9F000892B09F44EC02CED35E040E050E0209317
:10FA0000770E3093780E4093790E50937A0E0E94C1
:10FA1000E2A797FD3EC082349105C9F7AE014F5F62
:10FA20005F4F1A014A010E94E2A797FF39C08981FE
:10FA30008D3479F590E080E0D1012D911D01820F88
:10FA4000911DEAADFBADEA17FB07B1F78E5B9F4F47
:10FA50002E8D30E0322F22274F8D240F311D82173B
:10FA60009307B9F4EC80F12CFE2CEE248D81E80E86
:10FA7000F11CCE80D12CDC2CCC248F81C80ED11C63
:10FA8000A884B12CBA2CAA248985A80EB11CF1E057
:10FA9000FCAF62E370E080E090E00E943AA198CF72
:10FAA000D4018D934D01E8ADF9ADEA17FB0709F0DC
:10FAB000BACFBDCF0E94D6A76419750986099709E8
:10FAC000683B7B408105910518F43CAD3111BCC009
:10FAD0000E9415596FEB72E1CE0180960E944A99FF
:10FAE00042E350E066E070E0CE0180960E94DD5A6D
:10FAF000CE0180960E94E7984CAD442309F4B3C030
:10FB000082E090E090930F0C80930E0CB501CE0133
:10FB100080960E949E96B601CE0186960E949E9681
:10FB2000B701CE01C2960E949E96BE016E5C7F4FC9
:10FB3000CE018C960E944A996FEA78E0CE018C96AD
:10FB40000E94EB97BE016A5D7F4F0E9401986FEAA9
:10FB500078E00E94EB97BE01605E7F4F0E940198A3
:10FB6000BC0185EC92E10E949798CE018C960E9490
:10FB7000E798CE01C2960E94E798CE0186960E9431
:10FB8000E798CE0180960E94E79865EC72E1CE017D
:10FB900080960E944A994AE050E06FEF7FEFCE01D5
:10FBA00080960E945759CE0180960E94E79866E79A
:10FBB0007FE08CEC93E10E94BE9BB501CE01809664
:10FBC0000E949E96B601CE0186960E949E96B7012F
:10FBD000CE018C960E949E966CE47BE0CE01C2968C
:10FBE0000E945399BE01645D7F4FCE01C2960E9470
:10FBF000019862E67AE00E94EB97BE016A5D7F4F52
:10FC00000E94019862E67AE00E94EB97BE01605E76
:10FC10007F4F0E9401986CE57BE00E94EB97BC014E
:10FC200085EC92E10E949798CE01C2960E94E798D7
:10FC3000CE018C960E94E798CE0186960E94E798A6
:10FC4000CE0180960E94E79862E370E080E090E049
:10FC50000E943AA183E79EE00E94FF8E62E370E07B
:10FC600080E090E00BCD6BE67FE085EC92E10E94B6
:10FC7000729865EC72E1CE0180960E944A994AE042
:10FC800050E070E060E0CE0180960E945759CE01AE
:10FC900080960E94E79868E57FE085EC92E10E94FB
:10FCA000729880910E0C90910F0C029769F6109249
:10FCB0000F0C10920E0CC8CFE0907904F0907A04EB
:10FCC00062E67BE08FEB92E10E9467960E941559F5
:10FCD0006FEB72E1CE0101960E944A994AE050E032
:10FCE0006FEF7FEFCE0101960E94DD5ACE010196A3
:10FCF0000E94E798C7010E94461824966CAF7DAF1A
:10FD00008EAF9FAF24978090B5049090B604A090DA
:10FD1000B704B090B804A50194016091B10470914A
:10FD2000B2048091B3049091B4040E94BEB72B0139
:10FD30003C0120E030E0A9010E941EB6882309F4AE
:10FD40008EC0C090BD04D090BE04E090BF04F0907F
:10FD5000C00420E030E0A901C701B6010E941EB630
:10FD600018160CF07CC08091B9049091BA04A0914F
:10FD7000BB04B091BC048CAF9DAFAEAFBFAF9C01D4
:10FD8000AD01C701B6010E941EB6882309F467C001
:10FD9000A70196016CAD7DAD8EAD9FAD0E949DB863
:10FDA0000E94F5B96CAF7DAF8EAF9FAFA5019401F6
:10FDB00024966CAD7DAD8EAD9FAD24970E94BEB7ED
:10FDC000A30192010E949DB82CAD3DAD4EAD5FAD3B
:10FDD0000E9484B60E9417B99B01AC01C701B6010D
:10FDE0000E9484B66B017C016FEB72E1CE0101963B
:10FDF0000E944A994AE050E070E060E0CE0101962E
:10FE00000E94DD5ACE0101960E94E79820E030E67C
:10FE10004AEE56E4C701B6010E94A6B918161CF5B1
:10FE200063E97FE085EC92E10E94729865EC72E1F3
:10FE3000CE0101960E944A994AE050E06FEF7FEFB1
:10FE4000CE0101960E945759CE0101960E94E79873
:10FE500064E670E080E090E00E943AA106CCC12CFC
:10FE6000D12C7601C1CF21E0B701A601CE01809649
:10FE70000E94EF986CE67BE0CE0101960E945399B8
:10FE8000BE01605E7F4FCE0101960E94019860E73F
:10FE90007BE00E94EB97BC0185EC92E10E94979871
:10FEA000CE0101960E94E798CE0180960E94E798C5
:10FEB000BDCFE0900402F09005020E94155965E064
:10FEC00070E080E090E00E943AA18091541140E0FF
:10FED00050E0BA018330DCF4C7010E9435176B0192
:10FEE0007C016091551170915611072E000C880B02
:10FEF000990B0E9425B6A70196010E9484B620E0C6
:10FF000030EC4FE754E40E949DB8AB01BC0123E004
:10FF1000CE0101960E94EF9867E37BE0CE018096C8
:10FF20000E945399BE016F5F7F4FCE0180960E9461
:10FF300001986BE176E00E94EB97BC0185EC92E1C1
:10FF40000E949798CE0180960E94E798CE01019674
:10FF50000E94E79864E77BE00C9489768091E10C3D
:10FF600091E089278093E10C80910D0D882331F079
:10FF700065EC72E186ED9DE00E94AC9B68EC70E060
:10FF800080E090E07BCB10920D0DBEC881E08093A5
:10FF90000D0D8093C8118091BF11882349F16CE841
:10FFA00078E081ED92E10E94679686EE9FEF909354
:10FFB0000D0C80930C0C2091C2113091C3118091D3
:10FFC000C4119091C5118217930724F01092C511A6
:10FFD0001092C4111092B6111092B7111092B8116C
:10FFE0001092B9116CE271E080E090E00E943AA1B9
:10FFF00061ED72E187ED92E10E94979880910C0C7F
:020000021000EC
:1000000090910D0C9093040D8093030D7DC80E9478
:1000100008727AC880E19FE00E94FF8E40E052ECB7
:1000200061E070E080E19FE00E94E3598CED95E093
:10003000A0E0B0E08093140F9093150FA093160FDB
:10004000B093170F64E670E080E090E00E943AA160
:100050008091C50C9091C60C019779F583E090E0F2
:100060000E94AA17811104C01092C60C1092C50CF0
:100070008091C50C9091C60C0197C9F162ED7FE0AB
:100080008FEB92E10E9472986FEB72E1CE010196C4
:100090000E944A9944E150E06FEF7FEFCE01019654
:1000A0000E945759CE0101960E94E79866EC7FE0C6
:1000B00085EC92E10E94729826C181E090E00E9456
:1000C000AA17882339F081E090E09093C60C8093C2
:1000D000C50CCECF83E090E00E94AA178111F3CF28
:1000E00083E090E00E94AA178111EDCFC1CF6AEBA7
:1000F0007FE085EC92E10E94729865EC72E1CE019E
:1001000001960E944A99CE0101960E94DF5CCE01C1
:1001100001960E94E79862E370E080E090E00E9420
:100120003AA165EC72E1CE0101960E944A9942E340
:1001300050E06FEF7FEFCE0101960E94DD5ACE01B5
:1001400001960E94E7986EEA7FE08FEB92E10E94B1
:1001500072986FEB72E1CE0101960E944A9944E1D8
:1001600050E06FEF7FEFCE0101960E945759CE010C
:1001700001960E94E7988BEB88A38AEA89A381E025
:100180008AA368011801412C512C3201C6016AE092
:1001900070E00E9435BB892B49F443E050E0BE017A
:1001A000605E7F4F80E19FE00E94F08865E070E034
:1001B00080E090E00E943AA1BFEFCB1ADB0A780101
:1001C000812C912C540180E19FE00E946789892B4A
:1001D00039F4E4E08E169104A104B1040CF049C096
:1001E000F6E0EF16F1040CF044C080E19FE00E94BD
:1001F0006789892B71F080E19FE00E944589E1E0E9
:10020000F0E0EC0FFD1FEE0DFF1D80832FEFE21AD3
:10021000F20A65E070E080E090E00E943AA136E0EA
:10022000E316F10401F5998188A198131CC09A8105
:1002300089A1981318C09B818AA1981314C08D813D
:1002400090E0B0E0A0E0BA2FA92F982F88272C814A
:10025000820F911DA11DB11D480E591E6A1E7B1EE5
:100260004FEF241A340A5FEF851A950AA50AB50ADA
:10027000AACF94E02916310434F4A0E9CA16A1E00B
:10028000DA0609F083CFC301B2010E9425B620E04F
:1002900030E040E251E40E949DB820E030E040E8C8
:1002A0005EE30E9484B66B017C0120E030E040EA0E
:1002B00051E40E94A6B918160CF055C021E0B70110
:1002C000A601CE0101960E94EF986EEF77E0CE0175
:1002D00080960E945399BE016F5F7F4FCE0180963A
:1002E0000E9401986CE77BE00E94EB97BC0185ECD3
:1002F00092E10E949798CE0180960E94E798CE01E5
:1003000001960E94E79865EC72E1CE0101960E9489
:100310004A994AE050E070E060E0CE0101960E9408
:10032000DD5ACE0101960E94E79865EC72E1CE019C
:1003300001960E944A9962E67AE0CE0101960E94F7
:10034000EB976FEB72E10E940198BC0185EC92E1A2
:100350000E949798CE0101960E94E79880E19FE065
:100360000E94FF8E82C962EA7FE0A2CE6DE670E154
:10037000CE0101960E9441994AE050E06FEF7FEF75
:10038000CE0101960E945759CE0101960E94E7982E
:1003900060918A0470918B048091D6049091D70467
:1003A0000E94A45674E1872E912CA12CB12CD12C43
:1003B000C12CAFEFCA1ADA0AC501B4010E943AA1F2
:1003C00060918A0470918B048091D6049091D70437
:1003D0000E94A4567C01B3E0CB16D10434F08EE128
:1003E000C816D10444F4EF2851F094E1890E911C11
:1003F000A11CB11CDECFE114F10409F00CC1809105
:10040000D6049091D7048B30910509F0DFC080911C
:10041000231390912413A0912513B0912613809358
:10042000080C9093090CA0930A0CB0930B0C8091CC
:100430001F1390912013A0912113B0912213809348
:10044000040C9093050CA093060CB093070C4091FC
:10045000080C5091090C60910A0C70910B0C21E072
:10046000CE0101960E94EF9868EF76E0CE0180966B
:100470000E945399BE016F5F7F4FCE0180960E940C
:100480000198BC0185EC92E10E949798CE0180967C
:100490000E94E798CE0101960E94E7984091040CD3
:1004A0005091050C6091060C7091070C21E0CE0173
:1004B00001960E94EF9867EB77E0CE0180960E944C
:1004C0005399BE016F5F7F4FCE0180960E940198C5
:1004D000BC0185EC92E10E946B98CE0180960E944F
:1004E000E798CE0101960E94E79861E47BE085ECF5
:1004F00092E10E9461986EED7BE0CE0101960E9430
:10050000539944E150E070E060E0CE0101960E9412
:10051000DD5ACE0101960E94E798C090080CD09059
:10052000090CE0900A0CF0900B0C20E030E0A901DF
:10053000C701B6010E94A6B920E030E040E05FE3C9
:1005400087FD64C0C701B6010E94BFB70E9449B9C8
:10055000AB01BC01CE0101960E947196BE016F5F96
:100560007F4F8FEB92E10E94AE98CE0101960E94E0
:10057000E79860E087E00E94318C6FEB72E18CECD1
:1005800093E10E949E9B6FED8CEC93E10E94239A75
:100590006DEB77E08CEC93E10E949C9B6091040CE6
:1005A0007091050C8091060C9091070C0E9449B93E
:1005B0004AE050E08CEC93E10E944F9B61E47BE0C9
:1005C0008CEC93E10E949C9B0C94BC768631910547
:1005D00009F41DCF0C9709F03ACF8091FB0B909155
:1005E000FC0BA091FD0BB091FE0B8093080C909337
:1005F000090CA0930A0CB0930B0C8091F70B90910F
:10060000F80BA091F90BB091FA0B19CFC701B60105
:100610000E94BEB79BCFEFEFEE16FE06D4F06FE55B
:1006200070E1CE0101960E9441994AE050E070E0ED
:1006300060E0CE0101960E94DD5ACE0101960E9433
:10064000E7986CE370E185EC92E10E9472980C945B
:100650008478FEEFEF16FFEFFF0681F16EE270E1A6
:10066000CE0101960E9441994AE050E070E060E0BE
:10067000CE0101960E94DD5ACE0101960E94E798B4
:100680006FE170E185EC92E10E947298B701CE01B2
:1006900001960E949E96BE016F5F7F4F85EC92E1AE
:1006A0000E946B98CE0101960E94E79869E070E184
:1006B00085EC92E10E9414980C9484786EEF7FE0B0
:1006C000CE0101960E9441994AE050E070E060E05E
:1006D000CE0101960E94DD5ACE0101960E94E79854
:1006E0006EED7FE0B0CF80919404882311F40C94D8
:1006F00084786EED7BE0CE0101960E9453994AE02A
:1007000050E061E070E0CE0101960E94DD5ACE011A
:1007100001960E94E7980E94AD630C9484788091C2
:100720000D0D811109C08091BA116EE1462E512C38
:10073000612C712C882329F053E0452E512C612C1B
:10074000712C6BE770E185EC92E10E94729865EC88
:1007500072E1CE0101960E944A994AE050E06FEFA3
:100760007FEFCE0101960E945759CE0101960E945B
:10077000E798812C912C54011CAE1DAE1EAE1FAE0D
:1007800083E20E94168C87E090E00E94118C0E9408
:10079000FD9E66E970E080E090E00E943AA183E26D
:1007A0000E94168C80E290E00E94118C0E94FD9EB7
:1007B00066E970E080E090E00E943AA162E070E0BB
:1007C00083E290E00E94E49FC12CD12C76018091BD
:1007D000330D9091340D891B990B181619065CF492
:1007E0000E941D8FFE2CED2CDC2CCC24C80ED11CBD
:1007F000E11CF11CECCFC701B6010E9425B62AE925
:1008000039E949E95FE30E949DB80E9449B9AB010B
:10081000BC0184169506A606B70614F44A015C01CD
:10082000CE0180960E947196BE01605E7F4FCE0120
:1008300001960E944A996FE77BE0CE0101960E94E3
:10084000EB97BC018FEB92E10E949798CE01019645
:100850000E94E798CE0180960E94E7986FEB72E1C4
:10086000CE0101960E944A994EE150E070E060E0AE
:10087000CE0101960E94335ACE0101960E94E7985C
:100880002CAD3DAD4EAD5FAD2F5F3F4F4F4F5F4F36
:100890002CAF3DAF4EAF5FAF4216530664067506F0
:1008A0000CF06ECFB501A401CE0180960E94719626
:1008B000BE01605E7F4FCE0101960E944A996FE7AC
:1008C0007BE0CE0101960E94EB97BC018FEB92E199
:1008D0000E949798CE0101960E94E798CE018096DB
:1008E0000E94E7986FEB72E1CE0101960E944A994F
:1008F0004AE050E070E060E0CE0101960E94DD5ACF
:10090000CE0101960E94E798B501A401CE0101969F
:100910000E9471966CE876E0CE0180960E94539911
:10092000BE016F5F7F4FCE0180960E94019863E801
:100930007BE00E94EB9765EC72E10E940198BC019C
:1009400085EC92E10E949798CE0180960E94E798EC
:10095000CE0101960E94E79881C9E0900202F090D2
:10096000030281E08093E80464E670E080E090E0B8
:100970000E943AA10E941559C7010E9435170E9492
:1009800049B920E034E0A901461B570BBA01CE015A
:1009900001960E949E9668E87BE0CE0180960E94B8
:1009A0005399BE016F5F7F4FCE0180960E940198E0
:1009B000BC0185EC92E10E949798CE0180960E943E
:1009C000E798CE0101960E94E79860E087E00E94D8
:1009D000318C6BE870E1CE0101960E94419942E3AF
:1009E00050E068E070E0CE0101960E94DD5ACE0131
:1009F00001960E94E79865EC72E1CE0101960E9493
:100A00004A9942E350E06FEF7FEFCE0101960E94DA
:100A10005759CE0101960E94E7986FE87BE0CE011E
:100A200001960E94539965EC72E1CE0101960C94F7
:100A3000CC7B80910002909101020E9435170E94A8
:100A400049B97093C80C6093C70C62E370E080E012
:100A500090E00E943AA16091C70C7091C80CCE0141
:100A600001960E949E96BE016F5F7F4F85EC92E1DA
:100A70000E94AE98CE0101960E94E79880911D13C6
:100A800090911E13892B09F45EC069E173E1CE01D8
:100A900080960E944A99BE01605E7F4FCE0101960A
:100AA0000E944A9944E150E070E060E0CE01019676
:100AB0000E94DD5ACE0101960E94E79869E97BE029
:100AC000CE0101960E94539965EC72E1CE01019628
:100AD0000E940198BC018FEB92E10E949798CE0191
:100AE00001960E94E7986FEB72E1CE0101960E9499
:100AF0004A9944E150E06FEF7FEFCE0101960E94EA
:100B00005759CE0101960E94E798BE01605E7F4F63
:100B1000CE0101960E944A9962E67AE0CE010196E2
:100B20000E94EB976FEB72E10E940198BC0185EC8B
:100B300092E10E949798CE0101960E94E798CE011B
:100B400080960C94337B64EA7BE08FEB92E10E9409
:100B500067966FEB72E1CE0101960E944A9944E1DB
:100B600050E070E060E0CE0101960E94DD5ACE01B7
:100B700001960E94E79868E87BE0CE0101960E940A
:100B8000539965EC72E1CE0101960E940198BC0177
:100B90008FEB92E10E949798CE0101960E94E79810
:100BA0006FEB72E1CE0101960E944A9944E150E058
:100BB0006FEF7FEFCE0101960E945759CE0101964B
:100BC0000E94E79869E97BE02ACF8091940488230A
:100BD00011F40C94847880910D0D811104C08091E2
:100BE000BA11882331F082E090E00E94E2690C940F
:100BF0008478C0908104D0908204E0908304F090C7
:100C0000840420E030E040E450E4C701B6010E94D3
:100C1000A6B918160CF054C020E030E04AEF54E4B6
:100C2000C701B6010E9484B60E9449B96B017C01DC
:100C30000E94155960E080E00E94318C6CE970E1FF
:100C40008CEC93E10E94BE9B61E080E00E94318CBD
:100C500064E970E18CEC93E10E94BE9B64E670E075
:100C600080E090E00E943AA10E94D6A76093C90C50
:100C70007093CA0C8093CB0C9093CC0C0E94D6A797
:100C80008090C90C9090CA0CA090CB0CB090CC0C6A
:100C9000681979098A099B096C157D058E059F05E0
:100CA00014F00C94847883E090E00E94E2690E9442
:100CB000D6A764E170E080E090E00E943AA1DECF28
:100CC00030E3C32E35E7D32EE12CF12CB1CF0E94B7
:100CD000661986ED9DE00E940A8A0C9484786CEB7C
:100CE00070E18FEB92E10E9472986FEB72E1CE019E
:100CF00001960E944A994AE050E070E060E0CE011F
:100D000001960E94DD5ACE0101960E94E79830902C
:100D100006028091D90C811105C00E94D6A781E0FE
:100D20008093D90C8091D10C811105C00E94D6A767
:100D300081E08093D10C1092F50B1092F40BE090AF
:100D4000F40BF090F50B58E2E516F1040CF07EC0C0
:100D5000832D0E94C59DF701EE0FFF1FE95CF24F46
:100D6000918380830E945E8C20E030E040EA50E472
:100D70000E9484B620E030E040E85AE30E9484B646
:100D80006B017C014090AD045090AE046090AF04C4
:100D90007090B004A30192016091A9047091AA041B
:100DA0008091AB049091AC040E94BEB79B01AC0152
:100DB00060E070E080EC90E40E94BEB74B015C0103
:100DC00020E030E0A9010E941EB620E030E040E6BD
:100DD00050E481111CC0C701B6010E9484B6609323
:100DE000CD0C7093CE0C8093CF0C9093D00C64E11B
:100DF00070E080E090E00E943AA18091F40B909125
:100E0000F50B01969093F50B8093F40B98CFC701E7
:100E1000B6010E9484B6A30192010E94BFB720E0F0
:100E200030E040E850E40E94BEB7A50194010E9462
:100E30009DB820E030E040EC50E40E9484B620E011
:100E400030E040E850E40E94BFB7C9CFC090CD0C5D
:100E5000D090CE0CE090CF0CF090D00C20E030E0A1
:100E6000A901C701B6010E94A6B987FD22C022E0F0
:100E7000B701A601CE0180960E94EF9868EA7BE058
:100E8000CE0101960E945399BE01605E7F4FCE0154
:100E900001960E940198BC0185EC92E10E9497980E
:100EA000CE0101960E94E798CE0180960E94E798B5
:100EB00006C06DEA70E185EC92E10E94729865ECE3
:100EC00072E1CE0101960E944A994AE050E06FEF2C
:100ED0007FEFCE0101960E9457595BC08091940428
:100EE000882311F40C94847880910D0D81112EC00B
:100EF0008091BA1181112AC0C0908104D0908204DF
:100F0000E0908304F090840420E030E04AE754E469
:100F1000C701B6010E9484B60E9449B94B015C0129
:100F200020E030E040EA50E4C701B6010E9484B6F8
:100F300020E030E040EA50E40E94BFB70E9449B987
:100F4000A50194010E942E650C94847821E030E084
:100F500040E050E06AE070E080E090E0F3CFC7014D
:100F60000E9498520C948478C7010E9480280C94A7
:100F7000847880910E0D882311F40C9484786AE0B3
:100F800071E1CE0101960E944199CE0101960E9425
:100F9000E158CE0101960E94E7980C9484788091E4
:100FA000350D9091360D892B81F481E090E090937E
:100FB000360D8093350D8EE492E00E94338E68ECFE
:100FC00070E080E090E00E943AA16DEF70E1CE0108
:100FD00001960E94419944E650E06FEF7FEFCE0109
:100FE00001960E945759CE0101960E94E798F0E0C1
:100FF000E0E019950C9484780E946CA70E94155922
:101000000E94D4150C9484788091BF1191E08927B7
:101010008093BF11882309F48BC066EF70E185ECE3
:1010200092E10E9472980E94D6A76093B6117093C5
:10103000B7118093B8119093B9118091C21190911A
:10104000C311181619065CF42091C4113091C51112
:101050002817390724F01092C5111092C4119091ED
:10106000C6118091C111981724F01092C6111092E8
:10107000C7118091BF118093BA1165EC72E1CE0166
:1010800001960E944A994AE050E068E070E0CE0183
:1010900001960E94DD5ACE0101960E94E79861EE0A
:1010A00070E1CE0101960E9441994AE050E06FEF55
:1010B0007FEFCE0101960E945759CE0101960E9402
:1010C000E79863ED70E185EC92E10E94149866ED7B
:1010D00075E0CE0101960E94539965EC72E1CE0154
:1010E00001960E940198BC0185EC92E10E949798BC
:1010F000CE0101960E94E79880910D0D8093C81152
:101100008CE291E00E945E8E80910D0D882311F497
:101110000C9484786CE878E081ED92E10E94679607
:1011200086EE9FEF90930D0C80930C0C0C948478BA
:101130006EEE70E185EC92E10E9472989ACFF09287
:101140000D0CE0920C0C86ED9DE00E940A8A65EC85
:1011500070E185EC92E10E9472986EED7BE0CE0129
:1011600001960E9453994AE050E070E060E0CE01A1
:1011700001960E94DD5ACE01019698CE0E3FFFEFF8
:101180001F0711F40C943A766EED7BE085EC92E14A
:101190000E9467960C94077696E0899FD0011124EF
:1011A000AF5BBC4E90967C936E935F9791E0919667
:1011B0009C939197E091AE13F091AF139091AD1382
:1011C000992339F0309751F0811108C080915D1357
:1011D0001994309719F05C968C91FACF0895089580
:1011E000AF92BF92CF92DF92EF92FF920F931F9335
:1011F000CF93DF936C017B018B01040F151FEB0173
:101200005E01AE18BF08C017D10759F06991D60129
:10121000ED91FC910190F081E02DC6011995892B8B
:1012200079F7C501DF91CF911F910F91FF90EF905A
:10123000DF90CF90BF90AF900895FC01A089B18955
:101240008C91A689B78982FD0FC09C91818D8F5F9B
:101250008F73228D821749F0A18DAE0FBF2FB11D64
:101260005D969C93818F08958C910895FC01538D18
:10127000448D252F30E0842F90E0821B930B541770
:1012800010F0CF96089501970895FC01918D828DFD
:10129000981761F0A28DAE0FBF2FB11D5D968C9196
:1012A000928D9F5F9F73928F90E008958FEF9FEFD5
:1012B0000895FC01918D828D981731F0828DE80F91
:1012C000F11D858D90E008958FEF9FEF0895FC014B
:1012D000918D228D892F90E0805C9F4F821B910918
:1012E0008F739927089586ED9DE00E94678921E01C
:1012F000892B09F420E0822F089583E79EE00E9465
:10130000678921E0892B09F420E0822F089580E18C
:101310009FE00E94678921E0892B09F420E0822F59
:1013200008958DEA9FE00E94678921E0892B09F4E6
:1013300020E0822F0895FC01A48DA80FB92FB11DC4
:10134000A35ABF4F2C91848D90E001968F739927FB
:10135000848FA689B7892C93A089B1898C918370D9
:1013600080648C93938D848D981306C00288F389D2
:10137000E02D80818F7D80830895EF92FF920F93FF
:101380001F93CF93DF93EC0181E0888F9B8D8C8D31
:1013900098131AC0E889F989808185FF15C09FB725
:1013A000F894EE89FF896083E889F98980818370E8
:1013B000806480839FBF81E090E0DF91CF911F9197
:1013C0000F91FF90EF900895F62E0B8D10E00F5FB8
:1013D0001F4F0F731127E02E8C8D8E110CC00FB68E
:1013E00007FCFACFE889F989808185FFF5CFCE0126
:1013F0000E949B89F1CFEB8DEC0FFD2FF11DE35A7D
:10140000FF4FF0829FB7F8940B8FEA89FB898081A8
:101410008062CFCFCF93DF93EC01888D8823B9F022
:10142000AA89BB89E889F9898C9185FD03C08081EF
:1014300086FD0DC00FB607FCF7CF8C9185FFF2CF6C
:10144000808185FFEDCFCE010E949B89E9CFDF919E
:10145000CF91089580E090E0892B29F00E94918936
:1014600081110E94000080E090E0892B29F00E9409
:10147000878981110E94000080E090E0892B29F08B
:101480000E947D8981110E94000080E090E0892BFC
:1014900029F00E94738981110C94000008958150F5
:1014A000823108F05AC0E82FF0E08827E55AF54766
:1014B0008F4F0C9449BB7B8A7F8A6D8A738A778AA7
:1014C000AD8A828A888A8C8A928A968A9A8AA08A27
:1014D000A48AAD8AA88AAE8AB28A809180008F776A
:1014E000809380000895809180008F7DF9CF809156
:1014F0008000877FF5CF84B58F7784BD089584B54C
:101500008F7DFBCF8091B0008F778093B0000895DE
:101510008091B0008F7DF9CF809190008F7780937C
:1015200090000895809190008F7DF9CF8091900078
:10153000877FF5CF8091A0008F778093A0000895DA
:101540008091A0008F7DF9CF8091A000877FF5CF9B
:10155000809120018F778093200108958091200150
:101560008F7DF9CF80912001877FF5CF08958F92ED
:101570009F92AF92BF92CF92DF92EF92FF920F9322
:101580001F93CF93DF93DB01ED91FC91EC01AC85D0
:10159000BD8501E010E0EA17FB070CF045C0EF0144
:1015A000CC0FDD1FDC011A968D919C91DC01AC0FF4
:1015B000BD1FAD90BC908F01009510950170112753
:1015C0008CE99FEFE0FF02C084E690E0E9016A0148
:1015D0007B014C01820E931EB401C5010E94601371
:1015E00021E030E0892BB9F48C0E9D1EB401C501B9
:1015F0000E94601322E030E0892B69F4BE01680D7F
:10160000791DC5010E94601323E030E0892B19F495
:101610000FEF1FEF09C0E6018881998101968217BB
:10162000930784F499838883C801DF91CF911F9138
:101630000F91FF90EF90DF90CF90BF90AF909F9071
:101640008F90089519821882D7018D919C911197DE
:1016500001968D939C93E8CFFB0101900020E9F760
:101660003197AF01461B570BDC01ED91FC910280D5
:10167000F381E02D1994CF93DF93EC018881998158
:10168000009711F00E9437BC198218821D821C82BB
:101690001B821A82DF91CF9108950C9437BC0F936F
:1016A0001F93CF93DF93EC0188819981009759F0C4
:1016B0002A813B812617370730F081E0DF91CF91F7
:1016C0001F910F9108958B016F5F7F4F0E94C0BCE7
:1016D000009759F0998388831B830A832C813D816D
:1016E000232B59F7FC011082E8CF80E0E7CFEF927F
:1016F000FF920F931F93CF93DF936115710541F410
:1017000080E0DF91CF911F910F91FF90EF900895AE
:1017100041155105B1F07B01EC010C811D81040FD5
:10172000151FB8010E944F8B882351F328813981FE
:101730008C819D81B701820F931F0E94EBBD1D8399
:101740000C8381E0DECFEF92FF920F931F93CF9334
:10175000DF93EC017B018A01BA010E944F8B81115A
:101760000BC0CE010E943B8BCE01DF91CF911F9128
:101770000F91FF90EF9008951D830C83B70188812E
:1017800099810E94EBBDF0CF0F931F93CF93DF930E
:101790008C01EB0188E2FB0111928A95E9F74BE09D
:1017A00050E06CEA7BE0CE010E9400BE1B8681E027
:1017B00090E0A0E0B0E08C879D87AE87BF87F801FE
:1017C00085899689A789B08D888B998BAA8BBB8BCD
:1017D00082E090E0A0E0B0E08C8B9D8BAE8BBF8B65
:1017E0001CA21DA21EA21FA280E090E0A8E4B4E407
:1017F000888F998FAA8FBB8F80E090E0A8E4B4EC2B
:101800008C8F9D8FAE8FBF8F8DEC9CECACE4BEE3D4
:1018100088A399A3AAA3BBA3DF91CF911F910F9196
:101820000895682F8AE490E10C94FD0B91E0909369
:10183000B30D8093E1131092B40D1092D50D08955D
:10184000CF93C82F682F607F8CEC93E10E948412A5
:1018500080E1C89FB00111248CEC93E1CF910C94EE
:101860008412CF93DF9300D000D01F921F92CDB788
:10187000DEB798E0E3E6F5E0DE01119601900D9207
:101880009A95E1F79091D513961708F46FEF70E0F1
:10189000660F771F21E030E02C0F3D1F620F731F92
:1018A000FB019081890F806828960FB6F894DEBFFF
:1018B0000FBECDBFDF91CF910C94208C2F923F9221
:1018C0004F925F926F927F928F929F92AF92BF9250
:1018D000CF92DF92EF92FF920F931F93CF93DF93FC
:1018E00000D000D000D01F92CDB7DEB78090370D6A
:1018F0009090380D8091390D90913A0D8816990687
:101900002CF4382F292FC401832E922E0BE31DE0D7
:1019100027E83DE040E050E0BA01D801CD90DD90ED
:101920008D01C816D9060CF06DC0092E000CAA0B4B
:10193000BB0B480F591F6A1F7B1FC60120173107B9
:1019400061F7CB01BA010E9425B620E030E048E102
:1019500052E40E949DB86B017C01E7E3FDE0FA8749
:10196000E987812C912C5401A985BA856D917D91CF
:10197000BA87A987072E000C880B990B0E9425B601
:10198000A70196010E94BEB79B01AC010E9484B6DC
:101990009B01AC01C501B4010E94BFB74B015C01C2
:1019A000E985FA850E171F07F9F620E030E04CE1D3
:1019B00052E40E949DB80E94C7BA4B015C0120E02E
:1019C00030E040E85FE30E94A6B918168CF1C70129
:1019D000B6012A960FB6F894DEBF0FBECDBFDF91D9
:1019E000CF911F910F91FF90EF90DF90CF90BF901C
:1019F000AF909F908F907F906F905F904F903F90AF
:101A00002F9008958C149D0454F4092C000CAA08FE
:101A1000BB08480D591D6A1D7B1D46018FCF0D2C3B
:101A2000000CEE08FF084C0D5D1D6E1D7F1D86CF5E
:101A300087E3282E8DE0382E10E000E019821A820C
:101A40001B821C82D1018D919D911D019C01990FDA
:101A5000440B550B2D833E834F835887CA01B90130
:101A60000E9425B6A70196010E94BEB72B013C013A
:101A700020E030E0A9010E94A6B9181624F077FAF8
:101A8000709477F87094A5019401C301B2010E948B
:101A90001EB687FF12C089819A81AB81BC812D81DE
:101AA0003E814F815885820F931FA41FB51F8983E4
:101AB0009A83AB83BC830F5F1F4F49855A854215BC
:101AC000530509F0BFCF20E030E040EC5FE3C501F3
:101AD000B4010E9484B64B015C01053011050CF481
:101AE000A7CF69817A818B819C810E9425B66B0189
:101AF0007C01B801110F880B990B0E9425B69B0140
:101B0000AC01C701B6010E949DB86B017C015FCF9B
:101B10004F925F926F927F928F929F92AF92BF92FD
:101B2000CF92DF92EF92FF920F931F93CF93DF93A9
:101B300000D000D01F921F92CDB7DEB72B013C0121
:101B4000FF24F3940F2D10E0C801880F991F880F10
:101B5000991F9A838983FC01E95FFA4F8080918005
:101B6000A280B380A3019201C501B4010E941EB6F8
:101B700087FF02C0F394E6CFA981BA81A151BB4F80
:101B8000CD90DD90ED90FC90A3019201C501B401D0
:101B90000E941EB6882309F44DC00150104C000F5E
:101BA000111F000F111FF801E95FFA4F8081918129
:101BB000A281B38189839A83AB83BC8301511B4F7C
:101BC000D8018D919D910D90BC91A02D8D839E8308
:101BD000AF83B88729813A814B815C81C301B2010F
:101BE0000E94BEB72B013C012D813E814F8158855B
:101BF000C701B6010E94BEB79B01AC01C301B2018F
:101C00000E9484B66B017C0129813A814B815C8101
